:020000040800F2
:1040000000500020597D00082D7C0008317C0008FC
:10401000357C0008397C00083D7C00080000000069
:10402000000000000000000000000000457C0008C7
:10403000417C000800000000497C000805A700083A
:104040004D7C0008517C0008557C0008597C000814
:104050005D7C0008617C0008657C0008697C0008C4
:10406000000000006D7C0008717C0008000000006A
:104070000000000000000000000000000000000040
:104080000000000000000000917C0008957C000802
:10409000A57C0008B57C0008D17C000869460008B2
:1040A000E17C0008994A00080000000000000000C0
:1040B00075470008A546000849470008E57C000848
:1040C00021BF0008ED7C00089DBF0008F57C0008BA
:1040D000F97C0008FD7C0008E5450008D145000892
:1040E000097D00080D7D0008117D0008000000001A
:1040F00000000000000000000000000000000000C0
:0C41000000000000000000005FF800005C
:10410C0030BF704720BF704740BF7047BFF36F8F01
:10411C007047BFF34F8F7047BFF35F8F704701DF5E
:10412C007047EFF31480704780F31488BFF36F8FE0
:10413C007047EFF30980704780F309887047EFF3FD
:10414C000880704780F30888704772B6704762B673
:10415C00704771B6704761B6704780F3118870472D
:10416C00EFF31280704740BA704700BA70470000F6
:10417C00054A0649064B1160064A1360064A13604D
:10418C00064A1360704700BFCC040020A1930008BE
:10419C0059920008A804002078030020A0040020F5
:1041AC00064A074B1A60074A074B1A60074A084B26
:1041BC001A60084A084B1A60704700BF5DB70008C8
:1041CC007803002069B90008CC0400205DB9000810
:1041DC00A004002059B70008A8040020044B054A8D
:1041EC001360054A1360054A1360054A1360704753
:1041FC005992000878030020A8040020CC04002069
:10420C00A0040020704700BF704700BF30B597B0C6
:10421C0003F0ACFA03F0CAFA0AF024FD6F4B002449
:10422C004FF480301C700AF03DFD0AF0A1FE01280D
:10423C0032D10F300BF0D4FB02200BF0B9FB20462F
:10424C000AF080FD20460AF091FD4FF480600AF0E0
:10425C0083FD634B634A1B68934202D14FF4403099
:10426C0004E0614A934205D14FF480304FF4E011E1
:10427C000AF044FD01200AF04DFD39200AF062FEDF
:10428C000028FAD002200AF04BFD0AF053FD082852
:10429C00FBD1524B01221A70012001460AF008FE94
:1042AC004FF000604FF480410AF064FF4FF440700F
:1042BC000AF0C2FE4D4B1B78552B0ED14C4B1B7884
:1042CC00532B0AD14B4B1B78422B06D1FFF750FFD7
:1042DC00494B01221A70013A05E0FFF761FF464B8A
:1042EC0000221A700132454B454C1A7005F08CFABD
:1042FC0005F0C4FA07F060FD03F0E0FE06F0DEF90D
:10430C002046404905F066FD05F092FA3E4B1B78BD
:10431C00012B05D1207804F04DFDE07804F05AFC17
:10432C00354B1B78012B25D1384C0DF1100C254643
:10433C000FCDACE80F00AE46BEE80F00ACE80F00A6
:10434C009EE80F0030340DF1400E8CE80F000FCCBE
:10435C00AEE80F0094E8030005248EE803000094F7
:10436C0004AC0194042010AC294902221C230294B1
:10437C0005F0D4F8214B1B78012B05D1204B1A6981
:10438C005879996807F0F0FA00F04CF800F042F810
:10439C0000F0F8FC01F0D0F903F0D4F940F21670FB
:1043AC0006F03AFC40F2127006F094FC03F038FB75
:1043BC0003F0A6FA00F04CF820B902F0C7FE01F0A9
:1043CC0001F804E0012002F0C1FE00F069FD03F0E9
:1043DC00BBF906F057FC00F0C9FBE9E7B804002074
:1043EC005C0000200024F40000127A00FC3F00085E
:1043FC00FD3F0008FE3F000818000020510000207F
:10440C00D0040020E40300204E000020240E0108FC
:10441C0000080140024B00225A601A70704700BF1E
:10442C00A0010020084A094B12680021D20283F82F
:10443C002C109A629A605A611A62DA609A615A6216
:10444C001A61DA61704700BF14000020A00100203F
:10445C00014B93F82C007047A0010020014B186B06
:10446C00704700BFA0010020014B586B704700BF84
:10447C00A0010020014B1868704700BF30090020D4
:10448C00014B986B704700BFA001002008B5024B90
:10449C0018680CF09BFC08BD68090020014BD86B18
:1044AC00704700BFA0010020014B1868704700BF87
:1044BC0084090020014B1868704700BF38090020A0
:1044CC00014B1868704700BF40090020034B93F85C
:1044DC00422022EA000283F842207047E4030020C5
:1044EC00034B93F8423018420CBF00200120704758
:1044FC00E4030020034B93F8512040EA020283F8B6
:10450C0051207047E4030020034B93F8512022EA1A
:10451C00000283F851207047E4030020034B93F80A
:10452C00513018420CBF002001207047E4030020DA
:10453C00014B1868704700BF54090020014B1868E4
:10454C00704700BF1C090020014B5868704700BF22
:10455C001C090020014B1868704700BF6C09002033
:10456C00014B5868704700BF6C09002008B501204A
:10457C00FFF7D4FF48B1054B00220420DA63FFF7A4
:10458C00CDFF10B10120FFF7BFFF08BDA001002037
:10459C0008B506F091FD08BD08B506F0F1FB08BDA5
:1045AC0008B54FF4803005F003F908BD08B5044B8D
:1045BC0093F860301BB94FF4003005F0F9F808BDE2
:1045CC00E403002008B5034B1B78012B01D104F048
:1045DC0039FB08BD4F00002008B5034B1B78012B9D
:1045EC0001D104F08BFB08BD4502002008B5022068
:1045FC00FFF776FF38B1044BB3F8400006F08EFDA0
:10460C000220FFF763FF08BDE403002010B5012072
:10461C00FFF766FFD8B106F08FFD0D4991F82530F4
:10462C00CA6B5B08B2FBF3F3B0FBF3F202FB1303B0
:10463C00084AA1F84030147834B9074B4031186857
:10464C000222403005F0A4FA0120FFF73FFF10BD15
:10465C00E40300204A0200200400002008B54FF4B7
:10466C0080700BF02FFA88B14FF480700BF038FA91
:10467C00074B1B78012B03D0064B1B78012B05D164
:10468C00FFF7C4FFFFF7B2FFFFF770FF08BD00BFD5
:10469C004C0000204302002008B5044B1978012976
:1046AC0003D1034B186809F081FF08BD4C000020B2
:1046BC004800002038B51D4C0221206809F070FF1D
:1046CC00012827D10221206809F070FF002003F097
:1046DC00ABF9174C0546014694F8400006F018FB60
:1046EC00144B84F8405093F8212080B2062A11D143
:1046FC00E26B01B28A18E26360B193F861304BB19E
:10470C000D4B9A6812F0200F02D020225A6101E062
:10471C0020221A61054C0121206809F041FF012873
:10472C00014602D1206809F041FF38BD400000204D
:10473C00A0010020E40300200010014008B5074B45
:10474C001978012903D1064B186809F02FFF054B86
:10475C001B78012B01D1FFF7ADFF08BD43020020F0
:10476C00480000204400002008B5074B19780129A7
:10477C0003D1064B186809F019FF054B1B78012B68
:10478C0001D1FFF797FF08BD42020020480000202E
:10479C004102002038B5244B93F82120072A25D05C
:1047AC00082A39D0062A3DD1204A0128D36B1F4D47
:1047BC0008BF536401286A6C1D4C6B6402D1AB6C4E
:1047CC0023602FE09B1A184A206892F825104EF6A9
:1047DC0060225343490806225143223293FBF1F1E4
:1047EC0007F0D6FE20602368AB641BE001280F4A5B
:1047FC000F4C02D1D36C23600AE00E490868D96BC8
:10480C004EF66023434393FBF1F323602368D36498
:10481C00084B00221A6005E0074B18680CF0D6FA1A
:10482C00034B186038BD00BFE4030020A00100203A
:10483C0038090020800900206809002010B50446C2
:10484C004FF4804004F0B4FF034B0120DC639C6305
:10485C00FFF7A0FF10BD00BFA001002008B5034862
:10486C0004F09CF9024804F099F908BD1C090020D9
:10487C0054090020B0F5007F10B5044610D003DCBD
:10488C00B0F5807F37D121E0B0F5806F03D0B0F563
:10489C00006F30D10DE004F083FF4FF4807019E00D
:1048AC0004F07EFF4FF4807004F082FF4FF48060C0
:1048BC0014E004F075FF4FF4807004F079FF4FF4AE
:1048CC00806004F075FF4FF400700BE004F068FF9B
:1048DC004FF4806004F06CFF4FF4007004F068FF3C
:1048EC004FF4006004F064FF4FF4804004F060FF6C
:1048FC00024BA3F86240024B1C6010BDE403002085
:10490C003C09002010B504464FF4803004F058FFE9
:10491C00012808D0044B4FF400601C60FFF7AAFF7D
:10492C00024B00221A6010BD4409002068090020C7
:10493C0038B505464FF4803004F042FF01281CD0F6
:10494C000E4B4FF480601C680D4B9D63FFF792FF7C
:10495C004FF4804004F02CFFB4F5007F04D1094BD8
:10496C001A68094B1A6008E0B4F5006F05D1074BC3
:10497C0018680CF011F8044B186038BD3C09002085
:10498C00A00100206809002000090020380900203F
:10499C0008B5034BDB6BC018FFF7CAFF08BD00BF9F
:1049AC00A001002038B505464FF4803004F008FF14
:1049BC0001281AD00D4B4FF400701C680C4B1D6075
:1049CC00FFF758FFB4F5006F05D10A4B18680BF0D0
:1049DC00E3FF094B1860094B9B6813F4004F04D19B
:1049EC0004F008FF08B902F04FFF38BD3C09002065
:1049FC0084090020380900206809002000100140BB
:104A0C0008B54FF48070FFF735FF08BD38B51A4B69
:104A1C001B78012B02D106F055FB03E0174B1868ED
:104A2C0009F0B6FD164B0422D96B91FBF2F29042C1
:104A3C000ADA4FF0030C0CFB02FC124B1B6D6345A6
:104A4C0002DDCB1A1B180DE003235343984206DDFD
:104A5C000C4B1B6D934202DAC31A5B1A02E0094B32
:104A6C001B6DC31A074A0849D46B0D68E41AEB1A7C
:104A7C000B601065D46338BD4A020020480000204A
:104A8C00E4030020A00100208009002008B5224B7F
:104A9C001B8813F0100F31D1204A214B1068596D2F
:104AAC00013010601A780131012A596503D11D4B70
:104ABC004FF400521A611C4B93F82130072B08D18C
:104ACC001A4B1B78012B01D106F012FB0120FFF7CA
:104ADC009DFF154B93F82130082B05D1134B1B78F8
:104AEC00012B01D106F004FB0D4B5A6D132A0DD985
:104AFC00002210465A65FFF74DFE07E0094B4FF4B4
:104B0C0000520B4801215A610BF05AFC024801215A
:104B1C0009F04CFD08BD00BF002C01401809002015
:104B2C00A001002000100140E40300204A020020F4
:104B3C000024014008B502F0B7FEA0B904F05AFEFB
:104B4C0088B900F5005004F03BFE60B900F58070A8
:104B5C0004F036FE38B9044B4FF461729A861A870A
:104B6C009A8702F091FE08BD002C014010B505F0AB
:104B7C009FFD204CA36DC31A002BB8BF5B42B3F54D
:104B8C007A7F36DD1C4B9B6813F4006F2AD102F040
:104B9C008BFE60B1012004F003FE402004F000FE07
:104BAC0094F85C300A2B02D8013384F85C304FF453
:104BBC00807004F005FE20B9FFF7F4FE0F4B0022C5
:104BCC001A6002F071FE80B10A4B93F85C300A2B2C
:104BDC000BD8094B4FF480621A6140205A6104F0E3
:104BEC00E7FD02E0002384F85C3005F061FD014B29
:104BFC00986510BDA001002000100140680900203C
:104C0C0010B505F055FD194C236EC31A002BB8BF17
:104C1C005B42642B28DD164B186803F0BFF8154B6C
:104C2C00206393F82B30012B0AD103F55A63984279
:104C3C0006DD02F031FE042004F0B2FDFFF7E0FEC9
:104C4C000A4B1B6BB3F57A7F02DC022004F0A8FD43
:104C5C00064B1B6BB3F57A7F02DD022004F0A8FD36
:104C6C0005F026FD014B186610BD00BFA001002009
:104C7C0038000020E403002010B505F019FD264C87
:104C8C00636EC31A002BB8BF5B42B3F57A7F42DD6B
:104C9C00224B186803F082F86063082004F090FD42
:104CAC00B8B9636B40F6B322934209DD083004F0C7
:104CBC0077FD02F027FE02F0EFFDFFF7A1FE26E0E4
:104CCC00B3F5156F0ADC082004F072FD02F020FE2B
:104CDC0009E0626B40F60B239A4218DC082004F0C2
:104CEC0067FD02F01BFE0E4B9B6813F4004F0ED1B8
:104CFC0004F080FD58B900F5005004F061FD30B9A6
:104D0C0000F5807004F05CFD08B902F0BDFD05F003
:104D1C00CFFC014B586610BDA00100203C000020C8
:104D2C000010014008B5054A0346022093FBF0F041
:104D3C0080B282F8253006F07DF908BDE40300202E
:104D4C0010B50C4C23789BB90B4B4FF400611868D1
:104D5C0003F02CF8094B4FF40061186803F026F8A7
:104D6C00074B4FF40061186803F020F801232370FF
:104D7C0010BD00BFA00100203C020020300000202C
:104D8C003400002010B502F097FD012003F046F826
:104D9C00334C344803F002FF334803F0FFFE05F0B8
:104DAC00B5FD94F82130062B0ED14FF4004004F0E1
:104DBC00F7FC802004F0FCFC012006F059F894F874
:104DCC002500400806F01AF8254C94F82130072BE2
:104DDC0020D14FF4004004F0EBFC802004F0E8FC00
:104DEC0094F82A30012B02D1002006F041F81C4C1B
:104DFC00E06B94F82C1006F015FA94F82510E06B83
:104E0C00490806F023F906F031F903F0CDFA012038
:104E1C0006F032F9124C94F82130082B11D14FF4D2
:104E2C00004004F0C5FC002006F022F8E06B94F87A
:104E3C002C1006F0F7F994F82510E06B490806F0F1
:104E4C0005F90A4C4FF400730120236102F0ECFFCA
:104E5C004FF48043236102F017FDFFF771FF10BD83
:104E6C00E40300201C0900206C0900200010014004
:104E7C0038B5094C094D94F8682095F821309A42C0
:104E8C0008D0FFF77FFF0120FFF784FC95F8213055
:104E9C0084F8683038BD00BFA0010020E403002076
:104EAC002DE9F04190B005F003FC554C0646E36E3D
:104EBC00C31A002BB8BF5B42B3F57A7F0DDB00251C
:104ECC00206F04F0A1FB606F256704F0A3FBA06FBB
:104EDC00656704F0A5FBE666A5674A4A484B11686E
:104EEC00494A186F12690029B8BF49420130002A9B
:104EFC00B8BF52429142186703DC102004F050FCFA
:104F0C0002E0102004F054FCFFF7B2FF3E4DFFF717
:104F1C0077FEFFF7B1FE3D4BAA6919689142C0F0CC
:104F2C00B680374C0021A26F4FF40040013219605B
:104F3C00A26704F045FC012834D14FF4806004F0E2
:104F4C003FFC01282ED1A16B314BE26B284603F0BC
:104F5C0005FE304B186004F0A3FB60B104F00EFCAE
:104F6C00022808D1A26BE36B0E920F930EAB93E861
:104F7C00030004F0B1FB224A234B906BD16BDA682F
:104F8C00411A0029B8BF494291420BDC1D4A9B686B
:104F9C001268002AB8BF52429A4203DC4FF4804098
:104FAC0004F0FEFB184C94F82030012B38D14FF450
:104FBC00806004F005FC01280DD1114A1649D36B11
:104FCC00956B144A20461268009503F053F90BF0C8
:104FDC00E3FC124B18604FF4007004F0F1FB012855
:104FEC0029D10E4C20680BF0F1FE0A4B01461A68D1
:104FFC00054803F009F90BF0CFFC20601BE000BF63
:10500C00A001002038090020E403002088090020BA
:10501C0054090020840900200009002068090020A0
:10502C00924B216818680A46494207F091FA0BF036
:10503C00B3FC8F4B18604FF4007004F0C1FB0128D7
:10504C0005D04FF4806004F0BBFB01281FD1884DC4
:10505C00884C28680BF0BAFE26680146864B32460F
:10506C00864803F02FFD864B186004F019FB70B1D5
:10507C0004F084FB01280AD128680BF0A7FE2368F2
:10508C000E900F930EAB93E8030004F025FB7D4EBE
:10509C007A4B3168DA699142C0F065817A4F1A8D8A
:1050AC007B6F4FF0000EC6F800E003F1010C3E26BA
:1050BC00C7F874C00AAC0096744D06F5D276C821B8
:1050CC004B23204601964FF40266029602F042FFF3
:1050DC0094E8070085E807004FF4806004F070FB4B
:1050EC0001280BD04FF4007004F06AFB012805D0A6
:1050FC004FF4006004F064FB012840D15D4B624D1D
:10510C00D3F80080614A594B05F17C0E6F4607CAF3
:10511C00D3F800C087E80700CDF810E0DFF888E18D
:10512C00574ECDF814E0DFF848E1534B534858493B
:10513C00584A594CCDF818E0CDF81CC0CDF8208059
:10514C00039603F077F9B5F97C20B5F97E10336836
:10515C00524D8918206810222B6007F019FA206034
:10516C0004F09EFA58B104F009FB40B923682A6890
:10517C000F930E920EAB93E8030004F0ADFA464B7E
:10518C003E4D1868294605F0E9FC05F021FD6B6DD4
:10519C00984228D905F08CFA3B4CD4F88030C31ACD
:1051AC00002BB8BF5B42B3F57A7F1CDB05F0CEFC5D
:1051BC004FF4003004F0F4FA95F8603063B9384BD2
:1051CC0029461868012201F8602F603004F0E0FCD9
:1051DC0005F06EFAC4F8840005F00CFD05F068FAD1
:1051EC00294BC3F8800005F063FA274B2349D3F809
:1051FC0084208B6D821A002AB8BF52429A420BD37C
:10520C0091F86020012A07D1254B1868002301F87A
:10521C00603F603004F0BCFC184B93F86030012BFD
:10522C0003D14FF4003004F0BBFA4FF4003004F01B
:10523C00C7FA012808D1104803F0B0FC194803F054
:10524C00ADFC0020FFF75EFB02F05CFE124B1A680F
:10525C000A4B002A5B68B8BF52429A4226DD0120F5
:10526C0004F09EFA02F068FB25E000BF84090020E0
:10527C0068090020380900201C090020E4030020E4
:10528C004409002018090020A00100204809002032
:10529C006C0900200409002040090020300900207E
:1052AC00040000205409002000090020012004F013
:1052BC007FFA02F049FB2D4BDB790BB102F0B2FB0C
:1052CC002B4B93F8222012F0010F22D0294A12689E
:1052DC00002A1EDD93F8233013F0010F03D00020B9
:1052EC0002F04AFB40B9224B93F8230010F0010066
:1052FC000FD102F041FB60B90220FFF70FF910B19A
:10530C001D4B0022DA630020FFF74CFB1B4B0022E5
:10531C001A60174B93F8222012F0020F23D0154A73
:10532C001268002A1FDA93F8233013F0020F03D00F
:10533C00012002F021FB48B90D4B93F8233013F0F8
:10534C00020F10D1012002F017FB60B90220FFF709
:10535C00E5F810B1084B0022DA630020FFF722FBBE
:10536C00064B00221A6010B0BDE8F081D00400207A
:10537C00E403002038090020A00100206809002067
:10538C000A4938B5CC6B00238C630949094D0B6075
:10539C00094900220A602A60084A094D01202B6045
:1053AC001360FFF7F7F9FFF7EDFC38BDA001002003
:1053BC008409002068090020000900203009002021
:1053CC00440900202DE9F041534B93F82C2014464E
:1053DC00002A40F09E805A68254601325A60012D01
:1053EC0005D0022DDFF83C8108D04C4B07E04C4B2C
:1053FC00186802F0D3FC4B4B1F6805E04A4B186849
:10540C0002F0CCFCD8F800704743484B1A5997422D
:10541C0001D901321A51464B1A59974201D2013A1D
:10542C001A51434B03F10C021E5912591833B6187A
:10543C001B5976089E4201D95E1C01E038BF5E1EE6
:10544C00012D09D0022DDFF8DC800CD0D8F800102B
:10545C00324BB6FBF1F10BE0324B1968304BB6FB1B
:10546C00F1F1186805E0D8F800102F4BB6FBF1F1FC
:10547C00186802F09BFC2E4B2E491A590E51BA4259
:10548C0001D201321A51294B1A59BA4201D9013AA7
:10549C001A5101350434032DA1D1224B4FF47A72E9
:1054AC001B6853431C4A52689A4232DB1B4B1868E8
:1054BC0002F084FC1A4B0546186802F07FFC1A4B6C
:1054CC00A5F5F26504460D3D186802F077FCC62D73
:1054DC0009D8A4F5F2640D3CC62C04D8A0F5F260F2
:1054EC000D38C62811D90D4B4FF40061186802F025
:1054FC005DFC0B4B4FF40061186802F057FC0A4B33
:10550C004FF40061186802F051FC034B012283F840
:10551C002C20BDE8F08100BFA00100203C0200203F
:10552C00300000201400002034000020B4010020C2
:10553C00A8010020C001002010B5104B5B788BB97E
:10554C000F4A012091780F4A14680F4A10700F4AC5
:10555C0011700133E21812F8011C0C4A082B9954F3
:10556C00F7D10AE0012B08D1094B07221A71013A35
:10557C00DA7158329A7102225A7110BD6C030020F4
:10558C00D004002024000020D4030020D8030020E5
:10559C00C0040020044B5A6840F2D2439A4202D114
:1055AC00024B01221A7070476C0300208C090020FA
:1055BC0010B51C4A1C4B116801EA03031B498B42B2
:1055CC002ED152681A4B9A422AD102F065F9194B26
:1055DC001B78012B10D103F051FF05F069F804463C
:1055EC0001E002F08DF905F063F8001B0028B8BF4C
:1055FC004042B0F57A7FF4DB04F008F909F0EAFCDC
:10560C00002009F06FF900210B480AF00FFB0A4843
:10561C000AF06CFA09480BF013F8002004F000F9BA
:10562C0010BD00BF6C03002000FFFF000081920042
:10563C00D6C5B4A318000020080002400024014085
:10564C0010B5164B9A78012A08D003D3022A144CB1
:10565C000FD109E0587802F08FF902E0587802F087
:10566C00F9F90F4B586006E0587802F095F9606034
:10567C0001E0042323700B4B1B786BB1084B0A49D8
:10568C005A680A4B0A601AB91A6842F0080202E01A
:10569C001A6822F008021A6010BD00BF6C030020CB
:1056AC00C0040020A4040020D003002074030020B8
:1056BC0008B5104B9A78012A02D0022A16D10CE0B8
:1056CC005A7842B9586810B904F0A2F811E01046A3
:1056DC0004F0A2F80DE0032209E05A68587812B9D8
:1056EC0002F03AF905E002F03FF902E00422024B25
:1056FC001A7008BD6C030020C004002008B50B4BC9
:10570C009A78022A0ED15B78372B09D89B0008496E
:10571C0003F5E260C9180A30023204F0B7F804E06D
:10572C00032200E00422034B1A7008BD6C03002016
:10573C00FC040020C0040020144A00231360144A07
:10574C0010B51360134A1360134A1360134A137095
:10575C00134A002199500433B3F5806FF8D1114BE3
:10576C001B7E63B940F21A740F49204609190422B2
:10577C0004F08CF8043440F2FA739C42F4D1094AD8
:10578C000A4B527D02B101221A7010BD6C0400202C
:10579C00D0030020F80400207403002068030020CC
:1057AC00FC040020D0040020E2FDFF1FAC0400200C
:1057BC0008B5124B9A7812B1022A1AD10AE05B781A
:1057CC004E2B14D10E4B18680E4B0730D97904F0C0
:1057DC0081FA11E05B78372B09D89B000A4903F555
:1057EC00E260C9180A30042204F0D2F904E0032262
:1057FC0000E00422054B1A7008BD00BF6C030020AA
:10580C009C010020D0040020FC040020C0040020D7
:10581C0008B5604B9A781AB1022A40F0A68099E03C
:10582C005B78502B69D01FD8462B51D00ED8422B09
:10583C0043D005D8402B37D0412B40F089803AE03B
:10584C00442B40D0544B554A40D83AE04B2B48D0CF
:10585C0004D8472B3FD0492B7AD13FE04D2B46D073
:10586C0042D34E2B74D145E0812B5AD00ED8532BFA
:10587C004CD004D8512B43D0522B69D143E05A2B36
:10588C004AD0802B4BD0552B62D142E0842B53D085
:10589C0004D8822B4CD0832B5AD14BE0FE2B4ED00C
:1058AC0050D8F02B54D14AE03D4B186804F03CF82A
:1058BC00394B58605CE0394B42E0384B5A78364BE8
:1058CC004FE012794DE0354BDA69F8E7527948E050
:1058DC00324BDA68F3E7314B9A68F0E72F4BDA7DFD
:1058EC0032E02E4BDA78EAE72C4B9A78E7E72B4B31
:1058FC005A7DE4E7294BDA79E1E7284B9A7DDEE71C
:10590C00264B1A7DDBE7254B1A6AD8E7234B1A691D
:10591C00D5E7224B1A7ED2E7204B5A6ACFE7214BB0
:10592C000EE0204B1A78042A14BF00220122C6E78D
:10593C001D4B02E01D4B00E01D4B1A68BFE71D4BD1
:10594C001A78BCE71C4B1A78003A18BF0122B6E74C
:10595C0003220BE05A78104B372A04D8174951F818
:10596C0022205A6004E0032201E004220A4B1A7040
:10597C00134B1B786BB1084B12495A68124B0A60D7
:10598C001AB91A6842F0080202E01A6822F00802FA
:10599C001A6008BD6C030020C0040020D004002055
:1059AC000C000020AC0400206C04002094090020A2
:1059BC0090090020B80400209C040020FC04002066
:1059CC00A4040020D00300207403002010B58A4BDF
:1059DC009A781AB1022A40F0238104E15A784C2AB1
:1059EC0000F09E801ED8442A60D00CD8412A44D0A6
:1059FC0003D8402A40F012813BE0422A46D0432A89
:105A0C0040F00C814AE0472A68D005D8452A55D089
:105A1C00462A40F0038159E0492A67D04B2A40F0CE
:105A2C00FD8070E0532A00F0B38010D8502A00F0AB
:105A3C008B8005D84D2A7BD04E2A40F0EF807FE03A
:105A4C00512A00F08980522A40F0E88098E0832A9D
:105A5C0000F0BD8006D8552A00F0A2805A2A40F0EA
:105A6C00DD80A9E0842A00F0B680FF2A40F0D680C1
:105A7C00B6E01979614B186805E0614A1B7910682A
:105A8C00604A1946137004F025F9CCE05C4A1B7986
:105A9C0010685C4A013019465370F4E7584A1B7978
:105AAC001068584A043019461371ECE7544A5B6885
:105ABC00106854491C3041F81C3F84E0504A1B7953
:105ACC001068504A053019465371DCE74C4A5B6844
:105ADC0010684C490C3041F80C3F74E0484A5B6844
:105AEC0010684849083041F8083F6CE01A79454B7A
:105AFC0012B1454901224A60DA75414B1868414B95
:105B0C001730D97DBFE73E4A1B7910683D4C0330F6
:105B1C001946E37004F0DEF8E07803F05BF882E0FD
:105B2C00374A1B791068374A023019469370AAE736
:105B3C00334A1B791068334A153019465375A2E75E
:105B4C001A79304BDA716EE02D4A1B7910682D4AA8
:105B5C0016301946937596E72A4A127D12F0010FFA
:105B6C0005D01B7913F0010F01D103F06FFF244A0C
:105B7C00214B10681B79234A14301946137582E7A0
:105B8C001F4A5B6810681F49203041F8203F1AE01B
:105B9C001B4A5B6810681B49103041F8103F12E03B
:105BAC005A68012A3CD8164A1B79106815491830D6
:105BBC0001F8183F012207E0114A5B68106811498F
:105BCC00243041F8243F042203F0E2FF2BE00E4B7B
:105BDC005A680E4B02E00C4B5A680D4B1A6022E0CF
:105BEC001A790C4B1EE05A78372A17D859680A4B89
:105BFC0043F8221017E000BF6C0300200C000020BB
:105C0C009C010020D0040020C00400209409002036
:105C1C00900900209C040020FC040020032200E0DA
:105C2C000422014B1A7010BDC004002008B50020DE
:105C3C00FEF7B8FE08BD00BF08B5024B5868FEF76A
:105C4C00B1FE08BD6C03002008B5034B58684042F8
:105C5C00FEF7A8FE08BD00BF6C03002008B5AC4BD6
:105C6C009A78002A41F075805A78AC2A00F0EB84BF
:105C7C006BD81E2A00F0AF8230D8092A00F09C8124
:105C8C0013D8032A00F0078105D8012A00F0DB8025
:105C9C0000F2E780C9E0062A00F02881072A00F00C
:105CAC005F81042A41F05380FBE0192A00F0108236
:105CBC0008D80B2A00F0D781C0F0A9810D2A41F039
:105CCC004680FCE11B2A00F04A82C0F024821C2A88
:105CDC0000F04B821D2A41F03A8075E29B2A00F0BD
:105CEC00308317D8922A00F0E68209D8852A00F072
:105CFC008C82862A00F0B4821F2A41F028807DE233
:105D0C00972A00F01283982A00F01583962A41F006
:105D1C001E8004E3A22A00F0968309D89F2A00F083
:105D2C002F83A12A00F05A839C2A41F0108021E392
:105D3C00A42A00F00484C0F0CD83A52A00F02B84A3
:105D4C00A62A41F0048000F054BCD32A00F0C6858A
:105D5C0031D8C22A00F0608515D8BE2A00F02885FB
:105D6C000AD8B12A00F0BE84B22A00F0F884AD2A19
:105D7C0040F0ED8700F08EBCC02A00F0338500F2B5
:105D8C003E8500F022BDC62A00F07A8506D8C42ACA
:105D9C0000F05C8500F2678500F04BBDC82A00F06E
:105DAC008985C0F07A85C92A00F08A85D22A40F00C
:105DBC00CE8700F08CBDF12A00F03D8619D8E52A7B
:105DCC0000F0A9850AD8E22A00F09785E42A00F0B1
:105DDC009B85D42A40F0BB8700F087BDEA2A00F0EF
:105DEC00C985EB2A00F0FF85E62A40F0B08700F069
:105DFC0099BDFA2A00F0C5860AD8F52A00F07086FB
:105E0C00F92A00F09486F42A40F0A18700F03EBEF7
:105E1C00FC2A00F02487C0F0DE86FD2A00F04887BB
:105E2C00FE2A40F0948700F06CBF052805D1384B52
:105E3C005868FEF77DFD00F0A3BF062840F0A08750
:105E4C00FEF71EFB40E1052805D1314B5868FEF7E3
:105E5C00F5FC00F095BF062840F09287FEF71EFB7C
:105E6C0032E1052811D12A4B2A4A586800F54233F1
:105E7C0003F5A863934203D8FEF794FD00F080BFAE
:105E8C00254B04221A7000F07BBF062840F078875F
:105E9C00FEF70AFB18E1062840F07287FEF70AFBB2
:105EAC0012E105280AD11A4B1C495B688B4295BF3D
:105EBC001B4A194B13601A7000F062BF062802D1FE
:105ECC00174B1A6810E2072806D1164B14491868AC
:105EDC0003F05EFE00F054BF082840F05187114BD0
:105EEC000F49186803F0D2FC00F04ABF05281BD1FB
:105EFC00074B43F698225B68934203D8084A5360D9
:105F0C0000F03EBF044B04221A7000F039BF00BFF2
:105F1C006C030020801A0600C0040020400D030012
:105F2C00E403002004000020062802D1994B5A6893
:105F3C00DAE1072808D1984B042218689749801891
:105F4C0003F026FE00F01CBF082840F01987924B86
:105F5C00042218689149801803F098FC00F010BFD7
:105F6C0005280DD18E4B8F4A5B68934203D8894A22
:105F7C00936000F005BF8C4B04221A7000F000BF38
:105F8C00062802D1834B9A68AEE1072808D1824BD0
:105F9C00864918680422083003F0FAFD00F0F0BEC0
:105FAC00082840F0ED867C4B8049186804220830A4
:105FBC0003F06CFC00F0E4BE05280CD15B68794A58
:105FCC00934203D8734A136100F0DABE764B042275
:105FDC001A7000F0D5BE062802D16E4B1A6983E107
:105FEC00072808D16C4B724918680422103003F052
:105FFC00CFFD00F0C5BE082840F0C286664B6C4948
:10600C0018680422103003F041FC00F0B9BE0528DA
:10601C000DD1634B674A5B68934203D85D4AD360EA
:10602C0000F0AEBE604B04221A7000F0A9BE062828
:10603C0002D1584BDA6857E1072808D1564B5E4914
:10604C00186804220C3003F0A3FD00F099BE082858
:10605C0040F09686504B5849186804220C3003F0D7
:10606C0015FC00F08DBE05280DD14D4B514A5B68D7
:10607C00934203D8474A536100F082BE4A4B042234
:10608C001A7000F07DBE062802D1424B5A692BE1F2
:10609C00072808D1404B494918680422143003F0F2
:1060AC0077FD00F06DBE082840F06A863A4B4349F4
:1060BC0018680422143003F0E9FB00F061BE0628D6
:1060CC0040F05E86FEF7E2F9374B586000F046BEB2
:1060DC00052804D15A682F4B9A6500F051BE06284A
:1060EC0002D12C4B9A6DFFE0072808D12A4B34497A
:1060FC0018680422583003F04BFD00F041BE08280C
:10610C0040F03E86244B2E4918680422583003F088
:10611C00BDFB00F035BE052805D1214B5A681D4B3F
:10612C005A6500F02DBE062802D11A4B5A6DDBE0E1
:10613C00072808D1184B234918680422543003F05F
:10614C0027FD00F01DBE082840F01A86124B1D4991
:10615C0018680422543003F099FB00F011BE062895
:10616C0040F00E8604F034FDAEE7052805D10C4B4B
:10617C00586804F039FD00F003BE062802D104F083
:10618C002DFDA1E7072840F0FB8504F033FD00F05E
:10619C00F7BD00BFE403002004000020E80300204A
:1061AC006C030020400D0300C0040020EC03002011
:1061BC00F4030020A0860100F0030020F803002067
:1061CC003C04002038040020052840F0C585FEF76B
:1061DC00EDF900F0D5BD052804D1586804F034FD64
:1061EC0000F0CEBD062802D104F028FD6CE707288C
:1061FC0040F0C68504F02EFD00F0C2BD052840F02D
:10620C00AB85FFF7BDF800F0BBBD05280CD1A24B48
:10621C005B680A2B03D8A14A936100F0B1BDA04B77
:10622C0004221A7000F0ACBD062802D19B4B9A696F
:10623C005AE0072808D19B4B9B4918680422183058
:10624C0003F0A6FC00F09CBD082840F09985954B06
:10625C00954918680422183003F018FB00F090BD23
:10626C0005280CD18C4B5B680A2B03D88B4AD36165
:10627C0000F086BD8A4B04221A7000F081BD0628FE
:10628C0002D1864BDA692FE0072808D1854B874964
:10629C00186804221C3003F07BFC00F071BD082848
:1062AC0040F06E857F4B8149186804221C3003F046
:1062BC00EDFA00F065BD05280ED15B68012B06D800
:1062CC00754B1A79754B83F8202000F059BD744B2F
:1062DC0004221A7000F054BD062809D16F4B93F8B4
:1062EC002020003A18BF01226D4B5A6000F036BDD9
:1062FC00072808D16B4B6E4918680122203003F037
:10630C0047FC00F03DBD082840F03A85654B6849D4
:10631C0018680122203003F0B9FA00F031BD0628CC
:10632C0040F02E85FEF7CCF8CEE6062840F0288506
:10633C00FEF794F8C8E6062840F02285FEF794F89C
:10634C00C2E6052810D1586847F2305200F56A535E
:10635C001833934203D8FEF7D5FA00F011BD504B19
:10636C0004221A7000F00CBD062840F00985FEF7D7
:10637C0081F8A9E6062840F0038503F031FAA3E67C
:10638C0005280ED1444B5B689A1F022A04D8434A55
:10639C0082F8213000F0F4BC414B04221A7000F05A
:1063AC00EFBC062803D13D4B93F821209CE707282E
:1063BC0008D13C4B3F4918680122213003F0E8FB1F
:1063CC0000F0DEBC082840F0DB84364B39491868F5
:1063DC000122213003F05AFA00F0D2BC052813D167
:1063EC002D4A2E4B52683AB193F8512042F00102DB
:1063FC0083F8512000F0C4BC93F8512022F0010224
:10640C0083F8512000F0BCBC062805D1234B93F82F
:10641C00512002F0010267E7072808D1214B2649D9
:10642C0018680122513003F0B3FB00F0A9BC082816
:10643C0040F0A6841B4B204918680122513003F010
:10644C0025FA00F09DBC052812D15A68134B3AB1BD
:10645C0093F8512042F0020283F8512000F090BCD6
:10646C0093F8512022F0020283F8512000F088BCEE
:10647C00062805D1094B93F85120C2F3400233E7AB
:10648C0007281BD1074B0C4918680122513003F027
:10649C007FFB00F075BC00BF6C030020E403002000
:1064AC00C004002004000020FC0300200004002095
:1064BC00040400200504002035040020082840F0C6
:1064CC005F84924B924918680122513003F0DEF937
:1064DC0000F056BC052813D18E4A8F4B52683AB146
:1064EC0093F8512042F0040283F8512000F048BC8C
:1064FC0093F8512022F0040283F8512000F040BCA4
:10650C00062805D1844B93F85120C2F38002EBE6A8
:10651C00072808D17D4B7E4918680122513003F0C1
:10652C0037FB00F02DBC082840F02A84774B7849C3
:10653C0018680122513003F0A9F900F021BC05289C
:10654C000ED1744B5A68032A05D81A79724B83F80A
:10655C00222000F015BC714B04221A7000F010BC04
:10656C00062803D16C4B93F82220BDE6072807D1EF
:10657C00664B6B4918680122223003F009FBFFE3DC
:10658C00082840F0FD83614B6549186801222230D0
:10659C0003F07CF9F4E3052810D15E4B5B68B3F58E
:1065AC00803F07D25C4A9BB21846A2F8403004F0F8
:1065BC0099FDE5E3594B04221A70E1E3062803D157
:1065CC00554BB3F840208FE6072807D14F4B554960
:1065DC0018680222403003F0DBFAD1E3082840F0BF
:1065EC00CF834A4B4F4918680222403003F04EF9D2
:1065FC00C6E305280CD1474B5A68032A04D81A79EC
:10660C00454B83F82320BBE3444B04221A70B7E3B9
:10661C00062803D1404B93F8232065E6072807D1C1
:10662C003A4B414918680122233003F0B1FAA7E331
:10663C00082840F0A583354B3B49186801222330CC
:10664C0003F024F99CE305280AD15B68B3F5803F7D
:10665C0002D2314A136393E3304B04221A708FE356
:10666C00062802D12C4B1A6B3EE6072807D1274B84
:10667C002E4918680422303003F08AFA80E3082887
:10668C0040F07E83214B294918680422303003F0F6
:10669C00FDF875E305280BD11E4B5B68B3F5803F05
:1066AC0002D21D4A53636BE31C4B04221A7067E33E
:1066BC00062802D1184B5A6B16E6072807D1134B44
:1066CC001B4918680422343003F062FA58E3082896
:1066DC0040F056830D4B164918680422343003F0F1
:1066EC00D5F84DE305280CD10A4B44F620625B68C3
:1066FC00934202D8084A936342E3084B04221A706F
:10670C003EE3062816D1044B9A6BEDE504000020FD
:10671C00350400206C030020E4030020C00400209A
:10672C000604002024040020070400201404002088
:10673C0018040020072807D19D4B9E491868042295
:10674C00383003F025FA1BE3082840F01983984BE6
:10675C00984918680422383003F098F810E305289B
:10676C000BD1954B5B68012B03D8944A82F86130AE
:10677C0006E3934B04221A7002E3062803D18F4BD5
:10678C0093F86120B0E5072807D1894B8D4918682B
:10679C000122613003F0FCF9F2E2082840F0F082AB
:1067AC00834B884918680122613003F06FF8E7E2E7
:1067BC00052804D1824B586802F026FFE0E2062837
:1067CC0040F0DE8202F0E4FE7EE4052804D17C4B2E
:1067DC00586802F01FFFD3E2062840F0D18202F085
:1067EC00DDFE71E4052804D1754B586802F018FFE2
:1067FC00C6E2062840F0C48202F0D6FE64E4052806
:10680C0004D16F4B586802F011FFB9E2062840F032
:10681C00B78202F0CFFE57E4052804D1684B5868C4
:10682C0002F00AFFACE2062840F0AA8202F0C8FE91
:10683C004AE4052804D1624B586802F003FF9FE23A
:10684C00062840F09D8202F0C1FE3DE4052804D1EB
:10685C005B4B586802F0FCFE92E2062840F09082F6
:10686C0002F0BAFE30E4052804D1554B586802F00A
:10687C00F5FE85E2062840F0838202F0B3FE23E4A5
:10688C00052804D14E4B586802F0EEFE78E206283B
:10689C0040F0768202F0ACFE16E4052804D1484B99
:1068AC00586802F0E7FE6BE2062840F0698202F0BD
:1068BC00A5FE09E4062840F06382FDF74BFE03E4D5
:1068CC00062840F05D82FDF74BFEFFF7FDBB062866
:1068DC0040F05682FDF760FEFFF7F6BB062840F04D
:1068EC004F82FDF755FEFFF7EFBB062840F04882BC
:1068FC0001F062FD00B2FFF7E7BB062840F04082D2
:10690C00FDF716FEFFF7E0BB062840F03982FDF7D5
:10691C0015FEFFF7D9BB062840F03282FDF714FEB6
:10692C00FFF7D2BB05280BD1234B5B68B3F5803F37
:10693C0002D2224A536423E2214B04221A701FE232
:10694C00062802D11D4B5A6CCEE4072807D1184BF0
:10695C001D4918680422443003F01AF910E2082883
:10696C0040F00E82124B184918680422443002F091
:10697C008DFF05E205280BD10F4B5B68B3F5803F0B
:10698C0002D20E4A9364FBE10D4B04221A70F7E11C
:10699C00062802D1094B9A6CA6E4072818D1044B9F
:1069AC000A4918680422483003F0F2F8E8E100BF05
:1069BC00040000201C0400206C030020E4030020D1
:1069CC00C004002045040020280400202C040020D2
:1069DC00082840F0D5818F4B8F4918680422483025
:1069EC0002F054FFCCE105280BD18C4B5B68B3F55E
:1069FC00803F02D28A4AD364C2E18A4B04221A70C5
:106A0C00BEE1062802D1864BDA6C6DE4072807D16B
:106A1C00804B8549186804224C3003F0B9F8AFE17B
:106A2C00082840F0AD817B4B7F49186804224C301C
:106A3C0002F02CFFA4E105280ED15A687B4902F51F
:106A4C00423303F5A8638B4202D8754BDA6597E1A4
:106A5C00744B04221A7093E1062802D1704BDA6D44
:106A6C0042E4072807D16B4B7149186804225C304B
:106A7C0003F08EF884E1082840F08281654B6C4964
:106A8C00186804225C3002F001FF79E105280CD172
:106A9C00624B42F210725B68934202D8604AD38414
:106AAC006EE1604B04221A706AE1062803D15C4B3C
:106ABC00B3F9262018E4072807D1564B5D4918680E
:106ACC000222263003F064F85AE1082840F058817D
:106ADC00504B584918680222263002F0D7FE4FE17D
:106AEC00052808D14D4B5A684D4B003A18BF01226E
:106AFC0083F82B2044E1062804D1494B93F82B2032
:106B0C00FFF7EFBB072807D1424B4B49186801220E
:106B1C002B3003F03DF833E1082840F031813D4B38
:106B2C004549186801222B3002F0B0FE28E10528F7
:106B3C000BD13A4B5B68022B03D8394A82F82A30C6
:106B4C001EE1384B04221A701AE1062804D1344B8A
:106B5C0093F82A20FFF7C8BB072807D12D4B3749DC
:106B6C00186801222A3003F013F809E1082840F0D4
:106B7C000781284B3149186801222A3002F086FE21
:106B8C00FEE005280CD15B68B3F5803F04D2244AA3
:106B9C00D363FEF7F5FBF3E0224B04221A70EFE00F
:106BAC00062803D11E4BDA6BFFF79EBB072807D1D3
:106BBC00184B2349186804223C3002F0E9FFDFE04F
:106BCC00082840F0DD80134B1D49186804223C3026
:106BDC0002F05CFED4E005280AD1104B5A68104B29
:106BEC00003A18BF012283F82C20FEF7C9FBC7E03E
:106BFC00062804D10A4B93F82C20FFF772BB072808
:106C0C0022D1044B0F49186801222C3002F0C0FF2E
:106C1C00B6E000BF040000202C0400206C03002010
:106C2C00E4030020C004002030040020801A060079
:106C3C00400400200A0400200F0400200E04002051
:106C4C002004002010040020082840F099804D4BAF
:106C5C004D49186801222C3002F018FE90E00528EE
:106C6C000BD14A4B5B68012B03D8494A82F82D3073
:106C7C0086E0484B04221A7082E0062804D1444B6B
:106C8C0093F82D20FFF730BB072807D13D4B424925
:106C9C00186801222D3002F07BFF71E008286FD1BB
:106CAC00384B3D49186801222D3002F0EFFD67E0AA
:106CBC0005280BD1354B5868831EFC2B02D8FEF7E8
:106CCC0031F85DE0334B04221A7059E0062804D1E8
:106CDC002F4B93F82520FFF707BB072807D1294B2B
:106CEC002E4918680122253002F052FF48E008288E
:106CFC0046D1244B294918680122253002F0C6FDE3
:106D0C003EE0052808D1214B5A68214B003A18BFA8
:106D1C00012283F8242033E0062804D11C4B93F87D
:106D2C002420FFF7DEBA072807D1164B1C49186838
:106D3C000122243002F02CFF22E0082820D1114B34
:106D4C00174918680122243002F0A0FD18E0032234
:106D5C0000E004220F4B1A70062811D1114B1B783E
:106D6C0073B10C4B10495A68104B0A6022B91A685F
:106D7C0042F008021A6003E01A6822F008021A6056
:106D8C0008BD00BF04000020100400206C0300208C
:106D9C00E4030020C004002011040020090400209A
:106DAC0008040020A4040020D00300207403002059
:106DBC0008B5204B997811B15B78032B36D11D4B5C
:106DCC005B780A2B30D8DFE803F006090C0F141798
:106DDC001A1D22252A0002F0A7FC22E002F0A0FCDA
:106DEC001FE002F0A5FC1CE0124B586802F0A2FC5C
:106DFC0017E002F045FC1CE002F04AFC19E002F03E
:106E0C004FFC0EE00B4B586802F0A8FC11E002F0AE
:106E1C00B5FC06E0074B586802F0B6FC09E002F03E
:106E2C00B9FC054B586004E0032200E00422024B3D
:106E3C001A7008BD6C030020C004002008B50B4B71
:106E4C009A7872B95A7812B1012A08D103E05868BD
:106E5C00FDF76EFD08E05868FDF79AFD04E003228B
:106E6C0000E00422024B1A7008BD00BF6C03002026
:106E7C00C004002010B5A94AA94B107851686422AF
:106E8C00232859601A70587000F0F68053D81328D4
:106E9C0000F0CB8028D8082811D8052880F0B080C5
:106EAC00022800F0A48003D8012840F049819BE01F
:106EBC00032800F09F80042840F042819DE00B28BD
:106ECC0000F0A78006D8092800F09D800A2840F021
:106EDC0037819BE00E2800F0A2800F2800F0A280E2
:106EEC000C2840F02D8197E01B2800F0B08011D8C1
:106EFC00162800F0A38006D8142800F099801528D5
:106F0C0040F01E8197E0172800F09B80182840F075
:106F1C00178199E01F2800F0A38006D81C2800F0E8
:106F2C0099801E2840F00C8197E0212800F09E806B
:106F3C0000F29F8097E0822800F0C58029D8432872
:106F4C0000F0AC8011D8402800F09F8006D824288F
:106F5C0000F09580272840F0F38093E0412800F062
:106F6C009780422840F0EC8095E0462800F09F8006
:106F7C0006D8442800F09580452840F0E18093E045
:106F8C00802800F09A8000F29B80472840F0D8803F
:106F9C0090E0882800F0B68011D8852800F0A480F5
:106FAC0006D8832800F09280842840F0C98090E0B5
:106FBC00862800F0A180872840F0C280A5E08D28AB
:106FCC0000F0B28006D8892800F0A2808C2840F00E
:106FDC00B780A0E0F22800F0AD80FF2800F0AD8073
:106FEC008E2840F0AD80A2E0FEF726FEABE0FEF767
:106FFC002BFEA8E0FEF71AFEA5E0FFF71FFFA2E0AC
:10700C00FEF72CFE9FE0FEF7E1FC9CE0FEF700FC97
:10701C0099E0FEF7CDFB96E0FEF770FB93E0FEF7F0
:10702C0047FB90E0FEF70CFB8DE002F0B7FF8AE027
:10703C0003F092F887E003F01DF984E003F010F9F7
:10704C0081E003F071F97EE003F086F97BE003F058
:10705C00FDF978E003F092F975E003F095F972E030
:10706C0003F0AAF96FE003F0D7F96CE002F0EAFF45
:10707C0069E003F00FFB66E003F000FB63E003F054
:10708C003FF860E002F0E4FE5DE000F05FFB5AE0E8
:10709C0000F05EFB57E000F05DFB54E000F05CFBA1
:1070AC0051E000F05BFB4EE000F05AFB4BE000F0CF
:1070BC0059FB48E000F058FB45E002F019FF42E0B4
:1070CC0002F0E0FE3FE002F0EFFE3CE002F0F2FEE8
:1070DC0039E000F0E1FB134B1C7D02F081FB014613
:1070EC00204603F065F82EE003F07EF800F0CCFBB0
:1070FC000020FDF707FC26E00A4B197D987803F079
:10710C005BFA20E0FEF718FA1DE003F073F81AE0C2
:10711C0003F098FA17E003F023FA14E06C03002054
:10712C00C0040020D004002002F0E8FE0BE0FFF7C2
:10713C003FFE08E0FEF73CFA05E0FEF72BFA02E012
:10714C00014B02221A7010BDC00400202DE9F04F33
:10715C00764B8BB01B78044663B1754B1B78062BB2
:10716C0008D00A2B06D00F2B04D01F2B02D0714B4A
:10717C0000221A70704B1B78012B48D16D4B1A787A
:10718C00511EC9B2012942D858786C496C4BCD6854
:10719C001B78012A0CBF4FF0070C4FF0080C002293
:1071AC0001958DF800C08DF801008DF80220D3B93F
:1071BC00644A8E681578117992F801E092F807C04C
:1071CC00907952798DF808608DF809508DF80AE0A5
:1071DC008DF80BC08DF80C008DF80D208DF80E106D
:1071EC008DF80F300DE0012B09D1574B0132D15CDA
:1071FC000AA88318082A03F8211CF6D101E0022BF7
:10720C0005D0684604F002FB002800F03F824F4B8B
:10721C001B78012B4CD1474A1278032A20D1484BBA
:10722C001B7893B9454E474DB07877782A786B78B0
:10723C00C719BF18EA79FF18AB79BF186A79FF181C
:10724C002B79BF18FF18FFB218E0012B30D10025A5
:10725C003D4BE85C013501F0CDFC092DF8D127E060
:10726C00042A25D1354E374DB27877781046D71988
:10727C00013700222B706A60FFB26A7001F0BAFC11
:10728C00707801F0B7FC287801F0B4FC687801F054
:10729C00B1FCE87901F0AEFCA87901F0ABFC68799F
:1072AC0001F0A8FC287901F0A5FC384601F0A2FCFD
:1072BC00274B1B78012B73D11E4A1278072A49D110
:1072CC001F4B1B782BBB1D4A1E4B5578967893F899
:1072DC0000E093F801C0AF19D879774499796744E5
:1072EC005A79C7191B79CF19D719DF198DF818706E
:1072FC008DF810608DF811508DF812E08DF813C0D8
:10730C008DF814008DF815108DF816208DF81730A7
:10731C0009E0012B07D1013B0B4A995C04AAD1541B
:10732C000133092BF8D104A8092137E09C04002073
:10733C006C0300202802002051000020D004002003
:10734C00D4030020C0040020D80300204E000020ED
:10735C0018000020082A23D19B499C4A91F801C0AF
:10736C0091F802E000250EEB0C06013604A8092169
:10737C0055608DF812308DF813502F468DF814503F
:10738C008DF815508DF816508DF817508DF8186033
:10739C00557013708DF810E08DF811C001F058FF86
:1073AC008B4B8C491A7800230B708B490B7012B1E4
:1073BC00012002F035FA894B1D78012D3CD168462D
:1073CC0004F0A4F9002837D09DF80010844B9DF8E8
:1073DC0008A09DF809809DF80A709DF80B609DF837
:1073EC000CC09DF80D009DF80E907B4A9DF801B0E5
:1073FC00072983F8049083F800A083F801809F701C
:10740C00DE7183F806C0587182F801B001D1157095
:10741C0001E002231370734B1B785A1ED2B2012A5F
:10742C0005D9052B03D0704B01251D7005E06E4B63
:10743C0000221A70012500E000256C4B1B78012BF3
:10744C0059D10DF1270001F0AFFB002853D001F00A
:10745C00C7FB10B1604B00229A705F4B9DF8270060
:10746C0099784A1CD2B2C918092A08719A7041D16C
:10747C00554A18795178002288429A703AD11346AD
:10748C00554D291D895C01325B18082ADBB2F7D1F6
:10749C002A7B9A422CD1524B697AAA7AEE7A6F796E
:1074AC0095F806E095F807C0287A1E7199715A7103
:1074BC001F7083F801E083F802C0D87103F0F8F86C
:1074CC00484B4B4E1B783060591E4A480022C9B2BB
:1074DC00AA700270033201292A7005D9052B03D03A
:1074EC00414B01251D7006E03F4B00221A7001E054
:1074FC0004232B700125404B1B78012B49D107A885
:10750C0001F08EFE002844D02F4B9DF81C205B7898
:10751C009A4276D10022134607A9C95C013352184E
:10752C00082BD2B2F8D19DF824102B4C91422ED1BD
:10753C002B4B9DF821109DF822209DF81D609DF885
:10754C001EE09DF81FC09DF820009DF823509971F6
:10755C005A711E701D7183F801E083F802C0D87156
:10756C0003F0A6F81F4B22491B7808605A1E2149CC
:10757C000020D2B208700721012A217003D9052BF3
:10758C0001D0012200E00022174B1A7039E0237061
:10759C0037E0002D35D113490B78013BDBB2012BC1
:1075AC002FD8012C2DD1154B1A68B2F5006F27D8A6
:1075BC00104601321A600A4902F094FA064B09226D
:1075CC001A70094B1C701CE0D0040020C004002071
:1075DC008C090020D4030020280200205100002038
:1075EC006C030020AC040020A40400204E000020FA
:1075FC00BC040020C8040020180000206C040020EB
:10760C000D70244B1B78042B04D1234B93F90030C1
:10761C00002B2EDA214B1B783BB1042B05D0082B09
:10762C0003D0062B01D0FFF725FC1C4B1B78092B34
:10763C0005D1184A1178022901D103311170184A69
:10764C0012681AB3092B21D1124B1B78012B1DD1B7
:10765C001449013B096809E0134850F82300013331
:10766C00814203D10B4B05221A700FE09342F3D3E6
:10767C000CE0FDF7C5F9094B1B783BB1042B05D089
:10768C00082B03D0062B01D002F040FF0BB0BDE855
:10769C00F08F00BFAC0400206C03002028020020F7
:1076AC00B00400206C0400207004002073B5204B43
:1076BC00024640781F4D1870907800265870D0788C
:1076CC00EC46987010790C46D8715079987192F8F4
:1076DC0006E095E8030083F805E0D2798CE8030016
:1076EC001A71154B1E70FFF7C5FB144B1B7873B941
:1076FC00637023702B78A3706B78E370EB79237134
:10770C00AB7963716B79A3712B79E37108E0012B71
:10771C0006D10B4B9B195B78A3550136082EF8D17B
:10772C00044B6A4692E8030083E803007CBD00BF6B
:10773C006C030020C0040020A4040020D40300200B
:10774C00D8030020704700BF704700BF704700BFD0
:10775C00704700BF704700BF704700BF704700BF45
:10776C00704700BF704700BF704700BF0E4B10B58D
:10777C000022012002214FF4FA744FF0080C5C62D5
:10778C0083F805C09860D9601A621A7058709970A5
:10779C00DA701A719A711A611A755A759A75DA75C6
:1077AC001A76DA6110BD00BFD00400202E4B4FF4C6
:1077BC00FA7CC3F808C04FF4FA6CC3F814C04FF04D
:1077CC00020CC3F81CC00CF1040CF0B583F821C0FA
:1077DC000CF1020C83F825C00CF1C00CC3F85CC092
:1077EC0040F2DC5CC3F838C0ACF5966CC3F844C00E
:1077FC00DFF878C04FF47A640021012005274FF49C
:10780C0016764FF44875DC63C3F854C01C605C609A
:10781C0043F2903C4FF47A741F615E63A3F84010FE
:10782C00DD6483F85000C3F858C0DF60986183F8BA
:10783C00200083F8221083F8231083F82410DC84B2
:10784C00198583F82A0083F82B0083F82C101E630B
:10785C0083F842109D6483F8511083F8601083F80C
:10786C002D1083F86110F0BDE403002000390300F3
:10787C00014B10225A61704700080140014B102245
:10788C001A61704700080140024B4FF400421A6124
:10789C00704700BF00100140024B4FF400425A6188
:1078AC00704700BF00100140024B986800F4004084
:1078BC00704700BF00100140024B4FF480521A6118
:1078CC00704700BF00100140024B4FF480525A61C8
:1078DC00704700BF00100140704700BF704700BFE9
:1078EC00704700BF704700BF704700BF704700BFB4
:1078FC00704700BF704700BF704700BF704700BFA4
:10790C00704700BF014B04221A6170470008014008
:10791C00014B04225A61704700080140054B9A68DC
:10792C0012F0040F02D004225A6101E004221A6101
:10793C00704700BF00080140024B4FF400721A61FF
:10794C00704700BF000C0140024B4FF400725A61AB
:10795C00704700BF000C014010B9024B20225A6145
:10796C00704700BF0010014010B9024B20221A6171
:10797C00704700BF0010014018B1012803D000204F
:10798C0005E0034B00E0034B9868C0F380007047A0
:10799C0000140140000C014008B1002003E0024B30
:1079AC009868C0F34010704700100140064B1B78DC
:1079BC00012B04D1054B4FF480521A6102E0044BA9
:1079CC0001221A70704700BF18000020000C014003
:1079DC0038020020064B1B78012B04D1054B4FF4C9
:1079EC0080525A6102E0044B00221A70704700BFAB
:1079FC0018000020000C014038020020054B1B78B9
:107A0C00012B03D1044B0020DB6801E0034B1878F9
:107A1C00704700BF18000020000C01403802002005
:107A2C00704700BF704700BF094B10B59C68C4F38A
:107A3C0082140CB1072C05D1012803D11F3001F0A1
:107A4C00AFFE02E0202001F0B3FE204610BD00BFC7
:107A5C00000C014008B518B1012804D0002006E044
:107A6C00034B586801E0024B986800F097F908BD89
:107A7C001800002037B501AD002429464FF01F0334
:107A8C000848ADF804308DF8074007F05DFE4FF064
:107A9C000303294604488DF80740ADF8043007F07D
:107AAC0053FE3EBD00100140000C01402DE9F34790
:107ABC00584E01AD04200121032407F0F9F91027D9
:107ACC0030464FF0BE032946ADF804308DF8064021
:107ADC008DF8077007F038FEAE234FF00408DFF87E
:107AEC003CA130463761294673614FF04103ADF834
:107AFC0004308DF806408DF8078007F025FE08202D
:107B0C00012107F0D5F941F2386350462946ADF80A
:107B1C0004304FF020098DF806408DF8077007F0FF
:107B2C0013FE41F2182350462946CAF81090CAF8A1
:107B3C00143040F6C71306F50066ADF804308DF826
:107B4C0006408DF8078007F0FFFD3846012107F04D
:107B5C00AFF930464FF220432946ADF804308DF88A
:107B6C0007708DF8064007F0EFFD4FF4E0433361EA
:107B7C0003F5A1533046736129464FF43C63ADF8CD
:107B8C0004308DF806408DF8078007F0DDFD4FF0CE
:107B9C001F03304629460026ADF804308DF8064008
:107BAC008DF8076007F0D0FD4846012107F080F9F9
:107BBC004FF40040314607F057FE4823164829463B
:107BCC008DF80730ADF804808DF8064007F0BCFD49
:107BDC003046334611494FF480644C610A4689683B
:107BEC00013611F4006F4FF480611161926808BF87
:107BFC00013312F4006F18BF01300A2EEAD10A2BA0
:107C0C0001D0002003E00A2814BF00200120BDE8A9
:107C1C00FC8700BF0008014000140140000C01402B
:107C2C00704700BFFEE700BFFEE700BFFEE700BFE6
:107C3C00FEE700BF704700BF704700BF704700BF32
:107C4C00704700BF704700BF704700BF704700BF50
:107C5C00704700BF704700BF704700BF704700BF40
:107C6C00704700BF704700BF704700BF704700BF30
:107C7C00704700BF704700BF704700BF704700BF20
:107C8C00704700BF704700BF08B5024B1B68984790
:107C9C0008BD00BF7803002008B5024B1B6898474D
:107CAC0008BD00BFCC040020684620F00701044B3F
:107CBC008D4601B51B689847BDE801408546704765
:107CCC00A004002008B5024B1B68984708BD00BFF4
:107CDC00A8040020704700BF704700BF704700BF6A
:107CEC00704700BF704700BF704700BF704700BFB0
:107CFC00704700BF704700BF704700BF704700BFA0
:107D0C00704700BF704700BF704700BF704700BF8F
:107D1C00704700BF704700BF704700BF704700BF7F
:107D2C00704700BF704700BF704700BF704700BF6F
:107D3C00704700BF704700BF704700BF704700BF5F
:107D4C00704700BF704700BF704700BF684620F007
:107D5C0007018D4601B5002303E00B495958995092
:107D6C0004330A4A0A4998188842F6D3094B02E0B0
:107D7C00002243F8042B084A9342F9D3FCF746FA45
:107D8C00BDE80140854670479C12010800000020A8
:107D9C009C0100209C010020241D0020024B33F884
:107DAC00100080B2704700BF4C020020024B03EB66
:107DBC0040031982704700BF4C020020024B03EBBA
:107DCC004003188A704700BF4C02002010B50A4CC3
:107DDC0024781CB9002914BF0A461A46502148437E
:107DEC00064B424302991878039B002808BF0B46A8
:107DFC0092FBF3F010BD00BF980900209A090020F7
:107E0C00A5234343044AA3F5A52310684FF48052DD
:107E1C00584390FBF2F0704758000020014B18704B
:107E2C00704700BF9A090020014B1870704700BFC3
:107E3C0098090020074B10B51B68074C34F8130049
:107E4C0080B2FFF7DDFF20220146206A04F0A0FB80
:107E5C00206210BD340000204C020020F8B5114BFC
:107E6C00114E1B68044636F8130080B2FFF7C8FFAA
:107E7C000E4B05461B6836F8130080B2FFF7C0FFA7
:107E8C00064605FB05F006FB060077197F4207FB4B
:107E9C00070004F0E3FAA680A060678025802046E6
:107EAC00F8BD00BF3C0200204C0200203400002032
:107EBC00F8B5114B114E1B68044636F8130080B20E
:107ECC00FFF79EFF0E4B05461B6836F8130080B279
:107EDC00FFF796FF064605FB05F006FB0600771933
:107EEC007F4207FB070004F0B9FAA780A060668008
:107EFC0025802046F8BD00BF3C0200204C0200202B
:107F0C003000002038B5104C257885B1012D1AD1E0
:107F1C000E4B5B6A002BB8BF5B42B3F5E16F12DD11
:107F2C00FFF7D2FC00232370094B1D700BE0074BAD
:107F3C005B6AC733B3F5C77F05D8FFF7BDFC044AAE
:107F4C0001231370237038BD9A0900204C020020C5
:107F5C00990900202DE9F74F534C0025074665621F
:107F6C005248884692469946DDF834B006F000FB3C
:107F7C00C8F5E168404501D307241EE04C4B626A0A
:107F8C001B68002A34F8130004EB43010B8A80B2FF
:107F9C00B8BF5242C01A80EAE073A3EBE07393427D
:107FAC000E9BC8BF606251460193CDF800B04A46A3
:107FBC000C9BFFF70BFF062405463C4806F0DCFA49
:107FCC00404501D3002621E03A4A374B1268596AE2
:107FDC0033F8120003EB4206328A80B2801A81EA2F
:107FEC00E172A2EBE17280EAE071A1EBE0719142E7
:107FFC00C8BF58620E9BCDF800B0019351464A465B
:10800C000C9BFFF7E3FE24F002040646274806F01B
:10801C00B7FA404502D34FF0000822E0264A224B23
:10802C001268596A33F8120003EB420CBCF81020AA
:10803C0080B2801A81EAE172A2EBE17280EAE0710F
:10804C00A1EBE0719142C8BF58620E9BCDF800B015
:10805C00019351464A460C9BFFF7B8FE24F00404EA
:10806C008046022C07D0042C09D0012C0BD108EB34
:10807C0006056D4207E008EB0506764203E006EBC9
:10808C000508C8F1000805FB05F006FB060008FB17
:10809C00080004F0E3F9A7F80480B8607E803D8006
:1080AC003846BDE8FE8F00BF4C020020002C01407A
:1080BC003C020020300000203400002070B590B04D
:1080CC00FFF7D8FC0120014606F0E4FE01214FF435
:1080DC00007006F0EDFE414807F008FD404B00240F
:1080EC000093404B0726019380230593DB180693DE
:1080FC0003F540730793A3F57873384869460893E2
:10810C0003F5FF5309930294039604940A9407F021
:10811C005DFD0121314807F089FD01254FF46023F5
:10812C0031480BA90D930B948DF830508DF83140DC
:10813C000E948DF83C6008F0E1F82C4B2A48197825
:10814C002A46032308F05CF9294B022219782648A9
:10815C00032308F055F9274B0322197822481346BC
:10816C0008F04EF9244B042219781F48032308F019
:10817C0047F9224B052219781B48032308F040F9D4
:10818C001F4B062219781848032308F039F91D4BA8
:10819C00324619781448032308F032F92246124863
:1081AC004FF4FC6108F0EEF80F48294608F0E0F8AF
:1081BC000D48294608F0D2F80B4808F0EDF80A48AB
:1081CC0008F0F0F80028FAD1074808F0EFF8064854
:1081DC0008F0F2F80028FAD110B070BD0800024087
:1081EC004C2401404C0200200024014028000020B7
:1081FC00290000202A0000202B0000202C00002049
:10820C002D0000202E000020F0B54469856903463E
:10821C006543881A4FF47A7C002895FBFCF6B8BFAE
:10822C004042B042B8BF0CFB00F5104E4FF47A7CC4
:10823C0030682D1895FBFCF00CFB105737600CB90F
:10824C00114611E0914205DA1B6841189942A8BF0A
:10825C00194609E008DD064A1B6895FBF2F569181A
:10826C005B429942B8BF19460846F0BD7402002023
:10827C0018FCFFFF2DE9F047044690F821000D464D
:10828C00062816469846DDF820A027681ED10868F7
:10829C00014608F0D5FB3E4908F0D2FB814694F824
:1082AC002500400808F078FB0146484608F0C8FB5A
:1082BC00636981467820584308F06EFB01464846B6
:1082CC0008F072FC08F082FD034611E0072801D08B
:1082DC0000230DE00868014608F0B2FB2D4908F0B8
:1082EC0063FC08F073FDE36B6269434393FBF2F3A9
:1082FC00C245C8EB0A08B8BF7F42B8F1000FB8BF3F
:10830C00C8F100084FF480409845D8BF002701F011
:10831C0057FA012803D1304608F03EFB31E03846CD
:10832C0008F03AFB2E6880464146304608F026FDA0
:10833C0070B1A069636937B90B225043584308F0F8
:10834C0027FB154917E0584308F022FB134912E0AC
:10835C004146304608F030FDA0B1A069636937B9D9
:10836C000B225043584308F013FB0D4903E05843CC
:10837C0008F00EFB0B4908F017FC0146304608F0DC
:10838C0057FA2860286808F021FDBDE8F08700BF87
:10839C000000C0400000F04200401C4600007A443F
:1083AC0000401CC600007AC4024B00229A601A607E
:1083BC005A60704778020020014BB3F90C007047EB
:1083CC007802002070B546680446154608463246C9
:1083DC0071421E4604F0BCF8236B00B2B3607368A4
:1083EC00616B451BE818F1603560706011B1104B82
:1083FC0093FBF1F10A46494204F0AAF80346F068EF
:10840C00B168326858434A434FF4803190FBF1F025
:10841C00A1F57F4192FBF1F2801830617360A1F5F8
:10842C00014147F6FF7204F093F800B270BD00BF33
:10843C000000FF7F2DE9F04F89B0B44DBDF84840E6
:10844C00BDF84AC02C82A5F812C0044628699B4688
:10845C00DDF8548089460192169EDDF860A003F089
:10846C000BF9C0F30F43ADF81A30ADF81800069BAA
:10847C00B8F800706B6194F82130072B25D0082BCD
:10848C0000F05E82062B40F0D48202F0A5FC94F83A
:10849C002D3085B2012B0AD194F825101A98490871
:1084AC00E26902F073FC02F02DFC4519ADB294F8B0
:1084BC002430012B03D105F5FE45FF35ADB22DB2AD
:1084CC00284602F057FC0020F6E102F0DBFD012803
:1084DC0040F00D824FF4007001F072F9012801D1C7
:1084EC00199B5BB94FF4006001F06AF9012840F068
:1084FC00FB81D8F80030002B00F0F68194F82A00AC
:10850C00012800F07A8104D30228804B40F0D981F5
:10851C0073E07E4B42F210715A6801328A425A6003
:10852C0025D8A56BB4F862305543B3F5007FB5FB85
:10853C00F1F5ADB202D0B3F5806F02D12BB2C8F811
:10854C000030002002F016FC002002F0AFFD0021EC
:10855C006F4803F035F804A9C0F30F43ADF81000D1
:10856C0004223046ADF8123008F094F874E2694AEF
:10857C00002012785860012A12D1A58F02F0DCFD80
:10858C00281A80B2254625F8400F02F0ABFD624B4D
:10859C0029461B680222ED18281B01F0F9FA14E099
:1085AC0002F078FD94F82A302BB994F8423043F05D
:1085BC00010384F8423094F82A30022B05D194F848
:1085CC00423043F0020384F84230504B4FF000012C
:1085DC0059831983584600F0E1FA484600F0DEFA58
:1085EC00179A002300201360CAF8003002F044FDF3
:1085FC004FF4004001F0D4F819E21B68032B00F291
:10860C001682DFE813F004004800D200D200414A81
:10861C003E4B1278012A00F0C6805A6842F2107163
:10862C008A422BD8A56B013255435A600020B5FB0A
:10863C00F1F5009302F09EFB002002F037FD009B49
:10864C00002103F1140002F0BBFF0422C0F30F431E
:10865C00ADF8100004A93046ADF8123008F01AF845
:10866C00B4F86230ADB2B3F5007F03D0B3F5806FD0
:10867C0040F0F2812BB2C8F80030EDE100200093FD
:10868C0002F008FD94F8422042F0020284F84220E5
:10869C00009B012287E01F4A1C4B1278012A0FD144
:1086AC00B4F84000009302F01DFD02F057FD00F5F8
:1086BC000040009B013000B202221A609860B6E1C3
:1086CC009D6894F8252085EAE5705208A0EBE570CA
:1086DC00C2EB0241884265DAE16DE769C1EBC13159
:1086EC004F435743B4F862200C48B2F5007F97FB18
:1086FC00F0F702D0B2F5806F1AD1DAF800A00021A1
:10870C00504608F059FB58B1ED1B0FE078020020E1
:10871C008C0200204A02002004000020C02709001F
:10872C005046002108F02AFB70B17D19A54B0AE0D8
:10873C00B2F5006F08D1D8F80020002A01DDED1B3E
:10874C0001E001D07D199D609E4F0020258F02F025
:10875C0011FBB86802F0AAFCB7F9081007F1140075
:10876C0002F02EFF0422C0F30F43ADF8100004A951
:10877C003046ADF8123007F08DFFB4F86230B3F527
:10878C00007F02D0B3F5806F02D12BB2C8F8003055
:10879C0094F8427017F0020740F05E81894B022278
:1087AC001A605AE103221A6041E1864D4FF0000233
:1087BC002A836A83584600F0F1F9484600F0EEF936
:1087CC002A6817990023022A0B60CAF8003005D1D9
:1087DC00002002F051FC4FF4004000E08020794D65
:1087EC0000F0DEFF002002F0C5FAA86802F05EFC83
:1087FC00B5F9081005F114001EE1FFF715F9714DDC
:10880C0001468046287F02F083FA85F81C801FFA07
:10881C0080F802F0E1FA94F8243005B2012B04BF81
:10882C0005F5FE45FF35284602F0A4FA18F4004F72
:10883C0003D005F5D445AA3511E0B8F1000F00F0CE
:10884C00338105F5144505F5AA7508E000F5FE40E1
:10885C00FF3080B200F5FE45FF35ADB227E05A4B34
:10886C00E06B1A7894F82530012A0BD000B24543FE
:10887C005B0895FBF3F04FF6FF7390FBF3F080B2BF
:10888C0002F04CFC02F06AFC4E4B4FF000025A8393
:10889C001A830546584600F081F9484600F07EF9E7
:1088AC00002002F0E9FB4FF4004000F079FF05F5E1
:1088BC00004501352DB2284602F0F8FB2946434805
:1088CC0030E003F11400002102F07AFE0027C0F31F
:1088DC000F43ADF8100004A930460422ADF8123055
:1088EC003D4607F0D7FEB8E000213848A4E002F07E
:1088FC0035FC94F82A3000F500400130012B85B28C
:10890C0003D102F069FA00B200E000200FFA85F8FA
:10891C0002F030FA404602F0C9FB2A4B414603F103
:10892C0014009D8102F04CFE04A9C0F30F43ADF876
:10893C00100004223046ADF8123007F0ABFE76E0A2
:10894C00E26994F825304FEA0238DAF8000003FBAC
:10895C0008F808F03BFA0028B8BF404200FB08F8C2
:10896C002B6A40F2DC5298FBF2F89844642398FB93
:10897C00F3F203FB1283DAF800A02B6200215046BD
:10898C004FF0000508F018FA08B14FF00105EDB2F0
:10899C0025B10C4B6FF063019A8907E0504600211A
:1089AC0008F0ECF938B1074B64219A8998FBF1F87F
:1089BC009044A3F80C80034BB3F80C8045B108F538
:1089CC0080480CE0780200204A0200208C02002033
:1089DC005046002108F0D2F918B1A8F580481FFACA
:1089EC0088F80FFA88F1354802F0EAFD0422C0F34A
:1089FC000F43ADF8100004A93046ADF8123007F063
:108A0C0049FE02F0E9F994F8243080B2012B03D12D
:108A1C0000F5FE40FF3080B200B202F0ABF902F07C
:108A2C009DFB00F50040013000B202F03FFB002539
:108A3C0013E005F11400002102F0C2FD0025C0F383
:108A4C000F43ADF8100004A930460422ADF81230E3
:108A5C002F4607F01FFE00E0002739B24B46B6F94F
:108A6C0000202046FFF7AEFC154F019B388329B23E
:108A7C00B6F902202046FFF7A5FC788307F1180011
:108A8C0002F0FAFC07F1180002F01CFDC0F30F43D2
:108A9C00ADF80800ADF80A30029B18467B6201F075
:108AAC006FFE09B0BDE8F08F02F096F994F824300F
:108ABC0080B2012B7FF4CEAEC8E600BF8C02002042
:108ACC0078020020F8B5066804461546084632467A
:108ADC0071421E4603F03CFDA36C451BB360E36C76
:108AEC001D49F3600746356028464FF6FF7203F0C8
:108AFC002FFD03467068F16818183360706019B167
:108B0C0063681B0493FBF1F10A46494203F020FD14
:108B1C000346F068B168326858434A434FF48031D9
:108B2C0090FBF1F0A1F57F4192FBF1F280183061DE
:108B3C00736094F82130082B08D1002F01DDA06B55
:108B4C0009E016BFA06B3846404204E061680A4653
:108B5C00494203F0FDFCF8BD0100FFFF70B5466C07
:108B6C001D4604469E60881A0023EB6028600A4963
:108B7C004FF6FF7203F0ECFC0346A8684FF48072CA
:108B8C00584390FBF2F028612B6021680A46494259
:108B9C0003F0DEFC70BD00BF0100FFFF002303618A
:108BAC0003604360704700BF094B19685A689142D3
:108BBC0001D100200BE01A68D118097A013201703A
:108BCC001A601A68202A01D100221A60012070470D
:108BDC00A0020020014B9862704700BFA002002049
:108BEC00034B1A78104612B100221A7001207047FC
:108BFC009C09002038B50B4B8446DC6A1A6B013497
:108C0C00202C08BF002494420BD0DD6A064AED18D4
:108C1C00106885F834C040F227710122DC6204F040
:108C2C00E1FE38BDA00200206000002038B50546EA
:108C3C00002401E0FFF7DEFF2B5D01341846002B0A
:108C4C00F8D138BD70B5294C238813F0200F1AD0F9
:108C5C00FEF7D4FE08B1A38815E0254B5A681968B5
:108C6C000132202A08BF00228A4205D05968A08808
:108C7C00C918C0B208725A601E4B0A221A601C4BEB
:108C8C009A6A1D4B1A60194E338813F0800F1BD053
:108C9C00194B1C68C4B9164DEA6A2B6B9A420DD05D
:108CAC00FEF784FE2B6B5A1992F834200133B280F4
:108CBC002B632B6B202B07D12C6305E0304622460F
:108CCC0040F2277104F08EFE0848038813F0400F21
:108CDC000AD040F2266104F07DFF054B1A6BDB6A6B
:108CEC009A4201D1FEF776FE70BD00BF00480040ED
:108CFC00A0020020A0090020A409002070B5294C76
:108D0C00238813F0200F1AD0FEF778FE08B1A38841
:108D1C0015E0254B5A6819680132202A08BF002239
:108D2C008A4205D05968A088C918C0B208725A6026
:108D3C001E4B0A221A601C4B9A6A1D4B1A60194E64
:108D4C00338813F0800F1BD0194B1C68C4B9164D17
:108D5C00EA6A2B6B9A420DD0FEF728FE2B6B5A1940
:108D6C0092F834200133B2802B632B6B202B07D16C
:108D7C002C6305E03046224640F2277104F032FEA7
:108D8C000848038813F0400F0AD040F2266104F023
:108D9C0021FF054B1A6BDB6A9A4201D1FEF71AFED2
:108DAC0070BD00BF00440040A0020020A0090020BC
:108DBC00A409002070B57B4B86B01C780546012CAD
:108DCC002AD1794804F056FF21464FF4003006F0C2
:108DDC007DF82146042006F06BF80420002106F0F3
:108DEC0083F80820002106F03FFD06AC4FF0040389
:108DFC0024F8043D032321466C488DF816301533B6
:108E0C008DF8173006F0A0FC48238DF8173021465A
:108E1C0066484FF008032DE0654B1C78012C2DD1D2
:108E2C00644804F027FF21464FF4802006F04EF8EA
:108E3C002146082006F03CF80820002106F054F8E2
:108E4C005D48002106F010FD06AC4FF4806324F859
:108E5C00043D0323594821468DF8163015338DF8FF
:108E6C00173006F071FC042354488DF81730214656
:108E7C004FF40063ADF8143006F066FC684604F05D
:108E8C007BFD0B2D25D8DFE805F02406090C0F120D
:108E9C0015181B1E20224FF461531CE04FF496430F
:108EAC0019E04FF4E14316E04FF4164313E04FF48E
:108EBC00614310E04FF496330DE04FF4E1330AE0D8
:108ECC004FF4613307E03E4B05E03E4B03E03E4B75
:108EDC0001E04FF4165300933C4B1A683C4B9A42FA
:108EEC0002D1009B5B0800932E4B1B78012B04D105
:108EFC00384B2D4A1A60262307E02D4B1B78012B8B
:108F0C0005D1344B2B4A1A6027238DF81030314C85
:108F1C006946206804F066FE00250723012604A894
:108F2C008DF811308DF812508DF8136006F08EF814
:108F3C00206840F2FF3104F029FE206828212A46DF
:108F4C0004F050FD2068324640F2277104F04AFDCF
:108F5C002068324640F2266104F044FD2068324617
:108F6C0040F2255104F03EFD20682A4640F224418F
:108F7C0004F038FD20682A4640F6460104F032FD24
:108F8C0020682A4640F66A1104F02CFD2068602106
:108F9C002A4604F027FD2068314604F015FD06B082
:108FAC0070BD00BF45020020004400400008014095
:108FBC004F0000200048004010001400000C01403D
:108FCC0090D0030020A1070040420F005C0000205D
:108FDC000024F40060000020014B03221A6070474B
:108FEC00F4020020044A054B927A0AB1052200E0F3
:108FFC0001221A60704700BFB8090020F40200205B
:10900C00704700BF014B00225A607047F4020020E9
:10901C0008B5074B1A6892B242F008021A601A6837
:10902C0092B242F004021A60FFF7D6FF08BD00BFEF
:10903C00405C004010B5064C4FF6FB73226802EA08
:10904C0003032360FFF7CEFF4FF40643236010BDEC
:10905C00405C0040072818BF1F4B10B51E4C18BFB2
:10906C0018702378052B33D8DFE803F003060A0EBB
:10907C001621FFF7DFFF2BE0FFF7DCFF042328E0CE
:10908C0002236370013324E06378013BDBB263702D
:10909C006378FBB9042218E0104B1A6892B242F0C4
:1090AC0010021A6005232370DB18637012E06378DA
:1090BC00013BDBB26370637863B9084A4FF6EF7318
:1090CC00116801EA030313600622034B1A7001E0D6
:1090DC000623237010BD00BF1C0A0020405C00401A
:1090EC00034B9B7A13B1034B05221A60704700BFE8
:1090FC00B8090020F4020020014B04221A607047CA
:10910C00F4020020034B1A7A202A01D100221A7291
:10911C00704700BFF4020020704700BF212808B53B
:10912C0008D1124B1B681B7803F07F03212B1AD13B
:10913C000F4B0EE0202816D10C4B0E4A1B681B78E7
:10914C0010720D4A03F07F03212B0CBF1346002332
:10915C004BB1064A4FF00001126800205182936116
:10916C009847002000E0022008BD00BF180A00202C
:10917C00BD910008F4020020D9910008074B1B6830
:10918C001B7803F07F03212B05D1022801D0222864
:10919C0001D1002000E00220704700BF180A002017
:1091AC0019B9012801D8084600E00220704700BF19
:1091BC0028B9044B4FF008021B681A8200E00248E1
:1091CC00704700BF180A00206400002028B9044B27
:1091DC004FF008021B681A8200E00248704700BF7B
:1091EC00180A0020640000200B4B10B5DA6882B11D
:1091FC001B68052B01D000220BE0002303E007497C
:10920C00595CC15401330449CC68A342F7D3002301
:10921C00CB60104610BD00BFF4020020240A0020D1
:10922C00084BDB68082B01D800200AE00023064A13
:10923C009A5CC2540133092BF9D1024B0022DA603B
:10924C0001207047F4020020240A0020704700BF60
:10925C0010B5074C0B468AB2C021636003F0F6FDD3
:10926C000120A18803F01EFC012003F0E9FA10BDD7
:10927C00F402002008B5064B1B68DB78042B01D9DF
:10928C00002004E0034901EBC30104F03FF808BDE2
:10929C00180A00206C00002008B5024904F036F8CA
:1092AC0008BD00BF8C00002008B5024904F02EF860
:1092BC0008BD00BF94000020334B10B51B686FF045
:1092CC003F0200245A72DC729C72204603F030FA82
:1092DC0020464FF4007103F049FA1021204603F0A8
:1092EC005BFA4021204603F0B1FB8021204603F0BD
:1092FC009DFB204603F0DAFA244B204693F86410C9
:10930C0003F0F2FB204603F0A9FA0120214603F0FA
:10931C002DFA0120C02103F089FB0120202103F04C
:10932C003BFA0120214603F04FFA02204FF4C061B2
:10933C0003F01CFA02204FF4807103F077FB02203B
:10934C00214603F041FA0220202103F025FA0320E4
:10935C00214603F00BFA03204FF4887103F076FBDF
:10936C000320402103F0C0FB03204FF4405103F0D5
:10937C002BFA2146032003F00FFA204603F0D4FF0A
:10938C00034B01221A6010BD180A00206400002053
:10939C00F402002008B5174B174A196889B21180DE
:1093AC0016491288098801EA020212F4806F05D06E
:1093BC004FF6FF321A60124BDB6B98470E4B1A8834
:1093CC000E4B1B8803EA020212F4007F08D00949F5
:1093DC000C4A4FF6FF500860117C0131C9B2117470
:1093EC00054A1288134013F4004F01D003F09AFD84
:1093FC0008BD00BF445C0040AA090020640A00209C
:10940C0064000020F402002010B5032003F09CFB44
:10941C00064C034602464FF488710548E36003F09E
:10942C002DFD032003F01AFA10BD00BFF40200203A
:10943C00240A002008B5064A064B20B1106819888A
:10944C0006F0EAF903E01068198806F0E3F908BDA4
:10945C00B4090020B009002038B5064D01232B605B
:10946C00054B002420461C60FFF7E4FF03232B6010
:10947C00204638BD405C0040445C004008B5FFF716
:10948C00EBFF08BD08B50120FFF7D4FF064B012107
:10949C00196006494FF4E0520A8005490020186013
:1094AC0008601A6008BD00BF405C0040640A0020E0
:1094BC00445C0040084B10B51B6800249C72FFF7FD
:1094CC00E1FF064A4FF406431460043A1360044A61
:1094DC001460044A138010BD180A0020445C00403C
:1094EC00F4020020640A002007B5142200238DF832
:1094FC00042001A801228DF806308DF807208DF884
:10950C00053005F0A3FD0EBD002008B505F046FCA6
:10951C004FF40000012105F0D9FC08BDF7B5184C3B
:10952C00184E194F194D9DF820C031602A803860B3
:10953C000999302204F17E0084F8723084F873C0EB
:10954C0007F0A8F80A99182204F1B20007F0A2F863
:10955C00FFF7DAFFFFF7C8FF03F0A8FD3868012119
:10956C0005F0A6FC03232D888DF8063030680D33EA
:10957C0001A9ADF804508DF8073006F0E5F8FEBDF2
:10958C0064000020B4090020200A0020B00900204B
:10959C00014B1868704700BF2C1A0020014B18684B
:1095AC00704700BF241A0020014B1868704700BF99
:1095BC00201A0020014B1868704700BF181A0020B1
:1095CC00014B1868704700BF281A0020014B18681F
:1095DC00704700BF0C1A0020014B1868704700BF81
:1095EC00141A0020014B1868704700BF101A002095
:1095FC00014B1868704700BF1C1A0020014B1868FB
:10960C00704700BF680A0020014B1860704700BF0C
:10961C002C1A0020014B1860704700BF241A002040
:10962C00014B1860704700BF201A0020014B1860D6
:10963C00704700BF181A0020014B1860704700BF1C
:10964C00281A0020014B1860704700BF0C1A00202C
:10965C00014B1860704700BF141A0020014B1860B2
:10966C00704700BF101A0020014B1860704700BFF4
:10967C001C1A0020014B1860704700BF680A0020BC
:10968C00024B00225A6001321A7070470803002006
:10969C00024B00225A601A70704700BF080300206A
:1096AC00014B1878704700BF08030020014B586825
:1096BC00704700BF0803002008B5064B00215A680C
:1096CC0099600132B2F5FA7F5A6001D1FFF7E0FFE1
:1096DC0008BD00BF0803002013B50E4B6A4682E894
:1096EC0003000D499A680C680132A24201469A6047
:1096FC0001980DDB1A785AB15B68B3F5FA7F07DA7B
:10970C00064A02EBC304606042F83310FFF7D4FF43
:10971C001CBD00BF08030020940100206C0A00202F
:10972C004FF4FA70704700BF4FF47A60704700BF77
:10973C0002207047B0F5FA7F0CDA11B1012909D17A
:10974C0003E0054B53F8300005E0034B03EBC0007E
:10975C00406800E0002070476C0A0020012804D00B
:10976C00022802D0044B18B900E0034BD86001E08A
:10977C000022DA60704700BF08030020014BD86854
:10978C00704700BF08030020014B1860704700BFF2
:10979C0094010020014B1868704700BF9401002011
:1097AC00024B1A6840EA02021A6070471803002044
:1097BC00024B1A6822EA00021A6070471803002054
:1097CC00034B1B6818420CBF00200120704700BFE0
:1097DC001803002008B56D20FFF7EAFF08BD00BF95
:1097EC00034B10B51C68FFF7F5FF204610BD00BFFA
:1097FC0018030020034B10B51C68FFF7EBFF04F0B7
:10980C006F0010BD1803002062B6704772B6704727
:10981C0008B5FEF741F808BD08B5FEF735F808BDE8
:10982C0008B510B105F0B0FC01E005F0B5FC08BDC1
:10983C0007B5104B1B78E3B1FEF762F8FEF762F840
:10984C00FEF782F8002301E0019B01330193019A9A
:10985C00094B9A42F8D9FEF75BF8FEF76DF8002336
:10986C0001E0019B01330193019A034B9A42E3D827
:10987C00F7E70EBDD50300203F0D030008B5FEF73A
:10988C0015F9014B187008BDD50300202DE9F341E3
:10989C00234B05461B788846012B16461DD1002408
:1098AC0018E001AF4FEA152C39460222A6231D48B9
:1098BC008DF804C08DF8055002F0F8FBA62339464C
:1098CC001848022202F068FC9DF80430013508F8B3
:1098DC0004300134B442E4D31FE0002003210246DB
:1098EC0002F006FA0020C5F30721024602F000FA46
:1098FC000020E9B2024602F0FBF9002408E0944291
:10990C0014BF0022012202F0F3F908F8040001341C
:10991C000020721EB4420146F1D3BDE8FC8100BFA9
:10992C00490200200058004073B5174B050A1B78FC
:10993C000446012B13D101AE31460222A533134844
:10994C008DF804508DF8054002F0B0FB31460F48FD
:10995C000222A62302F020FC9DF8040013E0002054
:10996C000321024602F0C4F90020E9B2024602F0DB
:10997C00BFF90020E1B2024602F0BAF9002001461C
:10998C00012202F0B5F97CBD4902002000580040CC
:10999C0037B52D4B0C461B78012B4CD00725454376
:1099AC0000200321024602F0A3F905F50065002012
:1099BC00C5F30721024602F09BF90020E9B20246EA
:1099CC0002F096F900200146024602F091F98DF85A
:1099DC00000000200146024602F08AF98DF80100D1
:1099EC0000200146024602F083F98DF802000020A7
:1099FC000146024602F07CF98DF804000020014675
:109A0C00024602F075F98DF8050000200146024669
:109A1C0002F06EF98DF8060000200122014602F0DA
:109A2C0067F92368009A23F07F4322F07F429A4221
:109A3C008DF8070001D0002005E06368019898427A
:109A4C0014BF002001203EBD4902002038B5234B35
:109A5C001B78012B41D0224B1C683BE000200621D7
:109A6C00012202F045F900200521024602F040F9DE
:109A7C0000200122014602F03BF910F0020FF2D057
:109A8C0000200221024602F033F90020C4F3072122
:109A9C00024602F02DF90020E1B2024602F028F94C
:109AAC00002500203F2D14BF002201220146013564
:109ABC0002F01EF9402DF4D100200521024602F0DF
:109ACC0017F900200122014602F012F910F0010FE3
:109ADC00F2D14034B4F5804FC0D338BD49020020D8
:109AEC001000002038B5224B0C461B78012B3DD0C2
:109AFC000725454300200321024602F0F9F805F53D
:109B0C0000650020C5F30721024602F0F1F80020A1
:109B1C00E9B2024602F0ECF800200146024602F0DF
:109B2C00E7F8207000200146024602F0E1F8607070
:109B3C0000200146024602F0DBF8A070002001462E
:109B4C00024602F0D5F8207100200146024602F0D0
:109B5C00CFF8607100200146024602F0C9F8A071EE
:109B6C0000200146012202F0C3F8E07138BD00BFAD
:109B7C004902002010B500F09BFD044600F098FD52
:109B8C00001B0028B8BF40420628F7DD10BD00BFFF
:109B9C002DE9F3414D4B06461B780F46012B14461D
:109BAC001AD100250DE017F805E08DF804C08DF8EA
:109BBC0006E08DF8056002F079FAFFF7DBFF01365D
:109BCC000135A5424FEA162C01A94FF003024FF0C4
:109BDC00A6033F48E7D376E000200621012202F0DD
:109BEC0087F800200521024602F082F800200122AD
:109BFC00014602F07DF810F0020FF2D00020022195
:109C0C00024602F075F80020C6F30721024602F066
:109C1C006FF80020F1B2024602F06AF8002543E02A
:109C2C00013616F03F08795D01D1012204E0621E75
:109C3C00954214BF00220122002002F059F8B8F11D
:109C4C00000F30D1631E9D422DD20020052102460B
:109C5C0002F04EF800200122014602F049F810F003
:109C6C000100F2D10621012202F042F80020052168
:109C7C00024602F03DF800200122014602F038F8BD
:109C8C0010F0020FF2D000200221024602F030F850
:109C9C000020C6F30721024602F02AF80020F1B298
:109CAC00024602F025F80135A542B9D30020052162
:109CBC00024602F01DF800200122014602F018F8BD
:109CCC0010F0010FF2D1BDE8FC8100BF4902002069
:109CDC000058004037B5264B04461B780D46012B27
:109CEC0010D14FEA102C01A90322A53321488DF87D
:109CFC0004C08DF805408DF8065002F0D7F9FFF737
:109D0C0039FF33E000200621012201F0F1FF002091
:109D1C000521024601F0ECFF00200122014601F072
:109D2C00E7FF10F0020FF2D000200221024601F0F2
:109D3C00DFFF0020C4F30721024601F0D9FF002009
:109D4C00E1B2024601F0D4FF29460020012201F0C5
:109D5C00CFFF00200521024601F0CAFF002001229E
:109D6C00014601F0C5FF10F0010FF2D13EBD00BF5E
:109D7C00490200200058004038B5154B0C461B78A2
:109D8C00012B24D00725454305F5006528460978A5
:109D9C000135FFF79FFF284661780135FFF79AFFE1
:109DAC002846A1780135FFF795FF28462179013522
:109DBC00FFF790FF284661790135FFF78BFF2846A6
:109DCC00A179FFF787FF681CE179FFF783FF38BDA6
:109DDC0049020020194B70B5054618680C46FFF770
:109DEC00A3FD174B1B78834202D1164B1B78BBB1DA
:109DFC00124E00213068FFF76DFFFFF727FE124B64
:109E0C00294618682822FFF7C3FE104B2146186814
:109E1C006822FFF7BDFE0A4B30681978FFF75AFF2E
:109E2C00094B294618682822FFF730FD074B2146BD
:109E3C0018686822FFF72AFD70BD00BF0C000020D7
:109E4C0000000020D50300209C010020040000200D
:109E5C00084B9A7852B95B78142B05D8064A1168CE
:109E6C00064A42F8231004E0032200E00422044BCB
:109E7C001A7070476C030020D00300207C03002074
:109E8C00C0040020054B01205A7805498242087015
:109E9C0002D15A68034B1A60704700BF6C03002054
:109EAC00AC0400206C040020014B02221A70704795
:109EBC00AC040020074A00231360074A1370074ABA
:109ECC001360074A1360074A1370074A1360074A66
:109EDC001360704774030020AC0400206C04002055
:109EEC00B404002068030020D0030020F8040020F4
:109EFC00014B00221A707047AC04002030B5234B84
:109F0C005B78032B3ED8DFE803F008022F39204B97
:109F1C0018681E4B5C68002322E01D4A1368092B4D
:109F2C0007D81A491B484C68591C40F8234011604B
:109F3C002BE0092227E052F82350591CA5420ED1E0
:109F4C0002EB810204E052F8041C013342F8081CB5
:109F5C00411E04328B42F6D30D4B196015E00B46B3
:109F6C0083420C4AE7D310E0094A00231360094AE4
:109F7C00002199500433282BF9D106E0064B0A2214
:109F8C005A6002E00322044B1A7030BD6C030020AF
:109F9C00B004002070040020C0040020264A274B87
:109FAC005278092A3BD8DFE802F0050A0F141A226E
:109FBC00282E343720491A6849688A182EE01E4A20
:109FCC00196852688A1A29E01B4A196852684A4370
:109FDC0024E0194A1968526891FBF2F21EE0164A05
:109FEC001968526891FBF2F002FB101216E012494C
:109FFC001A68496801EA020210E00F491A684968B8
:10A00C0041EA02020AE00C491A68496881EA020234
:10A01C0004E01A68D24301E0074A52681A60074A02
:10A02C00074B12681AB91A6842F0080202E01A6863
:10A03C0022F008021A6070476C030020D003002045
:10A04C00740300202A4A2B4B52780A2A43D8DFE8A3
:10A05C0002F0060B11161C242A30363A3D00264914
:10A06C001A6809688A1803E0234A196812688A1A60
:10A07C001A6030E0204A196812684A43F8E71E4A11
:10A08C001968126891FBF2F2F2E71B4A1968126820
:10A09C0091FBF2F002FB1012EAE717491A68096803
:10A0AC0001EA0202E4E714491A68096841EA02026B
:10A0BC00DEE711491A68096881EA0202D8E70E4BFB
:10A0CC001A68D243D4E71A680B4BD1E70A4A1868CE
:10A0DC00116810601960074A084B12681AB91A689F
:10A0EC0042F0080202E01A6822F008021A60704777
:10A0FC006C030020D0030020F8040020740300201F
:10A10C00134B5B78052B22D8DFE803F003080D1204
:10A11C00171C104B1A6802F00F0217E00D4B1A684F
:10A12C0022F0100212E00B4B1A6822F020020DE014
:10A13C00084B1A6822F0400208E0064B1A6822F01D
:10A14C00800203E0034B1A6822F480721A60704795
:10A15C006C03002074030020124B1A68124B5B68CE
:10A16C009A4206DD114B196841F0040121F00301FC
:10A17C000CE00E4B05D1196821F0060141F00101EC
:10A18C0004E0196821F0070141F002011960074B46
:10A19C001AB91A6842F0080202E01A6822F00802A2
:10A1AC001A607047D00300206C0300207403002059
:10A1BC0010F0020F0CD111F0100F07D0064B042138
:10A1CC005A68064B1970064B1A6004E00A2200E02C
:10A1DC000822044B1A7070476C030020AC0400205A
:10A1EC0064030020C0040020014B00221A70704749
:10A1FC00AC0400200F4B5B78032B1AD8DFE803F07C
:10A20C00020413150C4B00E00C4B1A680C4B110A92
:10A21C0093F800C00B4B18780B4B1A7183F807C0DE
:10A22C009871597105E0094B00E0094B1A68064B0F
:10A23C005A6070476C030020640300206C040020FB
:10A24C00AC04002068030020C0040020D0030020D0
:10A25C00F8040020014B02221A707047D40300202E
:10A26C00024B5A68024B1A60704700BF6C03002007
:10A27C006C040020294B5B780C2B4ED8DFE803F0E4
:10A28C00070C11161C21262B30353A3F4400244B69
:10A29C001B6813F0080F3BE0214B1B6813F0080FF1
:10A2AC0008E01F4B1B6813F0010F31E01C4B1B68BF
:10A2BC0013F0010F31D12CE0194B1B6813F0040F74
:10A2CC0026E0174B1B6813F0050F21E0144B1B689D
:10A2DC0013F0020F1CE0124B1B6813F0030F17E076
:10A2EC000F4B1B6813F0100F12E00D4B1B6813F093
:10A2FC00200F0DE00A4B1B6813F0400F08E0084BD1
:10A30C001B6813F0800F03E0054B1B6813F4807F70
:10A31C0003D0024B5A68034B1A6070476C03002041
:10A32C00740300206C040020074970B50B68072BE0
:10A33C0009D8064A064816684068064D5C1C45F864
:10A34C0023600C60106070BDB40400206C0400200D
:10A35C006C0300204C040020054B1A6832B10549EF
:10A36C00013A51F822101A60034B1960704700BF74
:10A37C00B40400204C0400206C040020014B00228B
:10A38C001A707047AC040020084B9A784AB95A7876
:10A39C00142A04D85968064B43F8221004E003220F
:10A3AC0000E00422034B1A70704700BF6C030020BE
:10A3BC007C030020C0040020114B9A7852B95A78C3
:10A3CC00104B142A04D8104951F822205A6004E08A
:10A3DC00032201E00B4B04221A700C4B1B786BB15F
:10A3EC00084B0B495A680B4B0A601AB91A6842F0B1
:10A3FC00080202E01A6822F008021A60704700BFD7
:10A40C006C030020C00400207C030020A404002066
:10A41C00D00300207403002010B5094B9A7852B970
:10A42C005C78142C05D8FAF739F8064B43F824005D
:10A43C0004E0032200E00422034B1A7010BD00BF9D
:10A44C006C0300207C030020C004002038B5284B8E
:10A45C001B788BB9274A284B5268B2F1FF3F04BFD7
:10A46C00264A12680A214A431A6000F021F9244B4B
:10A47C00012218601E4B1A701E4B5C7814B1012C13
:10A48C0035D10EE000F014F91D4B1A681A4B821AE4
:10A49C00002A1B68B8BF52429A4224D9144B1C7034
:10A4AC0025E0FFF79DF910F4804507D0154B1049B6
:10A4BC001A68002022F01002087017E00E4C236876
:10A4CC008BB100F0F5F80E4A23681268821A002A44
:10A4DC00B8BF52429A4206D90A4B05491A680D7008
:10A4EC0042F0100202E0084B1A68013A1A6038BDBB
:10A4FC00680300206C030020FC080020D00300201F
:10A50C0098040020740300206C04002070B5104DDA
:10A51C00104E2868104C32787368B0F5006F62707A
:10A52C0063600FD83146FFF727FC31462868FFF7E8
:10A53C002FFA20B12B6801332B60652300E0072331
:10A54C00237004E007232370044B00221A7070BDA3
:10A55C00640300206C030020C0040020AC04002025
:10A56C0037B5124C657815B1012D1AD10FE0104B8F
:10A57C00042201A91868FFF789F96168019A0D4B4B
:10A58C00914202D101225A600EE05D600CE0A3788A
:10A59C002A2B06D1064B211D18680422FFF7F8FA66
:10A5AC0002E0044B03221A703EBD00BF6C03002076
:10A5BC0008000020C00400202DE9F3411E4B1F4C65
:10A5CC005B681F4A0125B3F5006F1570207027DCFE
:10A5DC0011EA050624D118466946FFF783FA9DF85F
:10A5EC0000809DF801709DF802C09DF807009DF851
:10A5FC0006109DF805209DF80430267284F8018021
:10A60C00A77084F803C020716171A271E3710B4BC8
:10A61C00E95C1A7A01358A18082D1A72F7D108E00C
:10A62C000123064A002199540133082BF9D11378E0
:10A63C001372BDE8FC8100BF6C030020D80300201E
:10A64C00D403002008B50A4B0A491A6802EA010132
:10A65C0069B95A6840F2D2439A4208D1064B18683D
:10A66C00FFF738FBFFF7F2F90120FFF7D9F808BD27
:10A67C006C03002000FFFF000C00002008B5034B0A
:10A68C001A68034B5A60FBF7A1F908BDD0030020F0
:10A69C006C03002008B5044B05201A68034B5A6064
:10A6AC00FBF7DCFA08BD00BFD00300206C030020D0
:10A6BC00014B1868704700BF1C03002008B50C4BF9
:10A6CC001B78012B01D1F9F79DFD042004F0DEF875
:10A6DC0048F6A04004F0EAF8012004F0EDF8054833
:10A6EC000321002204F080FD012004F0FBF808BDDA
:10A6FC00480200209AC3020008B5194B1A79EAB136
:10A70C001968184A013119601168174B0131116031
:10A71C00164A196812780131012A196005D1144BB7
:10A72C001A6812B11A68013A1A60124B1B78012B85
:10A73C0001D1F9F769FD0022094B00E001221A71E1
:10A74C000A4B1A78012A09D10B4B196831B11968D7
:10A75C00013919601B680BB9084B1A7008BD00BF92
:10A76C001C03002090090020880900204E000020C6
:10A77C00A409002048020020A00900209C09002008
:10A78C0043F2B60102B24A43494903144B434FF01A
:10A79C00020C991891FBFCF19A1A82B0002992FBD9
:10A7AC00FCF2019004DA002A2ADB002B6CDC04E0BA
:10A7BC00002A56DA002B47DC34E003F5E150801A0E
:10A7CC004FF4802190FBF1F000F5617080B200EB4A
:10A7DC006242A1F5003193FBF1F192B2511A89B2A8
:10A7EC00344BB3F820C02CF4005C4FEA0C4C4FEA0D
:10A7FC001C4CA3F820C098861A87998702B0704722
:10A80C0001F5E150801A4FF4802390FBF3F000F532
:10A81C006170A3F5003380B292FBF3F291FBF3F17C
:10A82C0082182EE0C3F5E150401880144FF400322A
:10A83C0000F5617091FBF2F180B2411A93FBF2F2D8
:10A84C0089B28A1892B2CBE703F5E150801A8014D2
:10A85C0000F561704FF4003180B292FBF1F2821876
:10A86C00B9E701F5E150801A4FF4802390FBF3F027
:10A87C0000F56170A3F5003380B291FBF3F100EBAE
:10A88C006242411A92B2AAE7C3F5E15040184FF464
:10A89C00802290FBF2F000F56170A2F5003291FB82
:10A8AC00F2F180B2411A89B201EB63439AB297E795
:10A8BC00E0E3FFFF002C0140064B00F5617001F551
:10A8CC00617102F5617280B289B292B29886198771
:10A8DC009A877047002C014037B501AD1A2300242C
:10A8EC0028468DF804308DF8074004F0AFFB28465D
:10A8FC0019238DF804308DF8074004F0A7FB0248AB
:10A90C0003F062FF3EBD00BF002C0140F0B5874B49
:10A91C008FB01C78012C07D12146402004F0C8FAD6
:10A92C0021464FF4006002E040F60C00012104F0D7
:10A93C00BFFA08AC7E4803F047FF204603F03AFB11
:10A94C004FF060024FF4E163214679484FF0000468
:10A95C00ADF822204FF48072ADF82430ADF82620EB
:10A96C00ADF820408DF8284003F0CCF9684603F090
:10A97C002BFB4FF07003ADF800306E4B4FF0010223
:10A98C001B78ADF802204FF00402ADF80420012B27
:10A99C0040F20552ADF8062010D14FF002034FF0F3
:10A9AC000802ADF80830ADF80A204FF480734FF46C
:10A9BC000072ADF80C30ADF80E200DE04FF0020334
:10A9CC00ADF80A304FF480724FF40073ADF80840C4
:10A9DC00ADF80C20ADF80E305548694603F0B4F9CB
:10A9EC005348694603F0F8F90DAC6946504803F03A
:10A9FC0043FA204604F0F2FE4C4B1978012916D18B
:10AA0C004D4804F031FF182321468DF837304FF4B0
:10AA1C007C52032349488DF83630ADF8342004F0CD
:10AA2C0093FE46484FF4285104F000FF15E018231C
:10AA3C008DF837300323424821468DF836304FF4D9
:10AA4C00E063ADF8343004F07FFE4EF20002214694
:10AA5C003C48ADF8342004F077FE354C08212046F4
:10AA6C0003F0E2FB2046082103F0E8FB2046082116
:10AA7C0003F0EEFB344B4FF480621B884FF0000563
:10AA8C00ADF816304FF4006304A92046ADF8103031
:10AA9C00ADF812204FF400534FF48042ADF81A3049
:10AAAC00ADF81C20ADF81450ADF8185003F06AFA4C
:10AABC002046012103F0C4FC01210A46204603F084
:10AACC00BFFA2046012103F0A1FB0121204603F02F
:10AADC0099FA0CAF4FF4A06004F0AEFA384604F0CB
:10AAEC00F7FA01261A230BA88DF82C308DF82D605F
:10AAFC008DF82E508DF82F6004F0A8FA19233846E3
:10AB0C008DF830308DF832508DF831608DF833601F
:10AB1C0004F09CFA2046314603F082FA4FF461733C
:10AB2C00A3862387A3870FB0F0BD00BF400200208F
:10AB3C00002C014052000020C000160000180140FB
:10AB4C0000080140000C014054000020024B1A6820
:10AB5C0001321A60704700BF341A00200028B8BFB9
:10AB6C00404240438B6DC9694FF0140C48430CFBB9
:10AB7C0003FC154B70B51A6844F620655C6890FBB5
:10AB8C00F5F5BCFBF1F064210132B0FBF1F02D19AD
:10AB9C0082421A605D6016DB9A680C4C501C90FB6C
:10ABAC00F1FC01FB1C01DE6854F822004FF47A7CA6
:10ABBC00B5FBFCF5361A76190020586044F8225083
:10ABCC00DE609960186070BD24030020381A0020E4
:10ABDC00014BD868704700BF24030020014B186854
:10ABEC00704700BF341A0020014B1860704700BF3B
:10ABFC00341A002008B5054B1B7C012B05D1044BE6
:10AC0C00044918680422FEF7C3FF08BD2403002082
:10AC1C00301A0020341A002008B5054B04221860A5
:10AC2C000449FEF733FE044B01221A7408BD00BF21
:10AC3C00301A0020341A002024030020014B18681D
:10AC4C00704700BFD01B0020014B1860704700BF3D
:10AC5C00D01B002008B5074B1B78012B09D1064BE4
:10AC6C00064918680422FEF793FFFFF721FD044BF9
:10AC7C00186008BD38030020CC1B0020D01B00201E
:10AC8C00C81B002038B50F4B1B78012B18D1FFF7D0
:10AC9C000FFD0D4C4EF65F222368C31A002BB8BF74
:10ACAC005B4293420CDD094B094A1D681068013563
:10ACBC00194604221D60FEF76BFFFFF7F9FC2060BC
:10ACCC0038BD00BF38030020C81B0020D01B00205B
:10ACDC00CC1B002008B5074B042218600649FEF770
:10ACEC00D5FDFFF7E5FC054B01221860044B1A70EB
:10ACFC0008BD00BFCC1B0020D01B0020C81B0020AF
:10AD0C0038030020014BB3F9000070473C030020CE
:10AD1C00884203D0164B4FF000021A8001380528E8
:10AD2C0022D8DFE800F00717030F0B13012916D008
:10AD3C00022912E0052912D003290EE004290ED0B5
:10AD4C0001290AE006290AD0052906E0022906D0C5
:10AD5C00042902E0032902D0062905D101E00120D3
:10AD6C0003E04FF6FF7000E0002000B2704700BF18
:10AD7C003C030020014B5860704700BF3C0300208F
:10AD8C00014B5868704700BF3C03002000F13B03A7
:10AD9C00762B10B50D4B0BD951430D4AB3F800C0AF
:10ADAC00800392FBF1F190FBF1F06044188002E01B
:10ADBC004FF000021A80054C0649B4F9000042F627
:10ADCC00AA2201F0C5FB208010BD00BF3C0300206F
:10ADDC00206CFBFF56D5FFFF012008B5FCF724FEC5
:10ADEC000138C0B2052801D9002002E0024B33F82B
:10ADFC00100000B208BD00BFDC0E010810B50B4CF2
:10AE0C0000222068022103F01BF920684FF44873DC
:10AE1C000385002103F060FB2068012103F0F2F8A8
:10AE2C0020680221012203F00BF910BD4000002024
:10AE3C000C4B07B51B78012B01D11B3304E00A4BDB
:10AE4C001B78012B02D11D338DF80430002301A88F
:10AE5C008DF8073004F0FAF8044B186803F0B4FCD2
:10AE6C000EBD00BF41020020440000204000002025
:10AE7C00F0B5694B89B01C780546012C16D12046DB
:10AE8C00214604F023F82146042006AC04F010F807
:10AE9C00204604F0A3FC03238DF81A3001338DF8FF
:10AEAC001B3021465D484FF0070335E05C4B1E78A4
:10AEBC00012E35D10420314604F008F8594B06AC6C
:10AECC001F78012F1AD13946202003F0F1FF2046BC
:10AEDC0004F084FC03238DF81A30013321468DF8DD
:10AEEC001B3051484FF4E043ADF8183004F02CFC03
:10AEFC0039464FF4805004F0B7FC11E0314608207D
:10AF0C0003F0D6FF204604F069FC482347488DF82F
:10AF1C001B3021464FF4E073ADF8183004F014FCEC
:10AF2C00434C03AE206803F04FFC304603F042F86C
:10AF3C004FF0FF3331462068ADF810304FF000036E
:10AF4C00ADF8123002F0DEFE684603F047F84FF021
:10AF5C000003ADF800304FF00203ADF802304FF0B3
:10AF6C000B0369462068ADF808304FF00303ADF8C9
:10AF7C00043003F0C5FB01224FF44871206803F044
:10AF8C00ADF8206803F07AF80121206803F066FA26
:10AF9C004021206803F0B0F80421206803F084FA03
:10AFAC000121206803F04CFA012D6E4628D11A4B72
:10AFBC001B78012B01D11B3304E0194B1B78012B9F
:10AFCC0002D11D338DF81C30194C012500230226AB
:10AFDC0007A88DF81E308DF81D608DF81F5004F0F9
:10AFEC0035F8206841F65F6103F0E0FA31462068DD
:10AFFC002A4603F025F8294620682A4603F020F853
:10B00C000B4C0021206803F067FA2068012102F044
:10B01C00F9FF09B0F0BD00BF41020020000801405B
:10B02C00440000204002002000140140000C0140AC
:10B03C0040000020014B1880704700BFD81B002037
:10B04C00014B1860704700BFD41B002010B504469C
:10B05C000846FFF7EFFF2046FFF7F2FF10BD00BFD9
:10B06C00014B1878704700BF44030020014B0022AD
:10B07C001A70704744030020014B1870704700BFD2
:10B08C0098010020014B1878704700BF98010020F0
:10B09C00704700BF034B1B781BB9034B80B21B6876
:10B0AC00988470474A02002048000020014B5860E9
:10B0BC00704700BF44030020014B5868704700BF25
:10B0CC00440300200549064B4A8909891B688A18E4
:10B0DC00B2FBF3F103FB112398B270474403002039
:10B0EC00D41B0020014B1881704700BF4403002083
:10B0FC0008B505200021012200F0BAFD054B801196
:10B10C001B7B1BB1044B1B68013B181A014B58816C
:10B11C0008BD00BF44030020D41B002008B5044B1D
:10B12C0001461B781BB9034B186803F0D5F908BD11
:10B13C004A0200204800002008B5054B1B7823B9B3
:10B14C00044B186803F024FA01E0034B588908BD3E
:10B15C004A020020480000204403002008B50E4B92
:10B16C001B7823B90D4B186803F012FA09E00C4B4D
:10B17C005A8918890B4B80181B68B0FBF3F203FB40
:10B18C001200084BC0EB00401A68074BB0FBF2F002
:10B19C001B88584380B208BD4A020020480000209A
:10B1AC0044030020D41B0020D81B002007B5184BEB
:10B1BC001B78012B2AD0174B1B78012B04D107339A
:10B1CC008DF80430143310E0134B1B78012B04D191
:10B1DC0016338DF80430063307E0104B1B78012B27
:10B1EC0014D116338DF8043007338DF8003001A8D4
:10B1FC0000238DF803308DF8073003F027FF6846E5
:10B20C0003F024FF064B186803F0DEFA0EBD00BFF6
:10B21C004A020020420200204C0000204302002081
:10B22C0048000020F0B58A4B8A4A1B788BB0012B62
:10B23C000D461173074600F00881874B1C78012CD2
:10B24C0018D12046214603F041FE2146042008ACCB
:10B25C0003F02EFE204604F0C1FA48238DF823306B
:10B26C0021464FF007037D48ADF8203004F06CFA0E
:10B27C001C233CE07A4B1C78012C1CD1022021466B
:10B28C0003F024FE08AE2146102003F011FE3046D8
:10B29C0004F0A4FA4823314672488DF823304FF459
:10B2AC00E073ADF8203004F04FFA21466E4804F0FC
:10B2BC00DBFA1D231BE06D4B1C78012C19D12146A8
:10B2CC00042003F003FE2146082008AC03F0F0FD37
:10B2DC00204604F083FA48238DF8233021464FF49E
:10B2EC00E0736348ADF8203004F02EFA1E238DF87D
:10B2FC0024300223002409A88DF82530013B8DF859
:10B30C0027308DF8264003F0A1FE5A4B013F1868F8
:10B31C0003F05AFA03A802F04DFE012D18BFADF848
:10B32C000E40ADF80C40ADF81240524C08BF102343
:10B33C0003A9206808BFADF80E30ADF8107002F00C
:10B34C00E1FC012D01D1002200E002220321134671
:10B35C00206802F0E5FE684602F040FE454B694667
:10B36C0018684FF00803ADF8083003F0C9F93A4BF0
:10B37C001B78012B02D14FF004030CE0384B1B78E7
:10B38C00012B02D14FF0080305E0384B1B78012B41
:10B39C0003D14FF00C03ADF80030364C69462068F1
:10B3AC0003F0AEF90121206803F000F901210A46EF
:10B3BC00206802F045FE20684FF0000301218384D1
:10B3CC0002F020FE244B1B78012B05D1002002211A
:10B3DC0004F078FA04230EE0214B1B78012B01D1E9
:10B3EC00022003E0214B1878012805D1082104F034
:10B3FC0069FA4FF480730693002308248DF81C30EF
:10B40C0006A801338DF81E308DF81D4004F002FBA8
:10B41C00114B1B78012B02D18DF824400AE0104B04
:10B42C001B78012B03D0114B1B78012B02D1163347
:10B43C008DF824300023012209A88DF826308DF8D0
:10B44C0027208DF8253003F001FE0BB0F0BD00BFB6
:10B45C004A02002044030020420200200008014060
:10B46C004C00002000100140000C1A004302002088
:10B47C00000C014048000020B0F90030B0F9022067
:10B48C0003FB03F102FB021110B50C4CA14214D9C1
:10B49C004FEA116CACF13A0C09495FFA8CFC31F8AB
:10B4AC001CC04FF4004102FB0CF203FB0CF392FBAB
:10B4BC00F1F293FBF1F14280018010BD0044FA3AA5
:10B4CC00E80E0108124B37B5B3F902C0B3F90010FE
:10B4DC00B0F90220B0F9000002FB0CF400FB01F5FE
:10B4EC0000FB0CFC4A434FF4004395FBF3F194FB37
:10B4FC00F3F492FBF3F264189CFBF3F3D31A0020E1
:10B50C00A2B262F30F009BB263F31F403EBD00BFBB
:10B51C0054030020A0F50040C0F3891000F44073E0
:10B52C00B3F5807F82B037D001DC23B305E0B3F5EF
:10B53C00007F05D0B3F5407F0FD00023184639E0CB
:10B54C00C0B21E4B420082F4FF7203EB4000D218D3
:10B55C00B0F88C00B2F88C302CE0184AC0B202EB78
:10B56C004003400080F4FF70B3F88C3082185B42CB
:10B57C00B2F88C000EE0114BC0B2420082F4FF72A4
:10B58C0003EB4000D218B0F88C00B2F88C3040427B
:10B59C005B4280B29BB20DE0C0B2084B420082F419
:10B5AC00FF72D218B2F88C2003EB40035242B3F86E
:10B5BC008C3090B243EA004002B07047E80E0108AC
:10B5CC0030B5044685B00846FFF7A4FFC0F30F431F
:10B5DC00ADF80230ADF80000134A00994FF4004367
:10B5EC001160B4F90210B2F90200B4F900C0B2F95A
:10B5FC00002001FB00F50CFB02F40CFB00F04A43AD
:10B60C0094FBF3F495FBF3F192FBF3F2641A90FBC9
:10B61C00F3F3D3180020A2B262F30F009BB263F3D2
:10B62C001F4005B030BD00BF54030020032903D8D0
:10B63C00DFE801F004081014002018E00D4B03EBB8
:10B64C00400004E040000B4B80F4FF70C018B0F8D1
:10B65C008C000CE0074B03EB400004E04000054B72
:10B66C0080F4FF70C018B0F88C00404280B200B279
:10B67C00704700BFE80E010883B244F6E6110014CF
:10B68C000FFA83FC484301FB0CF14FF4004291FB91
:10B69C00F2F190FBF2F290B24A42A2EB400200208F
:10B6AC0063F30F0092B284B062F31F4004B0704792
:10B6BC0030B585B06B4683E80300BDF90410BDF9C5
:10B6CC00020040F2C46202FB01F402FB00FCBDF973
:10B6DC0000506FF0020290FBF2F003236D0091FB1F
:10B6EC00F2F1091895FBF3F540F6B8339CFBF3FC2B
:10B6FC004A1994FBF3F3CCEB030392B2002062F3F0
:10B70C000F009BB263F31F4005B030BD30B50C4B3E
:10B71C000C4C844622681B689A4201D100200EE032
:10B72C002368094A5D1C02EB03130FCB8CE80F0056
:10B73C0025602368082B01D100232360012030BD34
:10B74C00681C0020DC1B0020E81B0020704700BF99
:10B75C007FB52B4B2B4A19681268914204D10120FA
:10B76C00002104F0B5FB48E01968274A02EB0111EF
:10B77C00487850B11B6802EB0312536804228DF811
:10B78C000C2000220192029307E01B68029002EB4E
:10B79C00031253688DF80C000193194B1A681A4B5D
:10B7AC0003EB02139B781BB102238DF80D3001E0E3
:10B7BC008DF80D30124B00221968134B0901CB5C2C
:10B7CC008DF80E300E4B0DF1180C18680CEB0201B5
:10B7DC0002EB001C0C4801326044007A082A01F884
:10B7EC00090CEFD11A6801321A601A68082A01D1C3
:10B7FC0000221A6001A804F079FB07B000BD00BF5D
:10B80C00E41B0020E01B00206C1C0020F0B54378EA
:10B81C0087B00646426833B104238DF80C30002300
:10B82C000292019303E0029301928DF80C30B378ED
:10B83C0003B102238DF80D30327800238DF80E20E1
:10B84C00F21801A8117AC2180133082BD172F7D162
:10B85C0004F04CFB042818D10D4D0E4B2C681B68C2
:10B86C000134082C08BF00249C4201D100200DE0BB
:10B87C0096E80F002F68084E06EB071C8CE80F00AB
:10B88C00012001462C6004F023FB012007B0F0BD21
:10B89C00E01B0020E41B00206C1C002030B5294D5F
:10B8AC00294B2C681B680134082C08BF00249C42CF
:10B8BC0087B043D001A904F0F5FB9DF80C20234B75
:10B8CC00042A09D12A68012103EB021251702A685B
:10B8DC0003EB0213029A08E02A68002103EB021220
:10B8EC0051702A6803EB0213019A5A609DF80D30CF
:10B8FC00144A022B154B04D1126803EB02130122DC
:10B90C0003E0126803EB021300229A700D4B9DF8B2
:10B91C000E101A680D4B1201D1540023094A06A9C6
:10B92C00C8181168094D03EB011110F8090C01330B
:10B93C004919082B0872F1D1146001E004F096FB50
:10B94C0007B030BD681C0020DC1B0020E81B002069
:10B95C0008B50120FFF7A2FF08BD00BF08B5002005
:10B96C00FFF79CFF08BD00BF2DE9F0470C238AB000
:10B97C008DF81C3003238DF81D30013800238DF811
:10B98C001B300C46154607281AD8DFE800F01613B2
:10B99C00100D0A1907044FF0020313E04FF00403D3
:10B9AC0010E04FF010030DE04FF014030AE04FF0DD
:10B9BC00280307E04FF0640304E04FF0C80301E0F4
:10B9CC004FF00803ADF81E3004F08CFC4FF0007003
:10B9DC00012103F07BFA0120014603F069FA0420EF
:10B9EC00012103F065FA0420002103F07DFA4FF4E5
:10B9FC00EA10002103F038FF0AAE4FF4805326F80A
:10BA0C00043D0323314667488DF8263015338DF8F5
:10BA1C00273003F099FE0423314662488DF8273015
:10BA2C004FF4006300260127ADF824301FFA84F888
:10BA3C0003F08AFE05A80DF1040A8DF81A608DF842
:10BA4C0014608DF815708DF816608DF817608DF8F0
:10BA5C0018708DF8197004F039F94FEA4813ADF8E5
:10BA6C00083050464FF0FF338DF804608DF80560B8
:10BA7C008DF80670ADF80A60ADF80C30ADF80E30EC
:10BA8C00ADF810608DF81270B14604F091F9BDB1AB
:10BA9C006B01ADF8083050464FF0FF338DF8056060
:10BAAC00ADF80A608DF812708DF804708DF8067080
:10BABC00ADF80C30ADF80E30ADF8107004F078F92C
:10BACC004FEAC80343F004030DF1040800270126D4
:10BADC0002226413ADF80A3040464FF0FF338DF864
:10BAEC000420ADF808408DF805708DF80660ADF8AF
:10BAFC000C30ADF80E30ADF810708DF8126004F00B
:10BB0C0057F9BD421BDDEB0043F004036D13032218
:10BB1C00ADF80A3040464FF0FF338DF804208DF815
:10BB2C000570ADF808508DF812608DF80660ADF810
:10BB3C000C30ADF80E30ADF8106004F039F908AFE8
:10BB4C00012407260025142338468DF820308DF863
:10BB5C0021608DF822508DF8234003F077FA1523DD
:10BB6C0038468DF820308DF821608DF822508DF8F4
:10BB7C00234003F06BFA132338468DF820308DF8F0
:10BB8C0021608DF822508DF8234003F05FFA0220DB
:10BB9C00214604F09DF92146102004F099F90AB0D1
:10BBAC00BDE8F0870008014030B52E4B87B01B78FC
:10BBBC000546012B03D1012801D12B4C00E02B4C65
:10BBCC002046002102F0ECFE4FF00003ADF80430EB
:10BBDC004FF48273ADF806304FF00003ADF8083027
:10BBEC004FF00203ADF80A304FF00103ADF80C3002
:10BBFC004FF40073ADF80E304FF00003ADF8123077
:10BC0C00ADF81430052D1ED8DFE805F00306061D2F
:10BC1C0009104FF0100318E04FF0080315E04FF433
:10BC2C000063ADF808304FF0100305E04FF40063EB
:10BC3C00ADF808304FF02803ADF810304FF000038A
:10BC4C00ADF80A3003E04FF01803ADF8103001A93D
:10BC5C00204602F069FE2046012102F0A1FE07B049
:10BC6C0030BD00BF440200200038004000300140CD
:10BC7C00F8B51D4D04462B780E468342174602D06C
:10BC8C00FFF792FF2C70042C05D0052C06D04CBB72
:10BC9C00FBF7EEFD04E0FBF72BFE01E0FBF72CFEBF
:10BCAC001248022102F010FF0028F9D031460F484B
:10BCBC0002F0AEFE0D48012102F006FF0028F9D07B
:10BCCC0067B1042C05D0052C06D05CB9FBF7D6FD6A
:10BCDC0004E0FBF70FFE01E0FBF710FE034802F057
:10BCEC0099FE00E00020F8BD580300200030014010
:10BCFC00F8B52D4D04462B780E468342174602D0DC
:10BD0C00FFF752FF2C70052C4CD8DFE804F003062B
:10BD1C00090C0F12FBF7ACFD0DE0FBF7DDFD0AE0A3
:10BD2C00FBF7DEFD07E0FBF7DFFD04E0FBF7E0FDD2
:10BD3C0001E0FBF7E1FD1D4B1B78012B03D1012C1E
:10BD4C0001D11B4D00E01B4D2846022102F0BCFE28
:10BD5C000028F9D03146284602F05AFE2846012127
:10BD6C0002F0B2FE0028F9D0BFB1052C1AD8DFE8DA
:10BD7C0004F00306090C0F12FBF780FD0DE0FBF736
:10BD8C00ADFD0AE0FBF7AEFD07E0FBF7AFFD04E00D
:10BD9C00FBF7B0FD01E0FBF7B1FD284602F03AFEDF
:10BDAC00C0B200E00020F8BD58030020440200207F
:10BDBC0000380040003001402DE9F041012186B0EF
:10BDCC004FF4805003F074F80120014605AF03F0E6
:10BDDC006FF8182403264FF0A00348483946ADF8F5
:10BDEC0014308DF816608DF8174003F0ADFC4FF051
:10BDFC00400342483946ADF814308DF816608DF882
:10BE0C00174003F0A1FC0120002103F02DFD4FF0A1
:10BE1C000003ADF800304FF48273ADF802304FF0F0
:10BE2C000003ADF804304FF00203ADF806304FF0CC
:10BE3C000103ADF808304FF4007331486946ADF892
:10BE4C000A304FF00003ADF80E30ADF81030ADF8FD
:10BE5C000C4002F069FD0121294802F0A1FD294B9B
:10BE6C00E8461D78012D42D14FF48040294603F05D
:10BE7C002DF84AF2000324483946ADF814308DF8F9
:10BE8C0016608DF8174003F05FFC4FF48043394681
:10BE9C001D48ADF814308DF816608DF8174003F07E
:10BEAC0053FC4FF00003ADF800304FF48273ADF843
:10BEBC0002304FF00003ADF804304FF00203ADF840
:10BECC0006304FF4007369461048ADF80A304FF055
:10BEDC000003ADF80C40ADF80850ADF80E30ADF8DD
:10BEEC00103002F021FD2946084802F059FD084B9C
:10BEFC004FF0FF321A7006B0BDE8F0810008014027
:10BF0C000030014044020020000C01400038004089
:10BF1C005803002082B000211C4A0191938A9BB2E5
:10BF2C000193019B13F4806F06D0938A23F48063F2
:10BF3C001B041B0C93820191019B13F4007F08D00E
:10BF4C00124A938A23F480631B041B0C93820023F4
:10BF5C000193019B13F4807F08D00C4A938A23F43D
:10BF6C0080731B041B0C938200230193019B13F41D
:10BF7C00006F08D0054A938A23F400631B041B0C42
:10BF8C0093820023019302B0704700BF005400401D
:10BF9C0082B000211C4A0191938A9BB20193019BB0
:10BFAC0013F4806F06D0938A23F480631B041B0C5C
:10BFBC0093820191019B13F4007F08D0124A938A5B
:10BFCC0023F480631B041B0C938200230193019BBD
:10BFDC0013F4807F08D00C4A938A23F480731B04DB
:10BFEC001B0C938200230193019B13F4006F08D068
:10BFFC00054A938A23F400631B041B0C93820023D1
:10C00C00019302B0704700BF0058004038B50D4690
:10C01C001F4C1946E3B91033A3601E4B6560984260
:10C02C00E2600AD110331C48236003F0FFFD1A486C
:10C03C00214603F0CBFD184826E0184B1848236026
:10C04C0003F0F4FD1648214603F0C0FD14481BE034
:10C05C00104B002198426560E260A1600AD1103358
:10C06C001048236003F0E2FD0E48214603F0AEFDBC
:10C07C000C4809E0094B0C48236003F0D7FD0A4833
:10C08C00214603F0A3FD0848012103F0CFFD38BD84
:10C09C00EC1C0020005400406C0002401058004082
:10C0AC0044000240800002405800024073B5002654
:10C0BC0001960096B0F804C004461FFA8CFC4CF4B0
:10C0CC00807CA0F804C01D4633464FF6FF760096E0
:10C0DC00FFF79CFFA3889BB243F40063A3802388E3
:10C0EC009BB243F48073238004E0009B5A1E0092A1
:10C0FC00002B46D0A38A13F0010FF6D0224B05F08B
:10C10C00FE054FF6FF7200921D701B78238204E02F
:10C11C00009B5A1E0092002B33D0A38A13F0020FFF
:10C12C00F6D0238B9BB20193184B9C420CD14FF44D
:10C13C00001003F093FD0028F9D01548002103F0FE
:10C14C0075FD4FF400100BE04FF4005003F086FD2A
:10C15C000028F9D00F48002103F068FD4FF400507F
:10C16C0003F08CFDA38A13F0040FFBD023889BB241
:10C17C0043F400732380238813F4007FFBD1012048
:10C18C0000E000207CBD00BF181D002000540040C2
:10C19C006C0002404400024037B500240194009426
:10C1AC00B0F804C004461FFA8CFC4CF4807C1D468D
:10C1BC00A0F804C00123FFF729FFA3889BB243F426
:10C1CC008053A380A3889BB243F40063A3804FF6F3
:10C1DC00FF73009323889BB243F48073238004E0A5
:10C1EC00009B5A1E0092002B42D0A38A13F0010F21
:10C1FC00F6D0204B45F001054FF6FF7200921D70F2
:10C20C001B78238204E0009B5A1E0092002B2FD037
:10C21C00A38A13F0020FF6D0238B9BB20193164B1B
:10C22C009C420CD14FF0007003F018FD0028F9D09F
:10C23C001248002103F0FAFC4FF000700BE04FF4B1
:10C24C00003003F00BFD0028F9D00D48002103F05D
:10C25C00EDFC4FF4003003F011FD23889BB243F446
:10C26C0000732380238813F4007FFBD1012000E0AE
:10C27C0000203EBD181D00200054004080000240EC
:10C28C005800024070B5012186B00646082002F025
:10C29C000FFE0120014602F0FDFD644B05AC9E42F1
:10C2AC0004AD28D14FF40010012102F00FFE03233E
:10C2BC008DF81630193321465D488DF817304FF044
:10C2CC004003ADF8143003F03FFA4FF080032146E1
:10C2DC005748ADF8143003F037FA4FF40010012131
:10C2EC0002F010FE4FF40010002102F00BFE284665
:10C2FC000123202227E04FF48000012102F0E6FD0B
:10C30C0003238DF816301933494821468DF8173020
:10C31C004FF48063ADF8143003F016FA4FF4006359
:10C32C0021464348ADF8143003F00EFA4FF4800068
:10C33C00012102F0E7FD4FF48000002102F0E2FD44
:10C34C002846012322228DF8102006228DF8133066
:10C35C008DF812308DF8112002F078FE334B002549
:10C36C009E4244F6206303934BF6FF73ADF8023004
:10C37C004FF48063ADF806304FF48043ADF80050B5
:10C38C00ADF8083069462B4C25D14FF028033046C8
:10C39C00ADF8043003F04CF9274803F0A7FB274B0A
:10C3AC00214623601023A3604FF6FF73E3608023C4
:10C3BC00636103F53E5320486362A56265602561A5
:10C3CC00A561E561256203F001FC1D4803F08EFBBD
:10C3DC0021461B4825E04FF0300369461948ADF85B
:10C3EC00043003F025F9184803F080FB174B214665
:10C3FC0023601023A3604FF6FF73E3608023636117
:10C40C0003F53E5310486362A56265602561A56122
:10C41C00E561256203F0DAFB0D4803F067FB0C487D
:10C42C00214603F0D3FB06B070BD00BF00540040A2
:10C43C00000C0140EC1C00206C0002401054004029
:10C44C008000024000580040440002401058004058
:10C45C005800024008B5FFF715FF08BD03464FF61C
:10C46C00FF70834246DDB3F1807F23DBB3F1805F45
:10C47C000FDBB3F1804F07DB334A934263DC334964
:10C48C001A168A5C12020FE030499A158A5CD201A6
:10C49C000AE0B3F1806F2D4A03DB1915525C92014F
:10C4AC0002E09914525C520193FBF2F101325218E2
:10C4BC00521019E0B3F5801F0BDBB3F5800F234A44
:10C4CC0003DB1914525C12010EE09913525CD2007A
:10C4DC000AE0B3F5802F1D4A03DB1913525C92005E
:10C4EC0002E09912525C520093FBF2F1501C40187E
:10C4FC0040101BE0FF2B1FDDB3F5805F0ADBB3F5AB
:10C50C00804F124A02DB1912505C0EE09911505CFC
:10C51C0040080AE0B3F5806F0C4A03DB1911505C3C
:10C52C00800802E09910505CC008013000FB00F25A
:10C53C009A4208DD013806E0002BA9BF034A4FF0F0
:10C54C00FF30D05C000970470080FE7F7411010839
:10C55C00904203DC8142ACBF0A460246104670474B
:10C56C0070B5044610460E4604F016FA05462946E8
:10C57C00204604F021FC40B9304604F00DFA054683
:10C58C002946204604F0FAFB00B12C46204670BD2B
:10C59C0070B514460E4604F0FFF90546204604F02B
:10C5AC00F7F904462146284604F0FEFA01462846CF
:10C5BC0004F03CF90546304604F0EEF9214604F04F
:10C5CC00F3FA0146284604F033F904F0FFFB70BD82
:10C5DC0070B51BB12D2301F8013B40424B1CB0FB45
:10C5EC00F2F402FB140C5D1EBCF1090F8CBF0CF1B4
:10C5FC00570C0CF1300C03F801CC1E4620460133CD
:10C60C00002CECD134702B780A7805F8012901F84C
:10C61C00013BA942F7D3304670BD00BF0A2A08B5CA
:10C62C00844613468E4603D1002801DA012303E029
:10C63C001A46604671460023FFF7CAFF08BD00BFCB
:10C64C00642303FB00F292FBF1F29A420BDD47F6F6
:10C65C00122359436FF00303584391FBF0F000F59C
:10C66C0074505C3019E012F1640F0BDA47F61223A8
:10C67C0059436FF00303584391FBF0F0A0F574504D
:10C68C005C380AE01C224B43424393FBF0F092FBD4
:10C69C00F1F1024B401893FBF0F0704700410F0092
:10C6AC00002908B502DDFFF7CBFF14E006D1002806
:10C6BC0011D0D4BF084843F65C500CE0002805DBD1
:10C6CC00FFF7BEFF00F5F440B83004E0FFF7B8FF09
:10C6DC00A0F5F440B83808BDA4C2FFFF014B1860A8
:10C6EC00704700BF405C0040014B186880B2704737
:10C6FC00405C0040014B1860704700BF445C004038
:10C70C00014B186880B27047445C0040014B1868BC
:10C71C0080B27047485C0040014B1860704700BF06
:10C72C004C5C0040014B186880B270474C5C004078
:10C73C004FF6F873024A00EA03031360704700BF18
:10C74C00505C0040014B186880B27047505C004050
:10C75C00014B43F820107047005C0040024B53F82B
:10C76C00200080B2704700BF005C0040054B10B544
:10C77C0053F8204048F68F1204EA02020A4343F8A9
:10C78C00202010BD005C0040024B53F8200000F448
:10C79C00C0607047005C00400A4B10B553F8202075
:10C7AC0048F6BF7402EA040411F0100F18BF84F0AD
:10C7BC00100411F0200F18BF84F0200443F820401F
:10C7CC0010BD00BF005C00400A4B10B553F8202090
:10C7DC004BF68F7402EA040411F4805F18BF84F4E2
:10C7EC00805411F4005F18BF84F4005443F82040C7
:10C7FC0010BD00BF005C004038B50D460446FFF785
:10C80C00ADFF012D02D120F4805003E0022D04D1A4
:10C81C0020F01000014B43F8240038BD005C0040B0
:10C82C00024B53F8200000F030007047005C0040D1
:10C83C00024B53F8200000F440507047005C00405D
:10C84C00054B48F6BF7253F8201001EA020282F041
:10C85C00300243F820207047005C0040054B4BF63B
:10C86C008F7253F8201001EA020282F4405243F80E
:10C87C0020207047005C0040054B48F68F6253F84F
:10C88C00201001EA020242F4807243F82020704723
:10C89C00005C0040044B48F68F6253F8201001EA0C
:10C8AC00020243F820207047005C0040044B48F61D
:10C8BC008F6253F8201001EA020243F820207047DF
:10C8CC00005C0040054B48F68F6253F8201001EADB
:10C8DC00020242F4807243F820207047005C004052
:10C8EC00054B48F68F6253F8201001EA020242F41D
:10C8FC00807243F820207047005C0040044B48F6DF
:10C90C008F6253F8201001EA020243F8202070478E
:10C91C00005C0040044B53F8200000F0300010285D
:10C92C0014BF002001207047005C0040054B53F8F9
:10C93C00200000F44050B0F5805F14BF00200120AF
:10C94C00704700BF005C0040044B40F68F7253F8F8
:10C95C00201001EA020243F820207047005C0040DE
:10C96C00044B48F60F7253F8201001EA020243F808
:10C97C0020207047005C0040054B48F68F7253F83E
:10C98C00201001EA020242F4804243F82020704752
:10C99C00005C0040054B48F68F7253F8201001EAFA
:10C9AC00020242F0400243F820207047005C004035
:10C9BC00084B53F8202012F4804F09D053F8201064
:10C9CC0048F68F7201EA020242F4804243F82020BA
:10C9DC00704700BF005C0040084B53F8202012F059
:10C9EC00400F09D053F8201048F68F7201EA02026A
:10C9FC0042F0400243F82020704700BF005C00402A
:10CA0C00054B10B553F8204048F68F7204EA020229
:10CA1C000A4343F8202010BD005C0040024B53F841
:10CA2C00200000F00F007047005C0040064B4908E6
:10CA3C001B6849009BB203EBC00303F1005303F5E1
:10CA4C0040535B0019607047505C0040054A064B30
:10CA5C001268490892B202EBC002D3185B0049007D
:10CA6C0019607047505C004004300020054B1B6877
:10CA7C009BB203EBC00303F1005303F540535B007F
:10CA8C0018887047505C0040044A054B126892B2FB
:10CA9C0002EBC002D3185B0018887047505C004052
:10CAAC0004300020044A054B126892B202EBC0021B
:10CABC00D3185B0019607047505C004002300020B6
:10CACC003E2909D94B0911F01F0F01D1013B9BB233
:10CADC009B0243F4004305E04B0811F0010F18BF13
:10CAEC0001339B02036070470D4A0E4B126892B2E1
:10CAFC00D31803EBC0035B003E2909D94A0911F096
:10CB0C001F0F01D1013A92B2920242F4004205E0A9
:10CB1C004A0811F0010F18BF013292021A607047D7
:10CB2C00505C004006300020054A064B126892B259
:10CB3C0002EBC002D3185B0018688005800D7047AB
:10CB4C00505C004002300020054A064B126892B23D
:10CB5C0002EBC002D3185B0018688005800D70478B
:10CB6C00505C0040063000200C4B30B51D681C6832
:10CB7C00C0001FFA85FC8444A4B2094B00190CF1C7
:10CB8C00005CC3180CF5405C490852084FEA4C0095
:10CB9C0049005B00520001601A6030BD505C0040DF
:10CBAC0004300020064B49081B6849009BB203EB7C
:10CBBC00C00303F1005303F540535B001960704749
:10CBCC00505C0040054A064B1268490892B202EBD1
:10CBDC00C002D3185B00490019607047505C0040DC
:10CBEC0004300020054B1B689BB203EBC00303F120
:10CBFC00005303F540535B0018887047505C0040AD
:10CC0C00044A054B126892B202EBC002D3185B00C7
:10CC1C0018887047505C004004300020012910B582
:10CC2C0024D1254B25491B68C0009BB25918091803
:10CC3C004B003E2A09D9510912F01F0F01D10139BD
:10CC4C0089B2890241F4004105E0510812F0010F4C
:10CC5C0018BF0131890219601749194B096889B24B
:10CC6C00CB18181840003E2A1ED913E0022922D1F5
:10CC7C00114BC0001C681B68A4B21FFA83FC0F493F
:10CC8C000F4B844400194118634449005B000A604F
:10CC9C001A6010E0530912F01F0F01D1013B9BB237
:10CCAC009B0243F4004305E0530812F0010F18BF38
:10CCBC0001339B02036010BD505C00400230002029
:10CCCC000630002001291BD11349144B096889B285
:10CCDC00CB1803EBC00040003E2A09D9530912F0CF
:10CCEC001F0F01D1013B9BB29B0243F4004305E0B3
:10CCFC00530812F0010F18BF01339B0203600AE0C6
:10CD0C00022908D10449054B096889B201EBC0001E
:10CD1C00C3185B001A607047505C00400230002062
:10CD2C0001291BD11349144B096889B2CB1803EBA9
:10CD3C00C00040003E2A09D9530912F01F0F01D13F
:10CD4C00013B9BB29B0243F4004305E0530812F0F5
:10CD5C00010F18BF01339B0203600AE0022908D1BE
:10CD6C000449054B096889B201EBC000C3185B008C
:10CD7C001A607047505C004006300020054A064B94
:10CD8C00126892B202EBC002D3185B0018688005DF
:10CD9C00800D7047505C004002300020054A064B65
:10CDAC00126892B202EBC002D3185B0018688005BF
:10CDBC00800D7047505C0040063000200D4BC000C9
:10CDCC0019680D4A89B241188A185200128812F457
:10CDDC007C4F01D001200CE01A68084B92B28018ED
:10CDEC00C3185B0018888005800D002814BF022032
:10CDFC0000207047505C00400630002002300020BC
:10CE0C00012909D10B4A48F68F7352F8201001EA18
:10CE1C00030343F040030AE002290AD1054A48F60D
:10CE2C008F7352F8201001EA030343F4804342F855
:10CE3C0020307047005C004041EA0020704700BF82
:10CE4C00030AC0B243EA0020704700BF01F1005151
:10CE5C00013201F5405110B549005208002308E099
:10CE6C0010F803C06478013A4CEA042C21F813C082
:10CE7C000233C418002AF3D110BD00BF01F10051D8
:10CE8C00013201F5405110B549005208002304E06D
:10CE9C0031F81340013AC4520233002AF8D110BDC4
:10CEAC0008B529E047F6FF700860198801F00F01FA
:10CEBC008B0003F18043117003F5B843196889B2F4
:10CECC0011F4004F09D0186840F68F7100EA010187
:10CEDC00196012780E4B013A0BE011F0800F0BD059
:10CEEC00186848F60F7100EA010119601278094BB5
:10CEFC00013A53F8223098470749084B0868084A0A
:10CF0C0080B21880188800B20028CBDB08BD00BFA7
:10CF1C004C01002030010020445C0040AA09002094
:10CF2C00B2090020F8B59AE047F6FF761E60168825
:10CF3C00564F06F00F06B30003F1804303F5B843D8
:10CF4C003E70002E64D127682668236807F4405C85
:10CF5C0003EA000080F400502060236806F03000E3
:10CF6C0003EA010181F0200121601388484A13F083
:10CF7C00100F1080A5F800C004D023689BB213F0EA
:10CF8C00800F08D0226848F60F7302EA030323606F
:10CF9C0000F0CEFA16E013F4006F08D0226840F6C9
:10CFAC008F7302EA0303236000F062FB0AE013F4C0
:10CFBC00004F54D0226840F68F7302EA03032360BB
:10CFCC0000F0F8F921682A884BF68F7301EA030305
:10CFDC0012F4805F18BF83F4805312F4005F2D4A63
:10CFEC0018BF83F400531360294B11681A8848F654
:10CFFC00BF7301EA030312F0100F18BF83F0100384
:10D00C0012F0200F234A18BF83F0200313603BE07B
:10D01C001C68A4B214F4004F0BD0196840F68F7240
:10D02C0001EA02021A603A781B4B013A53F822309B
:10D03C00984714F0800F12D0144948F60F720B78F1
:10D04C009B0003F1804303F5B843186800EA020221
:10D05C001A600A78114B013A53F822309847104B5A
:10D06C00104A1D680B4C1FFA85FCA2F800C0B2F8E0
:10D07C0000C04BF68F700FFA8CFCBCF1000F48F619
:10D08C00BF71094DFFF650AFF8BD00BFB2090020CB
:10D09C001C1D0020005C00404C01002030010020D1
:10D0AC00445C0040AA0900201A1D0020074A0221F6
:10D0BC0008B5074811720749074B086007490A6011
:10D0CC00074A13601B68984708BD00BFB8090020C9
:10D0DC006C010020D40900209C000020180A0020BC
:10D0EC00AC09002010B5074C20B922684FF00103A1
:10D0FC00138205E0044B1B681B68984720680A30B4
:10D10C0010BD00BF180A0020D409002010B50A4B2E
:10D11C000A4A1B685178DA7891420AD3997841B956
:10D12C009C8834B99A72064B1B685B6898472046FA
:10D13C0000E0022010BD00BF180A0020680100208A
:10D14C00D409002010B5074C20B922684FF0010318
:10D15C00138205E0044B1B689B68984720680C30D1
:10D16C0010BD00BF180A0020D409002038B50E4CA1
:10D17C000E4B22681B68D1789B69507998472368BD
:10D18C009A7A7AB170B91A7962B99D7855B9084B07
:10D19C001B68DB689847236828465979DA78D97276
:10D1AC001A7300E0022038BD180A0020AC090020D8
:10D1BC00D409002008B50246244B20B91B684FF057
:10D1CC000201198240E0224A4FF000011B681180D5
:10D1DC00197811F07F0113D15B7A13F0200F03D073
:10D1EC00117841F00201117013F0400F184B15BF6C
:10D1FC001A781A7822F0010242F001021A701EE02D
:10D20C00012921D0022901D000221DE0597911F009
:10D21C00800F01F00F0306D00E4951F8233003F0B4
:10D22C003003102B06E00B4951F8233003F4405324
:10D23C00B3F5805F03D1137843F001031370064BF1
:10D24C001B681B699847024A104608BD180A002043
:10D25C00201D0020005C0040D409002010B51E4B9E
:10D26C0019684A7912F0800F22F0800305D01B4810
:10D27C0050F8230000F0300004E0184850F8230068
:10D28C0000F44050164C94F800C0634522D24C88F0
:10D29C0004BBF8B1897AE9B112F0800F09D00F49BB
:10D2AC0048F6BF7251F8230000EA020282F0100225
:10D2BC0008E00A494BF68F7251F8230000EA02028B
:10D2CC0082F4805241F82320064B1B689B699847D7
:10D2DC00002000E0022010BD180A0020005C004075
:10D2EC0068010020D409002008B5064B1B685A7A47
:10D2FC0042F020025A72044B1B68DB6998470020ED
:10D30C0008BD00BF180A0020D4090020054B1A687C
:10D31C00538A18B98988CB1A138201E00868181847
:10D32C00704700BF180A002030B50E4B1C78002344
:10D33C0010E05FFA83FC4FEA8C0202F1804202F5A6
:10D34C00B842156848F68F7105EA010141EA0C01F3
:10D35C0011600133A342ECD3034B40F08000186002
:10D36C0030BD00BF680100204C5C0040704700BF1E
:10D37C0008B50C4B002093F82C10FFF7B5FB0A4BAB
:10D38C001B68187A082807D1084B4FF480521A8072
:10D39C00074B4FF010021A80092814BF00200120FF
:10D3AC0008BD00BF9C000020180A00201A1D002098
:10D3BC001C1D002070B52D4B1C68237A032B01D04B
:10D3CC00052B46D1A369228AABB1A2B1A58A95429D
:10D3DC0028BF154628469847228A638A521BEB18A9
:10D3EC000646228263820020FFF74EFB2A46014646
:10D3FC003046FFF743FD238A5BB11D4B4FF440527F
:10D40C0000201A800146FFF74DFB1A4B4FF03002FB
:10D41C001A80A28A238A9A4203D8144B03221B68CF
:10D42C0003E0124A1BB1136805221A720DE0126850
:10D43C0006211172104A1168104A89B28A185200DA
:10D44C0013600C4B4FF030021A80084B1B681B7A90
:10D45C0006E0072B03D10A4B1B68DB6898470823AF
:10D46C00024A12681372FFF783FF70BD180A00207E
:10D47C001A1D00201C1D0020505C004002300020B2
:10D48C00AC090020F8B5244B1C68238A267ABBB95A
:10D49C00042E15D1214822490278012A0BD1214CA6
:10D4AC00214A24680370A0B28218520013604FF016
:10D4BC0030020A802BE04FF010030B80072626E089
:10D4CC00A68AA2699E4234BF35461D462846B34201
:10D4DC0094BF04260226904707460020FFF7C6FAA1
:10D4EC002A4601463846FFF7B1FC29460020FFF7D3
:10D4FC00D9FA638A228AEB186382094B551B4FF0C9
:10D50C00300225821A80094B4FF440521A80024B8C
:10D51C001B681E72F8BD00BF180A002059030020BA
:10D52C001C1D0020505C0040023000201A1D002001
:10D53C0008B5144B1B681A7A022A01D0042A05D1AB
:10D54C00FFF7A0FF0F4B1B681B7A14E0062A11D1C2
:10D55C005A78052A0AD11A7812F07F0F06D1D8789A
:10D56C00FFF7E2FE084B1B681B6A9847074B1B68CA
:10D57C009B6898470823034A12681372FFF7F8FE5A
:10D58C0008BD00BF180A0020D4090020AC090020F7
:10D59C0038B5324B1B68187810F07F0004D15A7ADA
:10D5AC0022F020025A7258E0022855D15A88002ADB
:10D5BC0052D11A79002A4FD15A7912F0800F22F0E9
:10D5CC00800405D0264951F8241001F0300104E004
:10D5DC00234951F8241001F4405122480078844228
:10D5EC003AD2002938D09B7A002B35D012F0800F1C
:10D5FC000FD01B4B53F8243003F03003102B25D1E4
:10D60C00E4B22046FFF7E8F920463021FFF7C4F8D2
:10D61C001CE0134D55F8243003F44053B3F5805FF0
:10D62C0014D134B9104B204693F82C10FFF75CFA48
:10D63C0002E02046FFF7BCF955F824204BF68F7317
:10D64C0002EA030383F4405345F82430074B1B686C
:10D65C005B699847002000E0022038BD180A0020C2
:10D66C00005C0040680100209C000020D4090020D0
:10D67C00F7B58D4B8D4E1A6835688D4B92B2D31819
:10D68C002A7A5B00092A1B681BD09BB203F100535A
:10D69C0003F540535B001C4614F8012B03F10A07F9
:10D6AC002A705B786B70B4F80300FFF7C9FB6880D5
:10D6BC00B4F807003468FFF7C3FBA08033687F8899
:10D6CC00DF807A4C01212368DA8819725D78002A90
:10D6DC0062D11A7812F07F022ED1092D02D1FFF7F8
:10D6EC0015FD3BE0052D0DD193F90320002A4EDBEF
:10D6FC009A78002A4BD19A88002A48D19B7A002B21
:10D70C0037D044E0032D0BD1DA78012A27D19A883F
:10D71C002ABB5B7A13F0200F21D0FFF7E5FD1DE04B
:10D72C00012D1CD1DA78012A19D19A88BAB95B7A01
:10D73C0013F0200F13D00AE0012A04D10B2D0ED1C7
:10D74C00FFF714FD0AE0022A09D1012D02D1FFF7DF
:10D75C001FFF03E0032D02D1FFF780FD48B1554BAD
:10D76C0028461B685B699847032801D109230FE001
:10D77C0068B94D4A504B12684FF0300192B2D31831
:10D78C005B0000221A604D4B1980062300E0082331
:10D79C00464A12681372E3E0062D18D11A7812F07B
:10D7AC007F0F40F097809B78012B03D1414B1B6876
:10D7BC00DB696EE0022B03D13E4B1B681B6A68E0F1
:10D7CC00032B40F087803B4B1B685B6A61E0002DAC
:10D7DC003CD1598800297DD15A6822F47F42B2F598
:10D7EC00003F77D11A7812F07F0203D19B88002B6F
:10D7FC0070D129E0012A0BD158792E4B1B689B69FB
:10D80C009847002866D123689B7A002B62D01BE0D6
:10D81C00022A5FD15B7913F0800F03F00F0205D061
:10D82C00274951F8221001F0300104E0244951F845
:10D83C00221001F440512348007882424AD213F05E
:10D84C00700F47D1002945D01F4B23E0082D05D17F
:10D85C001B7813F07F0F3DD11C4B1BE00A2D39D1E7
:10D86C001A7802F07F02012A34D19A7A002A31D038
:10D87C00598800292ED15A6822F47F42B2F5803F94
:10D88C0028D158790B4B1B689B69984710BB104BE0
:10D89C0000E0FBB1054A4FF00001126800209361D3
:10D8AC0051829847002020E0505C0040180A00206C
:10D8BC0004300020AC090020023000201C1D002088
:10D8CC00005C004068010020C1D10008F1D00008C4
:10D8DC0051D10008244C254B22681B6850781B69D9
:10D8EC009847032801D1236806E01F4B4FF6FF71C0
:10D8FC001B681A8A8A4201D1092203E0022800D04F
:10D90C0012B908221A722BE093F90010002921DABF
:10D91C00D98801910198824202D9019A1A8211E0A8
:10D92C008A420FD21149096891F82C108A4201D20F
:10D93C00002105E092FBF1F001FB102212B901214C
:10D94C000B4A1170094A126892F82C209A82FFF740
:10D95C0099FD05E003221A72064B4FF440521A80CF
:10D96C00FFF706FDFEBD00BF180A0020AC09002021
:10D97C00590300201A1D0020002383814FF41652F6
:10D98C008380C38003814FF00C0302604381704796
:10D99C000A8810B54C88B1F804C0038AC98844EAD7
:10D9AC00020242EA0C0223F470630A431B041B0CB0
:10D9BC0092B242EA0303038210BD00BF0023C3806E
:10D9CC00038043808380704721B183899BB243F4E9
:10D9DC00005304E0838923F400531B041B0C838144
:10D9EC00704700BF01F01F034FF0010CC1F342114F
:10D9FC0061450CFA03F301D10C3004E0022901D18A
:10DA0C00103000E014301AB1026842EA030302E05D
:10DA1C00026822EA03030360704700BF1AB1838ACD
:10DA2C009BB2194303E0838A9BB223EA01018182F2
:10DA3C00704700BF038A23F00F031B041B0C0382E7
:10DA4C00038A9BB241EA030303827047838923F460
:10DA5C0000631B041B0C838183899BB241EA030383
:10DA6C008381704721B183899BB243F0020304E0A8
:10DA7C00838923F002031B041B0C8381704700BFB6
:10DA8C00038A23F020031B041B0C0382038A9BB222
:10DA9C0041EA03030382704721B1038A9BB243F42A
:10DAAC00804304E0038A23F480431B041B0C038291
:10DABC00704700BFC905C90D818070478088C005BB
:10DACC00C00D704783899BB243F00103838170477B
:10DADC00038BDBB20383038B9BB243EA01230383E7
:10DAEC00704700BF038B03F47F430383038B9BB20C
:10DAFC0041EA03030383704721B1838A9BB243F04D
:10DB0C00200304E0838A23F020031B041B0C838274
:10DB1C00704700BF21B1838A9BB243F0100304E02D
:10DB2C00838A23F010031B041B0C8382704700BFF5
:10DB3C0021B1838A9BB243F0080304E0838A23F06B
:10DB4C0008031B041B0C8382704700BF838A23F0DD
:10DB5C0004031B041B0C8382838A9BB241EA0303DC
:10DB6C008382704721B1838A9BB243F0020304E0A5
:10DB7C00838A23F002031B041B0C8382704700BFB3
:10DB8C00038819420CBF002001207047C94389B299
:10DB9C00018070474FF0010CC1F3421201F01F03DA
:10DBAC0062450CFA03F301D1828903E0022A0CBF0F
:10DBBC00028A828A92B21340028892B20BB918463A
:10DBCC0007E0090A012313FA01F111420CBF0020EE
:10DBDC0001207047090A01238B40DB439BB2038071
:10DBEC00704700BF038ACA8823F440531B041B0CE4
:10DBFC001343038283898A8830B5044608890D460D
:10DC0C0023F4B053498940EA020223F00C030A437F
:10DC1C001B041B0C92B242EA0303A381A38AAA89B8
:10DC2C0023F440731B041B0C134387B0A38201A87D
:10DC3C0001F0E8F80E4B2A689C420CBF049B039B36
:10DC4C001921594392006423B1FBF2F1B1FBF3F2B9
:10DC5C001201100903FB101109013231B1FBF3F36E
:10DC6C0003F00F0343EA020292B2228107B030BDE7
:10DC7C000038014008B5214B98422BD008D8A3F5A9
:10DC8C000063984216D003F58063984234D119E0B2
:10DC9C001B4B984226D003F5684398422CD10121A6
:10DCAC004FF4804001F020F94FF48040002101F046
:10DCBC001BF921E04FF40030012101F023F94FF45E
:10DCCC00003016E04FF48020012101F01BF94FF4D5
:10DCDC0080200EE04FF40020012101F013F94FF4E5
:10DCEC00002006E04FF48010012101F00BF94FF4F5
:10DCFC008010002101F006F908BD00BF004C004067
:10DD0C0000500040038803F08F0303800388B1F8B0
:10DD1C0006C04A889BB243EA0C0313439BB20380B0
:10DD2C008B8883850B880385064B984203D003F5BB
:10DD3C000063984201D10B7A03864FF00103838272
:10DD4C00704700BF002C0140038C2DE9F04123F0FB
:10DD5C0001031B041B0C0384038C0A894C8823F0DD
:10DD6C0002031C4E14431B048288B1F806C0058BB9
:10DD7C001B0CA4B2B04244EA030392B20C88ADB2BD
:10DD8C00A0F834C003D006F50066B04218D18E89D5
:10DD9C004F89B1F80E804FF6F77C03EA0C0C4CEA75
:10DDAC00070748EA06064FF6FB73898847F6FF4CCF
:10DDBC0002EA0C0C07EA0303B2B20B4342EA0C0270
:10DDCC004FF68F7105EA01012143828001830384A0
:10DDDC00BDE8F081002C0140038C2DE9F04123F0CB
:10DDEC0010031B041B0C0384028CB1F808C022F036
:10DDFC00200212048488120C4B8842EA0C1242EA6C
:10DE0C000313A2B21B4C068BB1F806C0A0420D88BE
:10DE1C00B6B29BB2A0F838C003D004F50064A0429F
:10DE2C001BD1B1F80A804FF67F748F8903EA040482
:10DE3C0047F2FF3C02EA0C0C44EA0814CA894FF67C
:10DE4C00BF73898804EA03034CEA870C43EA011385
:10DE5C004CEA82023C469BB292B248F6FF7106EA4B
:10DE6C00010141EA052189B2828001830384BDE866
:10DE7C00F08100BF002C0140038C2DE9F04123F40C
:10DE8C0080731B041B0C0384028CB1F808C022F4B1
:10DE9C00007212048488120C4B8842EA0C2242EA6B
:10DEAC000323A2B21A4C868BB1F806C0A0420D888F
:10DEBC00B6B29BB2A0F83CC003D004F50064A042FB
:10DECC001BD1B1F80A804FF2FF748F8903EA040466
:10DEDC0044F6FF7C02EA0C0C44EA0824CA894FF68B
:10DEEC00FF33898804EA03034CEA071C43EA012345
:10DEFC004CEA02123C469BB292B24FF68F7106EA84
:10DF0C0001012943828081830384BDE8F08100BF35
:10DF1C00002C0140038CF0B523F480531B041B0C24
:10DF2C000384B1F806C0078C0C8882880D89868B17
:10DF3C004B88A0F840C0DFF848C0BFB2604592B231
:10DF4C00B6B203D00CF5006C604505D192048989FA
:10DF5C00920C42EA811292B24DF6FF7C07EA0C0C4D
:10DF6C0048F6FF7106EA01014CEA053C41EA04213E
:10DF7C004CEA033389B29BB2828081830384F0BD67
:10DF8C00002C0140B1F802C00B888A884CEA0303CC
:10DF9C00B1F806C013430A8943EA0C03B1F80AC06E
:10DFAC0013438A8943EA0C0313439BB2A0F8443011
:10DFBC00704700BF00234FF0FF3203724380828012
:10DFCC000380C380704700BF0023C381038043805C
:10DFDC008380C380038143818381704700234FF08A
:10DFEC0001020381038043808280C380704700BF9D
:10DFFC0000238381038043808380C380038143811A
:10E00C00704700BF21B103889BB243F0010304E0C9
:10E01C00038823F001039B059B0D0380704700BF11
:10E02C0039B1B0F844306FEA43436FEA53439BB2C3
:10E03C0003E0B0F844305B045B0CA0F8443070474C
:10E04C001AB183899BB2194303E083899BB223EAFB
:10E05C0001018181704700BF818270470A43A0F89B
:10E06C00482070471AB183899BB2194303E0838916
:10E07C009BB223EA01018181704700BF038923F021
:10E08C0007031B041B0C0381704700BFB0F808C0CA
:10E09C005FFA8CFC41EA0C0C42EA0C0C4CEA032CA7
:10E0AC001FFA8CFCA0F808C0704700BF10B50446DE
:10E0BC00FFF7ECFF23899BB243F48043238110BD0F
:10E0CC0010B50446FFF7E2FF238923F077031B0406
:10E0DC001B0C43F07703238110BD00BF01858282A6
:10E0EC00704700BF038823F070039B059B0D41EA2A
:10E0FC0003030380704700BF038923F070031B04E4
:10E10C001B0C41EA03030381704700BF10B50446A2
:10E11C00FFF7F2FF23899BB243F00703238110BD65
:10E12C0030B50489B0F818C0058C2CF4407CADB225
:10E13C002CF0030C24F007044FEA0C4C25F02205BC
:10E14C0042EA050524044FEA1C4C45EA0315240C4D
:10E15C004CF4807C21434CF0010CADB20181A0F851
:10E16C0018C0058430BD00BF038B23F070031B0463
:10E17C001B0C41EA03030383704700BF038B23F49A
:10E18C00E0431B041B0C43EA01239BB2038370473F
:10E19C00838B23F070031B041B0C41EA0303838362
:10E1AC00704700BF838B23F4E0431B041B0C43EA32
:10E1BC0001239BB28383704721B103889BB243F048
:10E1CC00800304E0038823F080039B059B0D0380F0
:10E1DC00704700BF21B183889BB243F0040304E075
:10E1EC00838823F004031B041B0C8380704700BF3F
:10E1FC0021B183889BB243F0080304E0838823F0A9
:10E20C0008031B041B0C8380704700BF21B183885B
:10E21C009BB243F0010304E0838823F001031B0449
:10E22C001B0C8380704700BF038B23F008031B0477
:10E23C001B0C41EA03030383704700BF038B23F4D9
:10E24C0000631B041B0C43EA01239BB2038370473E
:10E25C00838B23F008031B041B0C41EA0303838309
:10E26C00704700BF838B23F400631B041B0C43EA31
:10E27C0001239BB283837047038B23F004031B049D
:10E28C001B0C41EA03030383704700BF038B23F489
:10E29C0080631B041B0C43EA01239BB2038370476E
:10E2AC00838B23F004031B041B0C41EA03038383BD
:10E2BC00704700BF838B23F480631B041B0C43EA61
:10E2CC0001239BB283837047038B23F080031B04D1
:10E2DC001B0C41EA03030383704700BF038B5B04F1
:10E2EC005B0C43EA01239BB203837047838B23F0BF
:10E2FC0080031B041B0C41EA03038383704700BF9C
:10E30C00838B5B045B0C43EA01239BB283837047D2
:10E31C00038C23F002031B041B0C41EA030303844C
:10E32C00704700BF038C23F008031B041B0C41EA4D
:10E33C0003030384704700BF038C23F020031B04EA
:10E34C001B0C43EA01139BB203847047038C23F02C
:10E35C0080031B041B0C43EA01139BB2038470471C
:10E36C00038C23F400731B041B0C43EA01239BB2A4
:10E37C0003847047038C23F400631B041B0C43EAD7
:10E38C0001239BB203847047038C23F400531B04BA
:10E39C001B0C43EA01339BB20384704701238B406F
:10E3AC008A40018C89B221EA03030384018C0A435D
:10E3BC0092B20284704700BF04238B408A40018CC8
:10E3CC0089B221EA03030384018C0A4392B20284CA
:10E3DC00704700BF01238B40B0F820C010B51FFA66
:10E3EC008CFC2CEA0303038409B1082909D11830E9
:10E3FC00490844584FF68F7304EA030343504358BB
:10E40C000CE004391830C1F34E01445848F6FF7340
:10E41C0004EA030343501202435892B243EA020245
:10E42C00425010BD21B103889BB243F0020304E0BB
:10E43C00038823F002039B059B0D0380704700BFEC
:10E44C0021B103889BB243F0040304E0038823F05A
:10E45C0004039B059B0D0380704700BF21B183888B
:10E46C009BB243F0800304E0838823F080031B04F9
:10E47C001B0C8380704700BF038823F008039B05A7
:10E48C009B0D038003889BB241EA03030380704712
:10E49C00838823F070031B041B0C838083889BB23E
:10E4AC0041EA030383807047038923F007031B04AD
:10E4BC001B0C038103899BB241EA03030381704760
:10E4CC00038923F080031B041B0C038103899BB27B
:10E4DC0041EA03030381704781847047818570474B
:10E4EC00818670470187704781877047A0F840107C
:10E4FC00704700BF038B23F00C031B041B0C03831E
:10E50C00038B9BB241EA030303837047038B23F411
:10E51C0040631B041B0C0383038B9BB243EA012354
:10E52C009BB20383704700BF838B23F00C031B0447
:10E53C001B0C8383838B9BB241EA03038383704759
:10E54C00838B23F440631B041B0C8383838B9BB250
:10E55C0043EA01239BB28383704700BF0388DBB27D
:10E56C00038003889BB241EA03030380704700BF1A
:10E57C00808E80B2704700BF008F80B2704700BFA2
:10E58C00808F80B2704700BFB0F8400080B27047F7
:10E59C00808C80B2704700BF008D80B2704700BF86
:10E5AC00038A19420CBF002001207047C94389B26D
:10E5BC0001827047038A828911EA030092B203D068
:10E5CC0011420CBF00200120704700BFC94389B223
:10E5DC0001827047B0F820C010B52CF0010C4FEA46
:10E5EC000C4C4FEA1C4CA0F820C0048BB0F820C097
:10E5FC00A4B21FFA8CFC24F0F30442EA04042CF0BD
:10E60C00020C44EA03144CF0010C4CEA010CA4B2C9
:10E61C000483A0F820C010BDB0F820C010B52CF0B9
:10E62C00100C4FEA0C4C4FEA1C4CA0F820C0B0F870
:10E63C0018C0048C2CF4407CA4B24FEA0C5C4FEA5A
:10E64C001C5C24F020044CEA022C44F010044CEA2C
:10E65C00033C44EA01141FFA8CFCA4B2A0F818C0C5
:10E66C00048410BD38B50D46602D1146044603D107
:10E67C000122FFF7D1FF02E00122FFF7ABFF294691
:10E68C002046FFF739FD23899BB243F00703238112
:10E69C0038BD00BFF8B50C46A2884988B4F800C054
:10E6AC00054600290CBF02270027012A0CBF0226B1
:10E6BC0001262389BCF1000F10D1FFF78BFF2846F0
:10E6CC00E188FFF717FF2846394632462389FFF7C2
:10E6DC00A3FF2846E188FFF719FF0FE0FFF79CFF27
:10E6EC002846E188FFF712FF28463946324623892F
:10E6FC00FFF770FF2846E188FFF7FCFEF8BD00BF6E
:10E70C0038B50B880C4605464BB94988A288238935
:10E71C00FFF760FF2846E188FFF7ECFE53E0042B7F
:10E72C0009D14988A2882389FFF776FF2846E1881A
:10E73C00FFF7ECFE47E0082BB1F802C0B1F804E09B
:10E74C00098920D1028C22F480721204120C0284EA
:10E75C00838B028C9BB292B223F0F30322F40072EF
:10E76C0043EA011142EA0C2C89B21FFA8CFC41EAF3
:10E77C000E0E4CF4807CA0F81CE0A0F820C0E188C0
:10E78C00FFF7D2FE1FE0028C22F480521204120C0E
:10E79C000284838B028C23F4407392B21B051B0DF5
:10E7AC0022F4005243EA0E2342EA0C3C43EA0133C2
:10E7BC001FFA8CFC9BB24CF4805C8383A0F820C0C5
:10E7CC00E188FFF7BDFE38BD08B52D4B984237D018
:10E7DC000BD8A3F50063984226D003F580639842CA
:10E7EC0028D0B0F1804F4AD118E0264B984233D054
:10E7FC0004D8A3F58063984241D127E0224B98427C
:10E80C0004D003F50063984239D12EE04FF4006038
:10E81C00012100F069FB4FF400602DE0012001465E
:10E82C0000F070FB01201CE00220012100F06AFBCB
:10E83C00022016E00420012100F064FB042010E00B
:10E84C000820012100F05EFB08200AE010200121C5
:10E85C0000F058FB102004E02020012100F052FBB6
:10E86C002020002100F04EFB09E04FF40050012164
:10E87C0000F03AFB4FF40050002100F035FB08BDCE
:10E88C00000C004000140040002C0140042804D16E
:10E89C00054B1A6842F0040203E0034B1A6822F09D
:10E8AC0004021A60704700BF10E000E0014B586092
:10E8BC00704700BF10E000E0012804D1084B1A6833
:10E8CC0042F0010206E010F1020F05D1044B1A6868
:10E8DC0022F001021A6002E0014B00229A6070479C
:10E8EC0010E000E020B1054B1A6842F0020203E090
:10E8FC00024B1A6822F002021A60704710E000E026
:10E90C00014B9868704700BF10E000E0C308022B71
:10E91C000BBF044B034B1B68DB6833FA00F000F0B1
:10E92C000100704710E000E00B884A88B1F804C081
:10E93C001A43CB8842EA0C02B1F808C01A434B893F
:10E94C0030B542EA0C028D89B0F800C0CC891A436C
:10E95C002A4322430CF4415313439BB20380838B11
:10E96C0023F400631B041B0C83830B8A038230BDCE
:10E97C0000234FF00702C38102820380438083800F
:10E98C00C380038143818381704700BF002343818F
:10E99C00038043808380C3804FF002030381704760
:10E9AC0021B103889BB243F0400304E0038823F0B9
:10E9BC0040031B041B0C0380704700BF21B1838BE9
:10E9CC009BB243F4806304E0838B23F480631B04C9
:10E9DC001B0C8383704700BF0909012313FA01F153
:10E9EC0089B21AB183889BB2194303E083889BB226
:10E9FC0023EA0101818070471AB183889BB21943C5
:10EA0C0003E083889BB223EA01018180704700BF39
:10EA1C0081817047808980B2704700BF4FF6FF63D9
:10EA2C00994205D003889BB243F48073038002E0C3
:10EA3C00038819400180704721B183889BB243F051
:10EA4C00040304E0838823F004031B041B0C838061
:10EA5C00704700BF038823F400631B041B0C038066
:10EA6C0003889BB241EA03030380704703889BB27F
:10EA7C0043F480530380704721B103889BB243F465
:10EA8C00005304E0038823F400531B041B0C038085
:10EA9C00704700BF012914BF008B808A80B2704779
:10EAAC00008A80B2704700BFB1F5804F04D1038853
:10EABC009BB243F4804304E0038823F480431B049B
:10EACC001B0C0380704700BF038919420CBF002048
:10EADC0001207047202906D1038903889BB243F09B
:10EAEC004003038008E0402901D0082901D10389A3
:10EAFC0002E0C94389B20181704700BF012301F0D4
:10EB0C000F0213FA02F2B0F804C000891FFA8CFC51
:10EB1C0080B2104006D009098B401CEA030F0CBFD1
:10EB2C0000200120704700BF552906D103890388B6
:10EB3C009BB243F0400303800DE0562901D05329CA
:10EB4C0001D1038907E001F00F01012313FA01F150
:10EB5C00C94389B201817047838BF0B523F47A6382
:10EB6C0023F01F031B041B0C83834FF0020303844D
:10EB7C000B89868B022B87B004460D46B6B201D1A9
:10EB8C00002225E001A88F8800F03CF9EB88002FCB
:10EB9C000CBF01270227B3F5007F2989019A06D102
:10EBAC00A3F5FB7353430902B3FBF1F305E00A230E
:10EBBC0049015A434F43B2FBF7F305330A229BB288
:10EBCC00B3FBF2F303F001021202C3F34F0392B250
:10EBDC00991E89B2FE2928BF002228BF0223E9888A
:10EBEC0042EA03030B439BB223842B886A8846EAD0
:10EBFC000303A98843F4006313436A890B4313434B
:10EC0C009BB2A38307B0F0BD08B5154B98421BD03F
:10EC1C0003F57443984204D0A3F5784398421DD170
:10EC2C000AE001214FF4805000F05EF94FF480505F
:10EC3C00002100F059F911E04FF48040012100F05F
:10EC4C0061F94FF4804006E04FF40040012100F0E0
:10EC5C0059F94FF40040002100F054F908BD00BFF1
:10EC6C00003C00400D4B0E4A196841F0010119603F
:10EC7C00596801EA02025A601A6822F0847222F47E
:10EC8C0080321A601A6822F480221A605A6822F4C0
:10EC9C00FE025A6000229A60704700BF00100240CA
:10ECAC000000FFF80C4BB0F5803F1A6822F480325C
:10ECBC001A601A6822F480221A6003D0B0F5802FF3
:10ECCC0008D103E01A6842F4803202E01A6842F478
:10ECDC00A0221A60704700BF00100240034B1A6854
:10ECEC0022F0F80242EAC0021A607047001002409B
:10ECFC00014B1860704700BF00004242044B5A6839
:10ED0C0022F47C1240EA02020A435A60704700BFA8
:10ED1C0000100240014B1860704700BF6000424277
:10ED2C00034B5A6822F0030240EA02025A60704711
:10ED3C0000100240024B586800F00C00704700BFF6
:10ED4C0000100240034B5A6822F0F00240EA020223
:10ED5C005A60704700100240034B5A6822F4E0627C
:10ED6C0040EA02025A60704700100240034B5A6896
:10ED7C0022F4605242EAC0025A607047001002400E
:10ED8C0019B1054B1A78104303E0034B1A7822EAA9
:10ED9C0000001870704700BF09100240014B18604A
:10EDAC00704700BFD8004242034B5A6822F44042DD
:10EDBC0040EA02025A60704700100240064B0022E3
:10EDCC0001281A701A7002D0042804D101E01870BE
:10EDDC0001E005221A70704720100240014B1860A8
:10EDEC00704700BF80044242024B1A6A40EA02029A
:10EDFC001A62704700100240014B1860704700BF48
:10EE0C003C0442421F4B10B55A6802F00C02042A13
:10EE1C0013D0082A11D15A685968C2F383420232BE
:10EE2C0011F4803F03D05B6813F4003F01D0164B04
:10EE3C0000E0164B5A43026001E0144B0360114A88
:10EE4C00134B51680468C1F30311595C34FA01F196
:10EE5C0041605468C4F3022C13F80C4031FA04F4EA
:10EE6C0084605468C4F3C22C13F80CC021FA0CF162
:10EE7C00C1605268C2F381329B181B7CB1FBF3F169
:10EE8C00016110BD0010024000093D0000127A0023
:10EE9C007412010819B1054B5A69104303E0034B76
:10EEAC005A6922EA00005861704700BF0010024006
:10EEBC0019B1054B9A69104303E0034B9A6922EA96
:10EECC0000009861704700BF0010024019B1054B5B
:10EEDC00DA69104303E0034BDA6922EA0000D861D7
:10EEEC00704700BF0010024019B1054BDA6810439F
:10EEFC0003E0034BDA6822EA0000D860704700BFD9
:10EF0C000010024019B1054B1A69104303E0034B82
:10EF1C001A6922EA00001861704700BF0010024015
:10EF2C00014B1860704700BF40044242014B18600F
:10EF3C00704700BF4C004242014B1870704700BF35
:10EF4C00071002404309012B02D1084B1B6805E056
:10EF5C00022B0BBF054B054B1B6A5B6A00F01F00B5
:10EF6C0033FA00F000F00100704700BF00100240BF
:10EF7C0008B53120FFF7E6FF094B18705A680132CB
:10EF8C005A601A7822B95A6840F2FF139A42F0D1AB
:10EF9C003120FFF7D7FF003818BF012008BD00BF94
:10EFAC005C030020024B5A6A42F080725A6270472E
:10EFBC0000100240034B9B6818420CBF002001203C
:10EFCC00704700BF00100240014B1870704700BF23
:10EFDC000A1002400B4B4FF0FF316FF07042C3F838
:10EFEC008010C3F88420C3F88011C3F88421002357
:10EFFC0003F1C001034A013300200F2B42F821001A
:10F00C00F6D1704700E100E0094B4FF020605860EA
:10F01C00084800224FF0FF319A60D8601A615A619B
:10F02C009A61DA611A625A629962D96219637047FD
:10F03C0000ED00E00000FA0540F0BE60024B40F429
:10F04C002020D860704700BF00ED00E030B5C278DA
:10F05C0003787AB31C4A4178D2684FF00F0CD24334
:10F06C00C2F302222CFA02FCC2F104029140807815
:10F07C0003F003020CEA000C4CEA010CD2004FEA3C
:10F08C000C1CFF2090400CFA02FC012403F01F0220
:10F09C00944099080D4AC03152F821500CEA000CEA
:10F0AC0025EA00004CEA00005B0942F8210042F816
:10F0BC00234008E003F01F02012191405B09034A41
:10F0CC00203342F8231030BD00ED00E000E100E0F9
:10F0DC000023C3700370437083707047024B5868F1
:10F0EC00C0F30930704700BF00ED00E0012200F0D2
:10F0FC001F0312FA03F34009044A403052F820006F
:10F10C001840984214BF00200120704700E100E035
:10F11C00014B1860704700BF00EF00E000F01F03C8
:10F12C0001229A404009024B603043F8202070477E
:10F13C0000E100E0024B58688005800D704700BF6D
:10F14C0000ED00E0012200F01F0312FA03F3400966
:10F15C00044A803052F820001840984214BF002016
:10F16C000120704700E100E0014B1868704700BFB8
:10F17C0000ED00E021F0604121F07F01014B0143E3
:10F18C009960704700ED00E0014A024BDA6070476D
:10F19C000400FA0500ED00E0014A024BDA6070470A
:10F1AC000100FA0500ED00E019B1054B1A69104396
:10F1BC0003E0034B1A6922EA00001861704700BF94
:10F1CC0000ED00E000F01F00012313FA00F019B16C
:10F1DC00044B5A6A104303E0024B5A6A22EA0000BD
:10F1EC005862704700ED00E0144B70B5DC684FF0CE
:10F1FC00FF0CE443C4F302242CFA04F5C4F1040418
:10F20C0011FA04F4C0F30126F6000CFA06FC02EA2B
:10F21C00050545EA0404240114FA06F6C0F381102E
:10F22C00063053F8202022EA0C0243F8202053F831
:10F23C002020164343F8206070BD00BF00ED00E0B5
:10F24C00C0F3832001238340044A506A03EA000080
:10F25C00984214BF00200120704700BF00ED00E071
:10F26C0000F01F0001228240024B59680A435A6089
:10F27C00704700BF00ED00E000F01F020123013ACF
:10F28C0013FA02F2024B59680A435A60704700BFE6
:10F29C0000ED00E0C0F3833001238340044A506A40
:10F2AC0003EA0000984214BF00200120704700BF01
:10F2BC0000ED00E0C0F3814313B90A4BD86A10E0AB
:10F2CC00012B0CD1074AC0F30153906ADA00D040ED
:10F2DC00022B14BF00F00F0000F0FF0001E0014B07
:10F2EC00186B704700ED00E010F4800F0BBF024B61
:10F2FC00014B586B986B704700ED00E008B5F4F7C4
:10F30C002FFF08BD08B50001F4F727FF08BD00BFAB
:10F31C0008B5F4F720FF08BD08B5F4F71AFF08BDCF
:10F32C0008B5F4F714FF08BD08B5F4F70EFF08BDD7
:10F33C00002341F28832C260C38003804BF6FF7217
:10F34C0083804FF4804342800381704721B103884E
:10F35C009BB243F0010304E0038823F001031B0478
:10F36C001B0C0380704700BF21B183889BB243F410
:10F37C00006304E0838823F400631B041B0C83806C
:10F38C00704700BF21B183889BB243F4805304E0E3
:10F39C00838823F480531B041B0C8380704700BFAD
:10F3AC0021B103889BB243F4807304E0038823F4F7
:10F3BC0080731B041B0C0380704700BF21B10388B2
:10F3CC009BB243F4007304E0038823F400731B0422
:10F3DC001B0C0380704700BF21B103889BB243F420
:10F3EC00806304E0038823F480631B041B0C0380FC
:10F3FC00704700BF838901F0FE019BB223F0FE032E
:10F40C0041EA03038381704721B183899BB243F0A6
:10F41C00010304E0838923F001031B041B0C83818B
:10F42C00704700BF21B103889BB243F0400304E056
:10F43C00038823F040031B041B0C0380704700BFA0
:10F44C001AB183889BB2194303E083889BB223EAE9
:10F45C0001018180704700BF01827047008AC0B2F1
:10F46C00704700BF12B141F0010101E001F0FE0153
:10F47C000182704782B0019B0190CB5A98B202B0C6
:10F48C00704700BF31B103886FEA43436FEA5343BF
:10F49C009BB202E003885B045B0C0380704700BFE7
:10F4AC00B1F5005F04D103889BB243F4005304E030
:10F4BC00038823F400531B041B0C0380704700BF0C
:10F4CC0021B103889BB243F4805304E0038823F4F6
:10F4DC0080531B041B0C0380704700BFB1F5006FF9
:10F4EC0004D103889BB243F4006304E0038823F443
:10F4FC0000631B041B0C0380704700BF21B1038801
:10F50C009BB243F0200304E0038823F020031B0488
:10F51C001B0C0380704700BF008BC0F307207047A3
:10F52C0021B103889BB243F0100304E0038823F05D
:10F53C0010031B041B0C0380704700BF21B9038808
:10F54C009BB243F0800304E0038823F080031B0488
:10F55C001B0C0380704700BFB1F5804F05D0838B27
:10F56C0023F480431B041B0C03E0838B9BB243F4FA
:10F57C0080438383704700BF828A038B90B240EA3A
:10F58C00034020F07F407047828A038B90B240EAA0
:10F59C00034020F07F40884214BF002001207047B8
:10F5AC00838A028B9BB243EA02430B4023F07F40D9
:10F5BC00003818BF012070470B0F012B03D1C94332
:10F5CC0089B281820EE0022B01D1838A0AE0062BDC
:10F5DC0006D1838A03889BB243F00103038001E0C8
:10F5EC00838A038B704700BF838A028B9BB243EAEA
:10F5FC0002430B4023F07F40003818BF01207047B6
:10F60C000B0F012B03D1C94389B281820EE0022B6F
:10F61C0001D1838A0AE0062B06D1838A03889BB228
:10F62C0043F00103038001E0838A038B704700BF22
:10F63C0070B586B00446868801A80D46FFF7E2FB3C
:10F64C000399304826F03F063604B1FBF0F0360C37
:10F65C0080B240EA0606A6802288EB6822F00102FE
:10F66C001204120C2280284A93420AD85B00B1FB88
:10F67C00F3F301309BB280B22084032B98BF042398
:10F68C0023E0B5F802C04BF6FF72944505D1032276
:10F69C005343B1FBF3F39BB206E019225343B1FB86
:10F6AC00F3F39BB243F480431A05120D0AB943F0ED
:10F6BC0001034FF49672504302F52F7290FBF2F057
:10F6CC00013080B2208443F40043A38323889BB28F
:10F6DC0043F0010323802388E98823F480632A887C
:10F6EC0023F00A031B0441EA02021B0C13439BB2D6
:10F6FC0023802B89AA8842EA03039BB2238106B09C
:10F70C0070BD00BF40420F00A086010008B50D4B34
:10F71C00984204D003F58063984212D107E04FF46D
:10F72C0000100121FFF7EEFB4FF4001006E04FF440
:10F73C0080000121FFF7E6FB4FF480000021FFF76A
:10F74C00E1FB08BD00540040CB78F0B513F0100F6E
:10F75C0018BF8A78098803F00F0C18BF4CEA020C0A
:10F76C0011F0FF0F1AD0046800220126964006EA19
:10F77C000105B5420ED196000F27B7400CFA06F6DC
:10F78C0024EA07043443282B01D1456102E0482BBD
:10F79C0008BF05610132082AE7D10460FF291CD992
:10F7AC004468002202F108050126AE4006EA010574
:10F7BC00B5420ED196000F27B7400CFA06F624EA94
:10F7CC0007043443282B01D1456102E0482B08BFC4
:10F7DC0005610132082AE5D14460F0BD0423C370F1
:10F7EC00022383704FF0FF33038070478368194204
:10F7FC000CBF002001207047806880B2704700BFAA
:10F80C00C36819420CBF002001207047C06880B249
:10F81C00704700BF01617047416170470AB10161D7
:10F82C0000E04161704700BFC160704741F4803314
:10F83C00836181618361836983697047064A10B56E
:10F84C0014684FF6807341EA001104EA030341EA9D
:10F85C000303136010BD00BF00000140014B186092
:10F86C00704700BF1C0020420304154A00F4401CE2
:10F87C001B0CBCF5401F30B5546806D1556824F0FC
:10F88C00706425F07065556011E010F4801F06D08F
:10F89C00C0F303424FF0030C0CFA02F203E0420DEA
:10F8AC00120113FA02F224EA020444F0706419B152
:10F8BC00400D000183401C43014B5C6030BD00BF18
:10F8CC000000014001F003039B000F229A4010FA44
:10F8DC0003F310B58908074C023154F8210020EAD3
:10F8EC00020244F8212054F82120134344F821301B
:10F8FC0010BD00BF000001400120014608B5FFF714
:10F90C00F3FA01200021FFF7EFFA08BD08B5264BEA
:10F91C0098422BD00CD8A3F5006398421AD003F56B
:10F92C00806398421CD0A3F5006398423AD10BE057
:10F93C001E4B984226D003F58063984228D0A3F53D
:10F94C00006398422ED117E004200121FFF7CCFA76
:10F95C00042024E008200121FFF7C6FA08201EE04D
:10F96C0010200121FFF7C0FA102018E020200121FF
:10F97C00FFF7BAFA202012E040200121FFF7B4FA79
:10F98C0040200CE080200121FFF7AEFA802006E039
:10F99C004FF480700121FFF7A7FA4FF4807000211B
:10F9AC00FFF7A2FA08BD00BF00140140001C014083
:10F9BC00044B1A6802F038021A601A6840EA020214
:10F9CC001A60704700200240044B1A6822F00802AB
:10F9DC001A601A6840EA02021A607047002002405E
:10F9EC00044B1A6822F010021A601A6840EA0202EC
:10F9FC001A60704700200240044B00221A605A60C3
:10FA0C009A60DA60024A5A61704700BF00040140F4
:10FA1C00FFFF0700837930B5016802794BB3184BAF
:10FA2C00CC431D6890F805C004EA05051D605D68AF
:10FA3C002C405C60D45844EA0101D15002689868AB
:10FA4C00D14301EA00009860D8680140BCF1100F66
:10FA5C00D96007D1996811439960D96841EA0202CB
:10FA6C00DA600BE05CF8031041EA02024CF8032068
:10FA7C0004E0034BD05820EA0101D15030BD00BF47
:10FA8C000004014000230C22837142710360037156
:10FA9C00704700BF024B1A6940EA02021A617047B4
:10FAAC0000040140034B5B6918420CBF002001208D
:10FABC00704700BF00040140014B5861704700BF04
:10FACC0000040140054B1A685B69034001D11846DC
:10FADC0003E010420CBF00200120704700040140DD
:10FAEC00014B5861704700BF0004014002680023BD
:10FAFC0022F001020260036043608360C3602D4BFF
:10FB0C00984233D011D83C3B984229D006D8283B98
:10FB1C00984221D0143398424BD11FE0264B984287
:10FB2C0020D01433984244D11EE0244B98422CD060
:10FB3C0008D8A3F5677398421DD003F562739842F9
:10FB4C0037D11DE01E4B984229D0143398422BD04C
:10FB5C00283B98422DD11DE01A4B12E0194B15E0B1
:10FB6C00184B18E0174B1BE0164B1EE0154B5A6850
:10FB7C0042F470021CE0134B5A6842F0706217E0BA
:10FB8C00114B5A6842F00F0212E00F4B5A6842F0C8
:10FB9C00F0020DE00C4B5A6842F4706208E00A4B1C
:10FBAC005A6842F4704203E0074B5A6842F47022E0
:10FBBC005A6070476C000240440002401C04024032
:10FBCC004404024000000240000402408A6870B500
:10FBDC000C6A0B6944EA02024C691A438B69224392
:10FBEC00CC6905684E6A42EA030323438C6A3343AB
:10FBFC0025F4FE4C23432CF0F00C43EA0C03036079
:10FC0C00CB6843600B6883604B68C36070BD00BFFA
:10FC1C0000238362036043608360C36003614361BC
:10FC2C008361C36103624362704700BF19B103680B
:10FC3C0043F0010302E0036823F001030360704703
:10FC4C0012B10368194302E0036823EA0101016061
:10FC5C00704700BF406880B2704700BF10F0805FF3
:10FC6C0014BF044B044B1B6803420CBF0020012043
:10FC7C00704700BF000402400000024010F0805F9B
:10FC8C0014BF024B024B5860704700BF0004024087
:10FC9C000000024010F0805F14BF044B044B1B6843
:10FCAC0003420CBF00200120704700BF000402403B
:10FCBC000000024010F0805F14BF024B024B5860F2
:10FCCC00704700BF0004024000000240374B012285
:10FCDC001A605A6812F0010201D1104664E00278F1
:10FCEC00012A0BBF1A681A6842F0800222F08002C7
:10FCFC001A604378012B04D12C4B1A6842F0400255
:10FD0C0003E02A4B1A6822F040021A608378012B18
:10FD1C0004D1264B1A6842F0200203E0234B1A68E8
:10FD2C0022F020021A60C378012B04D11F4B1A68F1
:10FD3C0042F0100203E01D4B1A6822F010021A6008
:10FD4C000379012B04D1194B1A6842F0080203E025
:10FD5C00164B1A6822F008021A604379012B04D161
:10FD6C00124B1A6842F0040203E0104B1A6822F09E
:10FD7C0004021A608279C37990F808C0920742EAAB
:10FD8C0003624189437A42EA0C4242EA0352013946
:10FD9C00064B0A43DA611A6822F001021A605868AD
:10FDAC0080F0010000F00100704700BF00640040CB
:10FDBC0090F800C0012202FA0CF23B4B2DE9F04501
:10FDCC00D3F8004292B244F00104C3F80042D3F8D5
:10FDDC001C42D14301EA0404C3F81C428478A4B940
:10FDEC000CF1480CD3F80C72B0F80AA0C688B0F825
:10FDFC00088085884FEACC0404F1804446EA0A4620
:10FE0C0045EA084501EA070715E0012C1AD10CF167
:10FE1C00480CD3F80C72B0F804A0C688B0F808806F
:10FE2C0045894FEACC0404F1804446EA0A4645EA87
:10FE3C00084542EA070704F5C844C3F80C7243F8B6
:10FE4C003C60656043782BB9174BD3F8044201EA48
:10FE5C00040404E0144BD3F8044242EA0404C3F84B
:10FE6C000442838923B9104BD3F81442214006E095
:10FE7C00012B06D10C4BD3F8141242EA0101C3F842
:10FE8C001412837B012B05D1074BD3F81C120A43A8
:10FE9C00C3F81C22044BD3F8002222F00102C3F851
:10FEAC000022BDE8F08500BF00640040032202720E
:10FEBC00013A002342724FF00102C3714281037078
:10FECC0043708370C370037143718371704700BFBB
:10FEDC0019B1054B5A69104303E0034B5A6922EAE6
:10FEEC0000005861704700BF00640040364B70B58D
:10FEFC009968024611F0806F01D000200CE09968DF
:10FF0C0011F0006F01D0012006E09B6813F0805FB8
:10FF1C0001D1042056E002202B4B00F118010901FD
:10FF2C00CC5804F00104CC50157A92F809C035B9BC
:10FF3C00146864051460CD584CEA050C07E054684D
:10FF4C0045EA0C0CE4005460CE584CEA060C4CEA22
:10FF5C000404CC50947A00F1180C4FEA0C1C04F0F9
:10FF6C000F040CF18043947203F5C8435D680101E2
:10FF7C0025F00F055D605D6801F180412C435C60EC
:10FF8C00537B947BD57A1B0443EA0463147B2B4389
:10FF9C0043EA042301F5C841C1F88831557C937CB0
:10FFAC00D47B2D0445EA0365137C45EA040242EA3E
:10FFBC000322054BC1F88C215CF8032042F00102AE
:10FFCC004CF8032070BD00BF00640040012810D025
:10FFDC0002D302282CD11AE0164A916893689268D1
:10FFEC0001F0010103F0020343EA8103C2F38062D2
:04FFFC001AE0104AAD
:020000040801F1
:100000009368916803F48073926801F400719B090E
:1000100043EA1123C2F3C0620CE0094A9368916875
:1000200003F48033926801F400319B0B43EA1143DF
:10003000C2F300721343034AD05C70470023FAE70F
:100040000064004088120108012808D002D3022869
:100050000FD109E0074B9A6842F0800208E0054B97
:100060009A6842F4004203E0024B9A6842F40002AC
:100070009A6070470064004018B9044B2022DA608F
:1000800002E0024B20221A61704700BF006400406A
:1000900010B9064BD86805E0012801D0002003E024
:1000A000024B186900F00300704700BF0064004075
:1000B000254B00F11B02120110B5D45804F00404C2
:1000C0000C721CB9D3585B0D0B6002E0D358DB08EF
:1000D0004B6000F11B021C4B1201D35802F180420D
:1000E00003F002034B7202F5C8425468030104F0A6
:1000F0000F0C81F80AC0526803F18043120ACA74D7
:1001000003F5C843D3F8B821CA72D3F8B821120A4C
:100110000A73D3F8B821120C4A73D3F8B821120E1F
:100120008A73D3F8BC21CA73D3F8BC21120A0A74AB
:10013000D3F8BC21120C4A74D3F8BC311B0E8B745B
:10014000FFF79AFF10BD00BF00640040044B1A681F
:1001500042F002021A601868C0F34000704700BF06
:1001600000640040054B1A6822F002021A60186809
:1001700080F00200C0F34000704700BF0064004000
:10018000034B9B6918420CBF00200120704700BF41
:1001900000640040024B9A6922EA00029A617047AB
:1001A00000640040202831D00CD8062820D004D884
:1001B000042825D0052844D118E007281DD0082898
:1001C0003FD11FE0B0F5007F2BD005D840281FD0CD
:1001D000B0F5807F35D11FE0B0F5803F2CD0B0F571
:1001E000003F2BD0B0F5806F2BD11FE0012201E042
:1001F0004FF48072134B9A6023E04FF48032F9E79A
:10020000082200E010220F4BDA601AE0082200E01A
:1002100010220C4B1A6114E00A4B9A6922F0010279
:1002200008E0084B9A6922F0020203E0054B9A6944
:1002300022F004029A6104E0082200E01022014B3F
:100240005A6070470064004001420CBF002001204A
:10025000704700BF202808B532D00CD8062821D01E
:1002600004D8042826D0052818D119E007281ED064
:10027000082813D120E0B0F5007F29D005D8402808
:1002800020D0B0F5807F09D120E0B0F5803F27D0A5
:10029000B0F5003F22D0B0F5806F1BD0002024E0E5
:1002A000012101E04FF48071104B98681BE04FF47E
:1002B0008031F9E7082100E010210C4BD86812E0EA
:1002C000082100E01021094B18690CE0012102E02F
:1002D000022100E00421054B986904E0102100E0B0
:1002E0000821024B5868FFF7AFFF08BD00640040CB
:1002F000012108B54FF00070FEF70AFE4FF00070C4
:100300000021FEF705FE08BD436830B523F47023D5
:100310000C680A7923F48073234343EA0223436081
:1003200082688D68CC680A4B45EA040C02EA030334
:100330004A794CEA030343EA420383600B7CC26AB6
:10034000013B22F47002DBB242EA0353C36230BDC8
:10035000FDF7F1FF002301220274C3600360037103
:1003600043718360704700BF19B1836843F0010394
:1003700002E0836823F001038360704719B183684A
:1003800043F4807302E0836823F4807383607047D2
:10039000C9B212B14368194302E0436823EA01017C
:1003A00041607047836843F008038360704700BF73
:1003B0008068C0F3C0007047836843F00403836023
:1003C000704700BF8068C0F38000704719B1836830
:1003D00043F4A00302E0836823F4A0038360704722
:1003E0008068C0F3805070474368013923F460434C
:1003F00043EA41334360704719B1436843F40063F3
:1004000002E0436823F4006343607047092930B574
:1004100011D94FF0030C0CFB01FC0725ACF11E0CAD
:1004200005FA0CF503FA0CFCC46824EA050343EA58
:100430000C03C3600EE04FF0030C0CFB01FC07251E
:1004400005FA0CF503FA0CFC046924EA050343EAF7
:100450000C030361062A0DD80523013A5A434FF0D5
:100460001F0C0CFA02FC9140436B23EA0C020A4376
:1004700042631CE00C2A0DD805235A434FF01F0C91
:10048000233A0CFA02FC9140036B23EA0C020A4364
:1004900002630CE005235A434FF01F0C413A0CFA5B
:1004A00002FC9140C36A23EA0C020A43C26230BDD7
:1004B00019B1836843F4801302E0836823F4801346
:1004C00083607047C06C80B2704700BF014B1868F2
:1004D000704700BF4C24014019B1436843F4806366
:1004E00002E0436823F480634360704719B14368B6
:1004F00043F4805302E0436823F480534360704721
:10050000836823F4E04341EA03038360704700BF3C
:1005100019B1836843F4004302E0836823F4004385
:100520008360704719B1836843F4021302E0836863
:1005300023F40213836070478068C0F34050704713
:10054000092930B511D94FF0030C0CFB01FC07252C
:10055000ACF11E0C05FA0CF503FA0CFCC46824EA95
:10056000050343EA0C03C3600EE04FF0030C0CFBE1
:1005700001FC072505FA0CF503FA0CFC046924EAD2
:10058000050343EA0C030361836BC3F3015CCCEB0B
:10059000020202324FF0050CD2B20CFB02F20CF157
:1005A0001A0C0CFA02FC914023EA0C030B43836300
:1005B00030BD00BF836B013923F4401343EA01537C
:1005C000836370470A5070472830405880B27047A4
:1005D000436823F4400323F4007341EA03034360B8
:1005E000704700BF41628262704700BF436823F0DA
:1005F0001F0341EA03034360704700BF20B1054B6E
:100600009A6842F4000203E0024B9A6822F4000266
:100610009A60704700240140036819420CBF002013
:1006200001207047C9430160704700BF43680068FC
:1006300010EA112004D0C9B219420CBF00200120D9
:10064000704700BF6FEA11210160704708B5134B76
:1006500098420FD003F5A053984213D0A3F5C0538E
:10066000984219D14FF400700121FEF743FC4FF47A
:1006700000700EE04FF480600121FEF73BFC4FF468
:10068000806006E04FF400400121FEF733FC4FF498
:1006900000400021FEF72EFC08BD00BF00280140ED
:1006A000032A2DE9F0070BD83AB1002311F803C053
:1006B00000F803C001339342F8D1BDE8F00770475A
:1006C00082180C46034603E014F8011C03F8011CD1
:1006D00003F003061946A44601330134002EF3D17A
:1006E0001CF00304634608BFC1EB020C68D06542EE
:1006F000C4F1040A0CEB050733464FEACA0A5CF85A
:1007000005604FEAC408551A08E057F8044F26461A
:1007100004FA0AF449EA0404CC5004335C18032DAB
:1007200026FA08F9A5F104050CEB0306EDDC00231D
:1007300002E0F15CE154013319199142F9D3BCE7AD
:1007400053F8404C41F8404C53F83C4C41F83C4C79
:1007500053F8384C41F8384C53F8344C41F8344C89
:1007600053F8304C41F8304C53F82C4C41F82C4C99
:1007700053F8284C41F8284C53F8244C41F8244CA9
:1007800053F8204C41F8204C53F81C4C41F81C4CB9
:1007900053F8184C41F8184C53F8144C41F8144CC9
:1007A00053F8104C41F8104C53F80C4C41F80C4CD9
:1007B00053F8084C41F8084C53F8044C41F8044CE9
:1007C0001C460D4640334031BCF13F0FACF1400CAC
:1007D000B6DC21462B46541B0FE051F8105C43F861
:1007E000105C51F80C5C43F80C5C51F8085C43F861
:1007F000085C51F8045C43F8045C0F2C0D469C46E1
:1008000001F1100103F11003A4F11004E5DCCCEBBD
:100810000201002303E0EC584CF8034004335E1956
:10082000032903EB0C04A1F10401F4DC7FE700BF12
:1008300080F0004002E000BF81F0004142001FBF95
:100840005FEA410392EA030F7FEA226C7FEA236C9E
:100850006AD04FEA1262D2EB1363C1BFD218414093
:1008600048404140B8BF5B42192B88BF704710F029
:10087000004F40F4000020F07F4018BF404211F0CC
:10088000004F41F4000121F07F4118BF494292EA34
:10089000030F3FD0A2F1010241FA03FC10EB0C0060
:1008A000C3F1200301FA03F100F0004302D54942ED
:1008B00060EB4000B0F5000F13D3B0F1807F06D39A
:1008C00040084FEA310102F10102FE2A51D2B1F192
:1008D000004F40EBC25008BF20F0010040EA030087
:1008E0007047490040EB000010F4000FA2F1010234
:1008F000EDD1B0FA80FCACF1080CB2EB0C0200FABE
:100900000CF0AABF00EBC25052421843BCBFD0400B
:100910001843704792F0000F81F4000106BF80F485
:1009200000000132013BB5E74FEA41037FEA226C48
:1009300018BF7FEA236C21D092EA030F04D092F013
:10094000000F08BF0846704790EA010F1CBF002047
:10095000704712F07F4F04D1400028BF40F00040A4
:10096000704712F100723CBF00F50000704700F0C4
:10097000004343F0FE4040F4000070477FEA2262EB
:1009800016BF08467FEA23630146420206BF5FEABC
:10099000412390EA010F40F4800070474FF00003BC
:1009A00004E000BF10F0004348BF40425FEA000C83
:1009B00008BF704743F0964301464FF000001CE02B
:1009C00050EA010208BF70474FF000030AE000BF81
:1009D00050EA010208BF704711F0004302D54042BF
:1009E00061EB41015FEA010C02BF84460146002031
:1009F00043F0B64308BFA3F18053A3F50003BCFA4C
:100A00008CF2083AA3EBC25310DB01FA02FC6344F8
:100A100000FA02FCC2F12002BCF1004F20FA02F2FF
:100A200043EB020008BF20F00100704702F12002F2
:100A300001FA02FCC2F1200250EA4C0021FA02F253
:100A400043EB020008BF20EADC7070474FF0FF0C58
:100A50001CEAD0521EBF1CEAD15392EA0C0F93EA53
:100A60000C0F6FD01A4480EA010C400218BF5FEAF5
:100A700041211ED04FF0006343EA501043EA511168
:100A8000A0FB01310CF00040B1F5000F3EBF490062
:100A900041EAD3715B0040EA010062F17F02FD2A66
:100AA0001DD8B3F1004F40EBC25008BF20F0010049
:100AB000704790F0000F0CF0004C08BF49024CEA60
:100AC000502040EA51207F3AC2BFD2F1FF0340EAF2
:100AD000C250704740F400004FF00003013A5DDC63
:100AE00012F1190FDCBF00F000407047C2F10002A4
:100AF000410021FA02F1C2F1200200FA02FC5FEA91
:100B0000310040F1000053EA4C0308BF20EADC70DA
:100B1000704792F0000F00F0004C02BF400010F44C
:100B2000000F013AF9D040EA0C0093F0000F01F0F9
:100B3000004C02BF490011F4000F013BF9D041EA1B
:100B40000C018FE70CEAD15392EA0C0F18BF93EA1D
:100B50000C0F0AD030F0004C18BF31F0004CD8D147
:100B600080EA010000F00040704790F0000F17BFCE
:100B700090F0004F084691F0000F91F0004F14D014
:100B800092EA0C0F01D142020FD193EA0C0F03D16C
:100B90004B0218BF084608D180EA010000F000406F
:100BA00040F0FE4040F40000704740F0FE4040F44A
:100BB000400070474FF0FF0C1CEAD0521EBF1CEAE9
:100BC000D15392EA0C0F93EA0C0F69D0A2EB030207
:100BD00080EA010C49024FEA402037D04FF08053A1
:100BE00043EA111143EA10130CF000408B4238BF66
:100BF0005B0042F17D024FF4000C8B4224BF5B1A74
:100C000040EA0C00B3EB510F24BFA3EB510340EAC1
:100C10005C00B3EB910F24BFA3EB910340EA9C006F
:100C2000B3EBD10F24BFA3EBD10340EADC001B01DF
:100C300018BF5FEA1C1CE0D1FD2A3FF650AF8B4283
:100C400040EBC25008BF20F0010070470CF0004C90
:100C50004CEA50207F32C2BFD2F1FF0340EAC250BB
:100C6000704740F400004FF00003013A37E792F07C
:100C7000000F00F0004C02BF400010F4000F013ADA
:100C8000F9D040EA0C0093F0000F01F0004C02BFD5
:100C9000490011F4000F013BF9D041EA0C0195E73E
:100CA0000CEAD15392EA0C0F08D142027FF47DAFD7
:100CB00093EA0C0F7FF470AF084676E793EA0C0FC7
:100CC00004D14B023FF44CAF08466EE730F0004CC5
:100CD00018BF31F0004CCAD130F000427FF45CAF55
:100CE00031F000437FF43CAF5FE700BF4FF0FF3CC3
:100CF00006E000BF4FF0010C02E000BF4FF0010C16
:100D00004DF804CD4FEA40024FEA41037FEA226CDE
:100D100018BF7FEA236C11D001B052EA530C18BF00
:100D200090EA010F58BFB2EB030088BFC81738BF65
:100D30006FEAE17018BF40F0010070477FEA226C53
:100D400002D15FEA402C05D17FEA236CE4D15FEA4F
:100D5000412CE1D05DF8040B704700BF8446084683
:100D60006146FFE70FB5FFF7C9FF002848BF10F144
:100D7000000F0FBD4DF808EDFFF7F4FF0CBF012089
:100D800000205DF808FB00BF4DF808EDFFF7EAFF13
:100D900034BF012000205DF808FB00BF4DF808EDCE
:100DA000FFF7E0FF94BF012000205DF808FB00BFC3
:100DB0004DF808EDFFF7D2FF94BF012000205DF849
:100DC00008FB00BF4DF808EDFFF7C8FF34BF012056
:100DD00000205DF808FB00BF4FEA4002B2F1FE4F71
:100DE0000FD34FF09E03B3EB12620DD94FEA0023ED
:100DF00043F0004310F0004F23FA02F018BF4042C6
:100E000070474FF00000704712F1610F01D14202AC
:100E100005D110F0004008BF6FF0004070474FF060
:100E20000000704754004D0043004D002D0031007C
:100E30003600330030002000280076006900720080
:100E40007400750061006C00200043004F004D00ED
:100E50002900200054004D0043004D0031003600B1
:100E60003300000000000000000000000902430001
:100E7000020100C032090400000102020100052441
:100E800000100105240100010424020205240600CB
:100E900001070582030800FF09040100020A00009F
:100EA0000007050302400000070581024000000022
:100EB0000403090426035400720069006E006100F7
:100EC0006D00690063004D006F00740069006F00E1
:100ED0006E002000430074006C0000005515AC6AE1
:100EE000004001C0ABEA57956B7FD87EB87DA07CEF
:100EF0008F7B857A827985780878147726763D7598
:100F000059747B73A172367264719670CC6F076FDF
:100F1000456EE66D2A6D726CBE6B0D6B5F6AB569CE
:100F20006169BB6819687967DC664266AB656065B4
:100F3000CC643B64AD63206396620F62CB61476112
:100F4000C4604460C65F495FCE5E925E1A5EA45D77
:100F50002F5DBD5C4B5CDC5BA55B385BCC5A625A99
:100F6000F95992592C59F95895583358D157715706
:100F70001257B4560000C90092015B022403ED032E
:100F8000B6047F0548061107D907A2086A09330A83
:100F9000FB0AC40B8C0C540D1C0EE30EAB0F72102D
:100FA0003A110112C8128F1355141C15E215A81618
:100FB0006E173318F918BE19821A471B0B1CCF1C69
:100FC000931D571E1A1FDD1F9F2061212322E5223A
:100FD000A62367242825E825A82667272628E528AC
:100FE000A329612A1F2BDC2B992C552D112ECC2ED9
:100FF000872F4130FB30B5316E322633DF339634E4
:101000004D350436BA366F372438D9388C39403AE2
:10101000F23AA53B563C073DB83D683E173FC53FF9
:1010200073402141CE417A422543D0437A4424453E
:10103000CD4575461C47C34769480F49B449584ACE
:10104000FB4A9D4B3F4CE04C814D204EBF4E5D4FC7
:10105000FB4F97503351CE51685202539B53325439
:10106000C9546055F5558A561D57B0574258D35844
:101070006459F359825A0F5B9C5B285CB35C3E5DFC
:10108000C75D4F5ED75E5D5FE35F6860EB606E617A
:10109000F0617162F1627063EE636C64E8646365D1
:1010A000DD655666CF664667BC673268A668196913
:1010B0008B69FD696D6ADC6A4A6BB76B236C8E6C59
:1010C000F86C616DC96D306E966EFB6E5E6FC16FB0
:1010D00022708370E27040719D71F9715472AE722A
:1010E00007735E73B5730A745F74B27404755575D3
:1010F000A575F37541768D76D87622776B77B377C1
:10110000FA773F788478C77809794A798979C879F4
:10111000057A417A7C7AB67AEE7A267B5C7B917B83
:10112000C57BF87B297C597C887CB67CE37C0E7D72
:10113000397D627D897DB07DD57DFA7D1D7E3E7EC7
:101140005F7E7E7E9C7EB97ED57EEF7E097F217F8D
:10115000377F4D7F617F747F867F977FA67FB47FC7
:10116000C17FCD7FD87FE17FE97FF07FF57FF97F79
:10117000FD7FFE7F0010161B2023272A2D303235DD
:1011800037393B3D4041434547494B4C4E50515305
:10119000545657595A5B5D5E606162636566676865
:1011A0006A6B6C6D6E707172737475767778797A1C
:1011B0007B7C7D7E80808182838485868788898A06
:1011C0008B8C8D8E8F909091929394959696979804
:1011D000999A9B9B9C9D9E9FA0A0A1A2A3A3A4A51E
:1011E000A6A7A7A8A9AAAAABACADADAEAFB0B0B147
:1011F000B2B2B3B4B5B5B6B7B7B8B9B9BABBBBBC80
:10120000BDBDBEBFC0C0C1C1C2C3C3C4C5C5C6C7C2
:10121000C7C8C9C9CACBCBCCCCCDCECECFD0D0D10C
:10122000D1D2D3D3D4D4D5D6D6D7D7D8D9D9DADA60
:10123000DBDBDCDDDDDEDEDFE0E0E1E1E2E2E3E3BB
:10124000E4E5E5E6E6E7E7E8E8E9EAEAEBEBECEC1B
:10125000EDEDEEEEEFF0F0F1F1F2F2F3F3F4F4F580
:10126000F5F6F6F7F7F8F8F9F9FAFAFBFBFCFCFDEE
:10127000FDFEFEFF00000000010203040102030462
:101280000607080902040608020000000000000129
:0C12900031363330563230370000000099
:10129C00CE00000040000000FB070000FF0700002C
:1012AC000008000014000000010000000500000010
:1012BC0006000000901201080B0C0D0A0E08090024
:1012CC000100000002000000030000000400000008
:1012DC000008004001000000000400400101010171
:1012EC000101010001000000A000000000127A00C2
:1012FC000048004000C2010000000800B00E0108C8
:10130C0004000000B40E010826000000E0000020DC
:10131C0032000000140100201A0000006C0E0108BD
:10132C0043000000CC00002012000000C194000813
:10133C00C592000811910008259100082991000818
:10134C0089910008AD910008B5920008A59200089B
:10135C008192000800000000400000001201100102
:10136C0002000040D0160000020701020301000039
:10137C00320354004D0043004D002D00300030006E
:10138C0030003000200028007600690072007400E4
:10139C00750061006C00200043004F004D002900D7
:1013AC00200000001A0354004D0043004D00300093
:1013BC003000300030000000000000000000000091
:1013CC001190000879D3000879D3000879D300086C
:1013DC0079D3000879D3000879D3000879D30008B1
:1013EC0079D300081594000879D3000879D3000844
:1013FC0079D3000879D300080401000079D30008E0
:10140C00ED90000879D3000879D3000879D300084F
:10141C0079D3000879D3000879D300080591000826
:0C142C00010000000100000001000000B1
:040000050800410CA2
:00000001FF
